:020000040000FA
:100000005805002085160000DD1600001D100000B8
:100010001D1000001D1000001D1000001D1000002C
:100020001D1000001D1000001D100000E10F000059
:100030001D1000001D1000009D0F00001D1000008D
:10004000411000004110000041100000411000006C
:10005000411000004110000041100000411000005C
:10006000411000004110000041100000411000004C
:10007000411000004110000041100000411000003C
:10008000411000004110000041100000411000002C
:10009000411000004110000041100000411000001C
:1000A000411000004110000041100000411000000C
:1000B00041100000411000004110000041100000FC
:1000C00041100000411000004110000041100000EC
:1000D00041100000411000004110000041100000DC
:1000E00041100000411000004110000041100000CC
:1000F00041100000411000004110000041100000BC
:1001000041100000411000004110000041100000AB
:10011000411000004110000041100000411000009B
:10012000411000004110000041100000411000008B
:10013000411000004110000041100000411000007B
:10014000411000002DE9E04F2746A046A146A246F7
:10015000A346A446A2B02DEC000A84F300882546ED
:100160002646A4473DEC000A22B0BDE8E08F00001F
:100170007BB972B90029BEBF00204FF0004106E0F4
:1001800008BF00281CBF6FF000414FF0FF3000F0A7
:10019000AFB9ADF1080C6DE904CE002909DB002BE5
:1001A0001ADB00F035F8DDF804E0DDE9022304B0E5
:1001B0007047404261EB4101002B1BDB00F028F847
:1001C000DDF804E0DDE9022304B0404261EB4101C7
:1001D000524263EB43037047524263EB430300F028
:1001E00017F8DDF804E0DDE9022304B0404261EBDA
:1001F00041017047524263EB430300F009F8DDF818
:1002000004E0DDE9022304B0524263EB430370478C
:100210002DE9F0478C46089D04468A46002B4AD1BA
:100220008A42174662D9B2FA82F64EB1C6F1200E62
:1002300001FA06F3B740B44020FA0EFE4EEA030A74
:100240004FEA1748230C1FFA87F9BAFBF8FE08FBA0
:100250001EAA0EFB09F243EA0A439A420BD9FB1885
:100260000EF1FF312CBF012000209A4202D9002854
:1002700000F02A818E469A1AA3B2B2FBF8F008FB6E
:10028000102200FB09F943EA0244A14507D93C19B1
:1002900000F1FF3302D2A14500F210811846A4EB11
:1002A000090440EA0E4000211DB1F4400023C5E9D5
:1002B0000043BDE8F0878B4208D9002D00F0F280A2
:1002C0000021C5E9000C0846BDE8F087B3FA83F1C8
:1002D00000294ED16345C0F0E880824240F2E580BB
:1002E0000846002DE5D0C5E9004AE2E702B9FFDE85
:1002F000B2FA82F6002E40F099808B1A4FEA124E25
:100300001FFA82F801214FEA144CB3FBFEF20EFBF8
:10031000123008FB02F94CEA004CE14508D917EB12
:100320000C0C02F1FF3302D2E14500F2CA801A46FA
:10033000ACEB090CA3B2BCFBFEF00EFB10CC08FB2F
:1003400000F843EA0C44A0450ED93C1900F1FF33F4
:100350002CBF4FF0010C4FF0000CA04503D9BCF1AD
:10036000000F00F0A8801846A4EB080440EA024001
:100370009AE7C1F120048B4002FA01FE0CFA01F663
:10038000E24020FA04F72CFA04FC00FA01F81343C7
:100390003E431F0C320C1FFA83F9BCFBF7F007FB3E
:1003A00010CC00FB09FA42EA0C4CE24508D913EBE9
:1003B0000C0C00F1FF3202D2E24500F289801046B7
:1003C000ACEB0A0CB6B2BCFBF7FA07FB1ACC0AFB83
:1003D00009F946EA0C42914506D99A180AF1FF3606
:1003E00001D291457AD8B2464AEA0040A2EB09020E
:1003F000A0FB0E67BA42B446B94602D307D1B04556
:1004000005D2B6EB0E0C67EB030301389946002DBD
:100410006BD0B8EB0C0362EB090202FA04F4CB4098
:10042000CA4000211C43C5E9004242E7B740C6F17B
:10043000200201FA06F3B44021FA02FC4FEA174EFB
:1004400020FA02F21FFA87F8BCFBFEF11A430EFBFA
:1004500011CC01FB08F0130C43EA0C4C604507D9A2
:1004600017EB0C0C01F1FF3301D2604533D819466C
:10047000ACEB000C92B2BCFBFEF00EFB10CC00FB10
:1004800008F342EA0C4C634507D917EB0C0C00F15A
:10049000FF3201D2634525D81046ACEB030340EA96
:1004A000014130E72946284603E7841A6CEB030331
:1004B00001209A4615E702383C4455E702383C448F
:1004C000EDE6023ABC4433E7AEF1020E3B44D2E61D
:1004D00002389C4474E70239BC44C9E7AAF1020A15
:1004E0001A4481E70238BC44D7E72946E1E600BF59
:1004F000704700BF830003F1A04303F54053D3F8D6
:10050000002810B4002A1BDAD3F8002802F00302F6
:10051000022A05D0D3F8002802F00302032A0FD1E3
:10052000012100F01F04A1404209074C203244F889
:100530002210BFF34F8FBFF36F8F044AC3F8002818
:10054000002110BC00F0C6BF00E100E00001008007
:100550008FB5564800F0D4FA002440F21717544ED5
:10056000544D04F5C073214646F8237028460134E3
:1005700000F0C6FA082CF4D140F207174C4E4E4D4D
:1005800004F5C073214646F823702846013400F074
:10059000B7FA202CF4D1494800F0B2FA002440F216
:1005A0001717434E464D04F5E073214646F8237075
:1005B0002846013400F0A4FA082CF4D140F20717C1
:1005C0003B4D404E04F5E073214645F8237030461C
:1005D000013400F095FA202CF4D100243A4800F0C0
:1005E0008FFAC5F8C0444FF480250520FFF782FF3D
:1005F0001520FFF77FFF2A20FFF77CFF3920FFF748
:1006000079FF3A20FFF776FF4220FFF773FF312092
:10061000FFF770FF0920FFF76DFF1C20FFF76AFF4F
:100620001D20FFF767FF2C20FFF764FF0A20FFF76C
:1006300061FF0B20FFF75EFF2968244800F060FA95
:1006400010222146684601F0D3F82B6868460093D3
:10065000029500F041F8012000F06EF8204600F00D
:1006600057F8204600F07CF80121204600F08CF875
:10067000174A1848D2F88C3043F44063C2F88C30E3
:100680004FF004131C6800F03BFA0820FFF732FF1C
:1006900024F00104BFF34F8FBFF36F8F6408640031
:1006A0002046214622462346FFF74CFDFC28000049
:1006B000003000501A290000452900007A29000066
:1006C00097290000C7290000FB2900001F2A00000D
:1006D00000ED00E0372A000082680C4B9A60036846
:1006E00083F38888436883F38988027B02F00101E1
:1006F000EFF3948323F00303920748BF43F0020310
:1007000009B143F0010383F39488704700ED02E0E0
:10071000084AD36848B123F400531B041B0C43F070
:10072000BF6343F40033D36070479BB243F400537C
:10073000F5E700BF00ED00E0084AD36840B19BB286
:1007400043F4804343F0BF6343F40033D360704706
:1007500023F480431B041B0CF4E700BF00ED00E012
:10076000084AD36840B19BB243F0080343F0BF632B
:1007700043F40033D360704723F008031B041B0CC1
:10078000F4E700BF00ED00E0084B1A6818B142F032
:1007900001021A60704722F001021A601A6811B152
:1007A00042F00202F5E722F00202F2E7D0ED00E0AB
:1007B00008B50446084611461A46A04701F070FDE8
:1007C00000F03CFF002070470B6801330B60014BC9
:1007D0001B681847980E00202DE9F04F85B00E9C3D
:1007E0009B46012CB8BF0124012B0CBF30232023D2
:1007F00015468046894601260A270022DFF870A0A8
:10080000019402930AF101040AB9AA451ED2B5FB6C
:10081000F4F049463030C04701220136B5FBF4F10F
:100820000A23013F012F04FB1155BAFBF3FAE9D16A
:10083000494605F13000C047BBF1030F03D1019BCE
:100840009C1B002C0FDC05B0BDE8F08F019BBB4268
:10085000E4DBBBF1020FE1D849460298039201366E
:10086000C047039ADAE749462020C047013CE8E741
:10087000FFC99A3B014B1860704700BF980E0020DB
:100880002DE9F04F4FF0000A06460F464FF0FF39B2
:10089000D04689B01C46531E0493002505E06DB96F
:1008A000252800F011813946B047049B13F8010F49
:1008B00004930028F3D109B0BDE8F08F642861D01B
:1008C00019D839280AD8312850D22D283CD03028C0
:1008D0003DD0252808D13946B047DEE7582800F03A
:1008E0008880632800F0EA8039462520B047049BC1
:1008F00039461878F0E7702871D006D8692841D0B9
:100900006C283CD06828D0D0EEE7752857D017D88F
:100910007328E9D1236804F1040B1C46254615F819
:10092000010B002840F0BF80B8F1030F40F0D580E4
:10093000E41AA9EB0404002C00F3BB805C46ACE78E
:10094000782856D07A28DEE74FF00308ADE7B9F1F2
:10095000000F0EDAB8F1000F00F0BC80A0F13009F2
:10096000B8F1000F08BF4FF002089EE7B9F1000F81
:10097000F4DB0A2303FB0909A9F13009F0E70AF1C6
:10098000010A92E7BAF1010FC5BF073424F007034B
:1009900025681D68D4BF043403F10804002D05DA6E
:1009A00039462D20B0476D4209F1FF3943462A46AA
:1009B000CDF8009039463046FFF70EFF6DE7BAF1EB
:1009C000010FC5BF073424F0070322681A68CCBFA3
:1009D00003F108040434CDF800904346EAE73946B1
:1009E0003020B04739467820B0474FF008094FF023
:1009F00001080822BAF1010FC5BF073424F007032C
:100A0000236803F10804CABF1B68059305934FF0E0
:100A100000039346D8BF0434039307930BF1FF3BC5
:100A2000059B4FEA8B0023FA00F010F00F0009D16C
:100A3000079B13B9BBF1000F24D14FF0300C07E036
:100A4000069AEBE709288CBF4FF0570C4FF0300C9B
:100A5000394660440692B047039B079501330393E0
:100A6000BBF1000FECD1B8F1030F7FF416AF039B7D
:100A7000C3EB4905002D7FF710AF39462020B04762
:100A8000013DF7E7531E91450693E9DBB8F1010FED
:100A900003D139463020B047E2E7B8F1020FDFD189
:100AA00039462020F7E7394603932C46B047039B8D
:100AB00034E739462020B047013C3CE72068251D3B
:100AC0003946B0472C46E8E6AA46A8464FF0FF391B
:100AD0000125EAE64FF00108E7E65C460546E4E654
:100AE000002313B502AC44F8043D02460B4603480C
:100AF0002146FFF7C5FE02B010BD00BFC9070000C8
:100B00000FB407B504A951F8040B0191FFF7E8FFF2
:100B100003B05DF804EB04B07047704710B54FF0B8
:100B20002003EFF3118483F3118800F011F8012200
:100B3000054BC3F840254FF0FF32044B9A62DA624E
:100B400084F31188002010BD0090035000ED00E0F8
:100B50001B4A136843F0020313601A4BDB69DB077F
:100B60002AD5194B1946D3F80024012AFBD1C3F822
:100B70000425D1F80034012BFBD1124AD36923F0AC
:100B80000103D361104B1A46D3F800140129FBD19D
:100B90000021C3F80415D2F80034012BFBD1BFF3B8
:100BA0004F8F0A490A4BCA6802F4E0621343CB60D4
:100BB000BFF34F8F00BFFDE7064B074A1A6070472F
:100BC000D0ED00E00080FF000090035000ED00E059
:100BD0000400FA059C0E00200090D0030A2838B5C6
:100BE0000446074D04D128680D2143685B68984787
:100BF0002868E1B243685B689847204638BD00BF6B
:100C0000000000200148FFF735BE00BFDD0B0000EB
:100C100008B5044801F0D2F8034B1860FFF7F2FF63
:100C2000002008BDA32A00000000002010B54FF0EE
:100C30002003EFF3118283F31188114C237823B939
:100C400082F311886FF0440010BD013BDBB22370CA
:100C500023B182F311886FF00F00F5E7094B0121F2
:100C6000187828B1217082F311886FF00A00EBE741
:100C7000197082F31188044A11601870E4E700BF0C
:100C800006000020050000200450005010B54FF071
:100C90002003EFF3118283F31188104C207888B180
:100CA00082F311884FF05022D2F81C34D2F8182465
:100CB00003F0030343F48033934314BF6FF0430006
:100CC000002010BD0123237082F311884FF05022C1
:100CD000C2F80401C2F818159360E3E7040000208D
:100CE0004FF0502330B5D3F80851D3F80423D3F88C
:100CF000004102F00102D3F80413D3F8040115B146
:100D00000025C3F80851B4B14FF050230024C3F8B4
:100D1000004122B14FF050230122C3F8082348B10B
:100D200000224FF05023C3F804218A0702D5022283
:100D3000C3F8082330BD002AF1D04FF05023D3F878
:100D40000C3403F00113B3F1011FE8D1E2E708B559
:100D500000220121052000F0A3FB052000F07CFB10
:100D6000002008BDF8B54FF02002EFF3118382F3A5
:100D70001188264A1078441C147070B183F31188CE
:100D80004FF05023D3F80C3403F00113B3F1011FDB
:100D90000CBF00206FF0430007E01D4D2F782FB1EE
:100DA000107083F311886FF00A00F8BD01262E70D1
:100DB00083F311884FF0502421B3052000F05CFB31
:100DC000C4F80071D4F80433C4F804632660D4F87E
:100DD00000219AB10022DB0758BF0123C4F800218B
:100DE0004FF0200258BFC4F808330A4B0520C3F85F
:100DF000802100F031FB00232B70C1E720BF40BFF2
:100E000020BFE4E7C4F800112660F4E706000020E4
:100E10000500002000E100E070474FF02003EFF3F1
:100E2000118083F31188704700230D4A10B5C2F872
:100E30004031FFF7F2FFD2F8043540F2471209497A
:100E40000C681B1B23F07F43B3FBF2F302FB03424E
:100E50000A6080F311881846BDE8104001F0B6BB67
:100E6000005001500800002038B51B4800F0A6FFD4
:100E700070B3436801211B689847002440F2471370
:100E8000164D4FF40012C5F80845C5F840354FF42B
:100E90008033C5F84433C5F80433114B01211C607D
:100EA000104B1520C3F88021224600F0F9FA1520D6
:100EB00000F0D2FA012320460B4A13602B60D5F8CC
:100EC000043503F2471323F07F43C5F8403538BD9E
:100ED0004FF0FF30FBE700BFC42A00000050015074
:100EE0004051015000E100E00850015070B54CF64F
:100EF0006905B0F1FF3F14BF02462A46FFF78DFF98
:100F0000114B12491E68531EAB42A8BF2B4640F23C
:100F10004715D1F8044523EAE373A21B22F07F4270
:100F200002F5A37205FB0323B3FBF5F305FB036393
:100F30001C1B1F2C98BF5B1923F07F43C1F8403561
:100F400080F3118870BD00BF0800002000500150E0
:100F500008B5FFF762FF084B084AD3F8043512685A
:100F60009B1A40F2471223F07F43B3FBF2F380F366
:100F70001188184608BD00BF00500150080000202D
:100F800004488168406A884203D003494FF0805288
:100F90000A6070472801002004ED00E0202080F363
:100FA00011880D498A684FF028001044EFF3098C2E
:100FB00080E8F01F094F4FF000664A6A8A603E6081
:100FC000506E0023536680F3118802F1280090E8E8
:100FD000F01F8CF3098870472801002004ED00E021
:100FE0001EF0040F0CBFEFF30880EFF30980816956
:100FF00031F8021C11F0FF010229FFD000B500F00A
:10100000EDFA00BD014910220A60704710ED00E0C2
:10101000404080F3118830BF704700BF404080F3EC
:1010200011884FF004007146014202D0EFF30980AD
:1010300001D1EFF30880714600B500F06FF900BDF3
:1010400000B572B60B4A106A00281EBF002111625B
:1010500000F0DAFE62B6EFF30580A0F110004FEA6F
:10106000C0000549014409C998475DF804EB0348ED
:10107000004700002801002094260000810F000096
:10108000002320210348C2180133412B82F80013AA
:10109000F9D1704700E100E0084A094993680968FE
:1010A0005866996607494B6843F080534B600023AC
:1010B00083F311889368986E704700BF2801002061
:1010C0008830000000ED00E038B5194C054619489D
:1010D000FFF716FDA36AD90602D51748FFF710FDE2
:1010E000A36A1A0702D51548FFF70AFDA36A9B07F2
:1010F0000ED51348FFF704FD616BA36A180607D5E8
:101100001048FFF7FDFC1DB1A36A23F08003A36222
:10111000074CA26AD20702D50B48FFF7F1FCA36A7D
:101120009B0602D50948FFF7EBFC002038BD00BF45
:1011300000ED00E0782C00008F2C0000A12C0000B6
:10114000B52C0000CE2C0000E52C0000052D000081
:1011500038B51E4C05461E48FFF7D2FCA36AD804DA
:1011600009D51C48FFF7CCFC184A0020936A43F4C9
:101170007F43936238BDA36A190501D51648F1E78C
:10118000A36A9A0514D51548FFF7BAFCA16BA36AA8
:101190001B0407D51248FFF7B3FC1DB1A36A23F463
:1011A0000043A362094B9B6A5805DDD50D48D9E77A
:1011B000A36A5905FAD4A36ADA0501D50A48D1E72A
:1011C000A36A9B04D0D50948CCE700BF00ED00E03E
:1011D000E42A00008F2C0000A12C0000FB2A000054
:1011E000152B00002B2B0000472B0000052D0000C5
:1011F00010B51C4C1C48FFF783FCA36A9A0102D56A
:101200001A48FFF77DFCA36ADB0102D51848FFF7F7
:1012100077FCA36ADC0202D51648FFF771FC114C7B
:10122000A36A180302D51448FFF76AFCA36A59039E
:1012300002D51248FFF764FCA36A9A0302D510484E
:10124000FFF75EFC074CA36ADB0302D50D48FFF7EE
:1012500057FCA36A00206FEA03436FEA1343A362BB
:1012600010BD00BF00ED00E0152E00002E2E000086
:10127000422E00005D2E00006F2E00008E2E00001A
:10128000B42E0000CF2E000010B51A4C1A48FFF7FC
:1012900037FCA1696369580602D51848FFF730FC8E
:1012A0006369D90707D51648FFF72AFC636943F03D
:1012B000FF03636110BD63699A0701D51148F3E725
:1012C00063695B0701D51048EEE76369180701D52C
:1012D0000E48E9E76369D90601D50D48E4E763697B
:1012E0009A0601D50B48DFE763691B06DED50A487D
:1012F000DAE700BFD0ED00E0352D00004F2D0000F3
:10130000602D0000772D0000962D0000B22D00000A
:10131000D02D0000E62D0000012E00003B4B70B5E3
:101320005D6801F07F43B3F17F4F04460E4618D14C
:10133000CA0716D54B061FD40168354B0B44012B49
:1013400098BF016C3348FFF7DBFB16F0080F2F4BFB
:101350000DD0EFF389845B6818050DD42E48FFF794
:10136000CFFB2146BDE87040002000F005B9EFF347
:1013700088845B681905F1D4C5F30805EA1E092ABB
:1013800039D8DFE802F0053234282F3838383836BB
:101390002248FFF7B5FB1D4BDA6A920701D52048BA
:1013A000DDE7DB6A5B00DCD51E48FFF7A9FB1E4BBF
:1013B0001B782BB10120FFF787FE0628D1D170BD25
:1013C0001A4B1B781BB10120FFF7C2FEF5E7184B43
:1013D0001B889BB213B1FFF70BFFEEE7154B5B6960
:1013E000002BBED0FFF750FFBBE70020E3E7002053
:1013F000EAE71148B3E711481149A5F110020F2D92
:10140000D8BF01460F48FFF77BFBAAE700ED00E0DD
:10141000A6ED05018E2B0000AE2B0000D32B0000A3
:10142000EB2B00000D2C000028ED00E029ED00E082
:101430002AED00E0D0ED00E02D2C0000602B000034
:10144000752B0000642C0000024A536943F010031E
:101450005361704700ED00E043B2002B08DB01222E
:1014600000F01F0002FA00F0024A5B0942F8230074
:10147000704700BF00E100E043B2002B0DDB01220A
:1014800000F01F0002FA00F05B09044A203342F822
:101490002300BFF34F8FBFF36F8F704700E100E071
:1014A00043B2002B01F10101A8BF03F160434FEAF1
:1014B0004111B8BF054BC9B2ABBF03F5614300F0A2
:1014C0000F0083F800131954704700BF14ED00E0BB
:1014D000FFF7A4BD43B2A9B1002B12DB01215B09C8
:1014E0009B0003F1604303F56143D3F8802200F0D1
:1014F0001F0001FA00F022EA0000C3F88002D3F8CE
:1015000080327047002BFCDB01225B099B0003F15A
:10151000604303F56143D3F8801200F01F0002FA24
:1015200000F00843E9E70000F8B516460C461F46F0
:1015300004220A9B0999054600F09CFF0023A6F1AE
:1015400020010C4A214421F0070122F00102C5E9E3
:101550001333C5E916468A61069A0F604A60079AF6
:101560008A60089ACA604FF08072CA61A9646B668B
:10157000F8BD00BFB107000038B504460D46052888
:101580001AD8DFE800F00319191315170D48FFF7F3
:10159000B7FA00F085FEAA6901460B48FFF7B0FADA
:1015A00029462046BDE8384000F01CB80748EEE761
:1015B0000748ECE70748EAE701460748FFF7A0FAC3
:1015C000E7E700BFFB2E0000992F00001B2F000053
:1015D000412F00005B2F0000762F000001460068BD
:1015E000FFF7CABF052810B50CD000F08BFE60B124
:1015F00000F088FE0C490D4B002808BF19460C4826
:10160000FFF77EFAFFF704FDFCE700F08BFE0028F1
:10161000EED1084C0848A168FFF772FAA068BDE84F
:10162000104000F00BB800BFD52F0000D92F0000EC
:10163000EA2F0000280100200A30000038B50546D6
:101640004FF02003EFF3118483F3118800F0A4FE20
:101650000A4B9B68AB420BD1094B5A68C2F3080294
:1016600012B92046FFF718FD5A6842F080525A60BE
:101670002046BDE8384000F037BD00BF28010020FB
:1016800000ED00E0202080F3118806484FF400614F
:10169000401880F30988022080F31488BFF36F8F0D
:1016A00000F006F89806002030BFFFF7FDBF00BF2E
:1016B00008B5084B084A23F07F039360BFF34F8FB0
:1016C000BFF36F8F00F0BAFB00F0C2FBFFF7D8FC4E
:1016D00000F0E2FB0000000000ED00E008B5FFF7BD
:1016E000E3FFBDE80840FFF74BBC00000522034BB9
:1016F0005A60BFF34F8FBFF36F8F704790ED00E0DC
:10170000BFF35F8F0022014B5A60704790ED00E0FD
:10171000184919480B6870B50468C3F307239C4245
:1017200025D8FFF7EDFF4FF6AA73426800200B6340
:10173000844202F1100603D1FFF7D8FF002070BDEC
:10174000157A56F8103C05F01F0223F01F031A43C8
:1017500056F8043C6D0923F01F0343F0010343EAEC
:1017600045038860CA6001300B613246E0E74FF004
:10177000FF30E4E790ED00E06C2A00000138013909
:1017800010F8013F11F8012F934202D1002BF7D13D
:101790001A46981A7047F0B581EA0004A507034677
:1017A0000BD0013B0A4491421DD1F0BD002AFCD070
:1017B00011F8014B013A03F8014B9C07F6D10C4696
:1017C0001D1F8F183E1B032E08D86FF003059408C9
:1017D00005FB0422A40023442144E2E754F8046BEF
:1017E00045F8046FEEE711F8014B03F8014FDAE713
:1017F0000346F0B5C9B29C070FD11D4641EA01244A
:1018000044EA04449F187E1B032E0CD8940803EB73
:10181000840413449C4209D1F0BD002AFCD003F893
:10182000011B013AE7E745F8044BECE704F8011B1C
:10183000F0E710B504688068A46801292468C069CD
:1018400003D158406060002010BD00334FF001010B
:1018500018BF0123D04000F001009140834214BF23
:10186000A160E160EFE770B504688068A468C069B2
:10187000256801296E692C696D6880EA040084EA94
:10188000050404EA060480EA04001CBFD04000F00E
:1018900001001860002070BD8368186872B108608C
:1018A0005A68196002B95960002070471060586882
:1018B000814208BF5A600DE0024600680028F3D05C
:1018C0008842F9D10868002AF0D15A68186091421C
:1018D00000D1586000230B60E6E7000008B5094B13
:1018E0001A786AB901210D2019700521FFF7D8FD7A
:1018F0000D20FFF7B1FD4FF00042034BC3F8042366
:10190000002008BD0C00002000D000500A4A10B58D
:1019100093681268926812681469D3E9052111432B
:10192000D3E902020240D8691B6922EA0102584049
:10193000604022EA000010BDFC0E0020F8B51F4EEA
:101940003368012B30D1FFF7E1FF05460023012763
:101950009C461B4CD4F8042307FA03F1114211D022
:1019600003F1A05202F5515292001168012909D1E8
:1019700003F5A27054F82000C2F800C0C0F30420A0
:1019800081400D430133082BE4D17DB10D4FBB687D
:101990001C685CB1A3681D4204D063682A462146D6
:1019A000384698472468F4E70025CFE73368012BD1
:1019B00003D1FFF7ABFF00B93060F8BD7CD1005018
:1019C00000D00050FC0E0020F0B50368554D9B6818
:1019D00084681A7901F01F0343EA42130022D5F804
:1019E0000403C0B202F5A27655F82660C6F30426B9
:1019F000B34270D120FA02F6F6076CD5900000F1E0
:101A0000A04000F55040D0F8106526F00106C0F85F
:101A10001065012000FA02F2C5F80823424A02EBE1
:101A20008302D2F8000220F44030C2F80002D2F85B
:101A30000002C2F80002A068C84010F0010049D0BE
:101A4000E068C84010F0010044D06069C84010F060
:101A500001004CD0A269CA40D20740D4226922FAC0
:101A600001F0E26922FA01F101F0010100F0010246
:101A70008A420CBF0221012100252A4E05F5A272DF
:101A800056F8220010F003002BD1AA0002F1A04268
:101A900002F55047D7F810451B0224F4473424F4CC
:101AA0004074C7F81045D7F8104503F4F85343EADB
:101AB0000141214302F55142C7F810151060D7F8D3
:101AC000103543F00103C7F81035012303FA05F57B
:101AD000C6F80453F0BD0132082A83D19EE70321E2
:101AE000CAE70135082DC9D16FF01200F2E723696A
:101AF000E469CB4024FA01F103F0010301F0010194
:101B00008B420CBF4FF440334FF40033D2F8004205
:101B100024F44034C2F80042D2F800422343C2F811
:101B20000032D7E700D00050002584502DE9F74F50
:101B30008046856803F47040B0F5804F1E4649D05A
:101B40002CDCB0F5805F3DD0B0F5405F3ED060BB8F
:101B500006F44077B7F5807F3ED0A7F50074634266
:101B60006341012919BFD4B2A1464FF01F090024D7
:101B70004FF0010B06F0010C4FEA4C0747EA0C0747
:101B800047EA0020DFF8C8A040EA830706F0020316
:101B9000A14523D2002003B0BDE8F08FB0F5E04F9F
:101BA00016D005DCB0F5A04F0ED06FF01500F2E7AF
:101BB000B0F5404F04D0B0F5504FF6D10720C7E73D
:101BC0000620C5E70120C3E70320C1E70420BFE7E3
:101BD0000520BDE70220BBE70323C2E7D8F80020B9
:101BE0009268117904F01F0242EA411280324AF8E9
:101BF0002270A9680BFA04F2002B25D01143A960CA
:101C00006969B0064CBF114391436961A9697006C7
:101C10004CBF11439143A961296970074CBF11431F
:101C200091432961E96930064CBF0A4321EA020267
:101C3000EA61214640460193FFF7C6FE0028AAD17B
:101C40000134E4B2019BA3E721EA0201D7E700BF18
:101C50000025845001292DE9F04118BFD4B2064671
:101C600012BF25461F2500244FF001088768AC42AB
:101C700002D90020BDE8F081FB6808FA04F223EAEB
:101C80000203FB6021463046FFF79EFE0028F1D19B
:101C90000134E4B2EBE701292DE9F04118BFD4B2D9
:101CA000064612BF25461F2500244FF0010887680D
:101CB000AC4202D90020BDE8F081FB6808FA04F2CA
:101CC0001343FB6021463046FFF77EFE0028F2D129
:101CD0000134E4B2ECE7036882689B681B68D3F8C0
:101CE000100138B1127800200A700122C3F81001E7
:101CF0001A6070474FF0FF30704782B002AA02F8B6
:101D0000011D002103689B681B68C3F82011C3F8FC
:101D100044250122C3F848259A60D3F820110029F0
:101D2000FBD09DF80700DA6002B0704703689B683B
:101D30001B68D3F8240118B1D3F88004C3F88004D9
:101D400070470000036881684FF000509B68104A9C
:101D50001B6890600320C2F874020020C2F8700271
:101D60001D22C3F80C251C22C3F814254FF0EB727A
:101D7000C3F86C05C3F824250822C3F80025012206
:101D8000C3F81001C3F83415C3F838251A6070473A
:101D90000025845038B5084B53F82040013053F8E3
:101DA00020502046854204F10C0400D838BD54F878
:101DB0000C3C5B689847F4E774300000104B70B53A
:101DC00005461E460F4C9C4204D10E4CB44209D12C
:101DD000002412E062681AB122681268AA420CD08C
:101DE0000C34F0E763680BB90C34EFE7236828463E
:101DF0001968FFF7C3FC0028F6D1204670BD00BF6C
:101E0000080F0020A80E0020FFF706B808B50A4DFD
:101E10004FF02002EFF3118382F3118800F06CFB86
:101E2000012104460228D8BF084600F01BFC2C62A2
:101E3000FFF7EEF8ECE700BF280100200248034A54
:101E40000021121AFFF7D4BC000000205801002026
:101E50000248034A0349121AFFF79DBC980E00205E
:101E60001C0F0020DC30000008B50220FFF792FFB5
:101E70000748FEF745FE0320FFF78CFF00F0ACFAA1
:101E8000FEF766FB034A137B23F00103137308BDBF
:101E90009C300000A000002080B586B0374B06AF14
:101EA00083F308880024E022354B364D83F8222046
:101EB000DC771C765C769C76DC765A6A324E42F48D
:101EC000E0225A625A6A42F400225A629C63DA683B
:101ED00092B242F0BF6242F40832DA60FFF7B4FA1D
:101EE000FFF790F82046FFF755FF0120FFF752FF5C
:101EF00000F0CAF9254B756205930123CDE9014431
:101F0000CDE903430094224B4FF4806221492846D7
:101F100000F028FA6B7B344623F0040213F01B0F09
:101F20006A7305D12B6A013302D1284600F02EF9DD
:101F3000194B012205930F23CDE903320023174EDD
:101F4000CDE9013300934FF4A072154B154930468B
:101F500000F008FA737BE66023F004037373124BFE
:101F6000A560C4E906330A4A104B114C83F3098873
:101F700063B6002181F3118810462047980E002097
:101F800000ED00E0A0000020280100208C300000BF
:101F9000691E00005801002091300000340000202C
:101FA0000D1E0000580500204001002058050020AB
:101FB000B1070000D0E900231A600268536070473F
:101FC00008B5FEF7C5FF054B054A1B6800211844FC
:101FD00010611846BDE8084000F044BB1001002025
:101FE000280100204FF02003EFF3118083F31188C4
:101FF0007047000038B5104C234653F8285F9D42C7
:1020000000D005B9E568A36878B973B15A7BD206E8
:102010000BD11A6A013208D1DA897F2A05D9074A19
:102020001268934201D0636238BDAB4201D0FFF722
:10203000C7FF6562F8E700BF280100209830000064
:10204000F8B50D460746FFF7CDFF4FF400460022D6
:1020500000210446094B0A481A61C6FB07014FF4E8
:10206000A0220023FEF784F8064B1860064B1D6083
:10207000FFF7A6FF84F31188F8BD00BF28010020F8
:10208000FFFF0400100100200C01002010B50146E4
:10209000FFF7A8FF4B7B04465A060DD50846FFF70D
:1020A00089FF4B7B23F040034B73054B9868431A21
:1020B00058425841FFF79EFF84F3118810BD00BFBE
:1020C0002801002010B50146FFF78CFF04460846A2
:1020D000FFF770FF4B7B23F002034B7384F31188EF
:1020E00000238B6010BD0000EFF305830D2B0BD890
:1020F0001BB1074B5B681B0506D5064B9A685B6AEC
:102100009A4201D0FEF7C8BF80F31188704700BF24
:1021100000ED00E02801002010B5FFF763FF0A4B37
:1021200004469A680120D37B0133D373FFF762FF23
:1021300084F311884FF02003EFF3118083F31188AB
:10214000BDE81040FFF7D0BF28010020036810B59C
:10215000984213D093B191F90E2093F90E40944216
:1021600006DD5A68C1E900325A681160596010BD35
:102170004468A34202D01B68002BEED1436808607C
:102180004B60436819604160F1E7000038B50446D0
:10219000FFF728FF214605460648FFF7D7FF637B78
:1021A000002043F040036373FFF724FF85F3118899
:1021B00038BD00BF50010020427BD20604D1036A23
:1021C000013301D1FFF7E2BF704738B550F8103C3A
:1021D0000446A0F1180513B12846FFF773FF14F861
:1021E0000B3C284623F0040304F80B3CBDE83840C0
:1021F000FFF7E2BF70B50446FFF7F4FE0B4D06464D
:102200002046FFF7D7FE21462846FFF79FFF637B56
:1022100055F8200C43F040036373031B58425841A8
:10222000FFF7E8FE86F3118870BD00BF5001002063
:10223000114B10B51B68EBB110498B68DA897F2A06
:1022400018D80F4A93F90E401268944212DB0D4AD7
:10225000126893420ED01A6A01320BD10A69824287
:1022600006DC1846FFF7C6FFBDE81040FFF7A8BE22
:10227000121A0A6110BD00BF1001002028010020C1
:102280000C010020983000000021044B084603F1A7
:102290002802C3E90A22FFF7D3BE00BF28010020AD
:1022A000014B9868704700BF28010020F8B505462B
:1022B0000F464FF02003EFF3118483F311884FF49E
:1022C00000460021084800234FF4A022C6FB070166
:1022D000FDF74EFF0549421C05F1180000F03AF9E0
:1022E00084F31188F8BD00BFFFFF0400CB2100007C
:1022F000427BD20604D1036A013301D1FFF746BF06
:1023000070470000EFF305800D2807D838B1044B63
:10231000586880F40060C0F3C02070470120704707
:1023200000ED00E0024B9B68187B00F00100704755
:102330002801002010B54FF02003EFF3118483F340
:102340001188437B590702D484F3118810BD23F010
:1023500004034373FFF7CCFF2046BDE81040FFF7AE
:10236000C3BE000030B587B00E9D044604950D9D98
:1023700003950C9D02950B9D01950A9D0095FFF715
:10238000D3F8044B9B6813B9236607B030BD1B6EAE
:10239000FAE700BF28010020036D10B5044603B121
:1023A0009847637BDA060AD1226A013207D12046B8
:1023B000FFF76CFE637B43F00803637310BD9B075C
:1023C00002D52046FFF77EFE236A0133F2D004F1E6
:1023D000180000F081F8EDE7F0B5234F234D3E469D
:1023E00087B0BD4205F1300414D3214B9A68D37BEA
:1023F000013BD3734FF02003EFF3118583F3118872
:102400001A4CB44223D385F3118807B0BDE8F040DD
:10241000FFF782BE54F8043C059354F8103C049333
:1024200054F8143C039354F8183C029354F81C3CA1
:10243000019354F8203C009354E90A2354E90C0119
:10244000FFF790FF54F8303CDD642546C9E7616A28
:102450004B1C03D0206819B9FFF76CFF3034D0E76C
:10246000FFF724FFFAE700BF080F0020080F002045
:102470002801002003730023C3734FF0FF3342731E
:102480008173036270470000034B1B680BB9FEF7B2
:102490005FBD0020704700BF140100204FF02003F3
:1024A000EFF3118083F3118870470000036840B197
:1024B000084A5268904204D01BB19A6881680A4465
:1024C0009A604268136003685A604FF0FF3383607C
:1024D000704700BFA00E002010B50246FFF7DEFFD8
:1024E00004469068431C03D01046FFF7DFFF00202E
:1024F00084F3118810BD0000134B70B51B78002BBE
:1025000014BF4FF0FF326FF00042FFF7C7FF0F4BD1
:1025100006461C689C420AD04CB1A568FFF7B4FF80
:10252000281A00280DDBA468FFF7AEFF221A86F3F5
:102530001188074B1B6913B19A42A8BF1A4610466F
:1025400070BD0022F3E700BF18010020A00E00209C
:102550002801002070B5C16016460446FFF79EFFB3
:102560000546FFF791FF012EACBF80190130164BD5
:10257000A0601A689A4201D05E6832B95A68236036
:1025800062605A6814605C600BE09068A1688842E1
:1025900014DD411A91605168C4E9002151680C6052
:1025A00054601A689A4206D0944204D1FFF7A4FFFF
:1025B0000021FEF79BFC85F3118870BD091A964235
:1025C000A160DBD01268D8E7A00E00202DE9F04B07
:1025D00004464FF00008204D204E214FFFF728FE03
:1025E0002C60FFF75BFF34688146B4421CD094B185
:1025F000A1682B68994215DC5B1A2B60D7E9002390
:1026000012EB010B43EBE17CC4F808802046C7E9DC
:1026100000BCFFF74BFF89F311883CB1E36820460B
:102620009847DEE7C91AA1600024F4E7FFF736FFF8
:102630000B490646D1E9002328682C60171843EBA4
:10264000E078C1E90078FFF757FF2146FEF74EFC1E
:1026500086F31188BDE8F08B14010020A00E002045
:102660002001002070B50E460446FFF717FF05460F
:10267000FFF742FF431C01D0A04203DD3146204654
:10268000FEF734FC85F3118870BD704784DBFF7F53
:102690000100000000000000D11400000000000054
:1026A000D114000000000000D11400000000000060
:1026B000D114000000000000D11400000000000050
:1026C000E10C000000000000D11400000000000038
:1026D000D114000000000000D11400000000000030
:1026E000D114000000000000D11400000000000020
:1026F000D114000000000000D11400000000000010
:102700003D19000000000000D1140000000000008E
:10271000D114000000000000D114000000000000EF
:10272000D114000000000000D114000000000000DF
:10273000D114000000000000D114000000000000CF
:10274000290E000000000000D1140000000000006D
:10275000D114000000000000D114000000000000AF
:10276000D114000000000000D1140000000000009F
:10277000D114000000000000D1140000000000008F
:10278000D114000000000000D1140000000000007F
:10279000D114000000000000D1140000000000006F
:1027A000D114000000000000D1140000000000005F
:1027B000D114000000000000D1140000000000004F
:1027C000D114000000000000D1140000000000003F
:1027D000D114000000000000D1140000000000002F
:1027E000D114000000000000D1140000000000001F
:1027F000D114000000000000D1140000000000000F
:10280000D114000000000000D114000000000000FE
:10281000D114000000000000D114000000000000EE
:10282000D114000000000000D114000000000000DE
:10283000D114000000000000D114000000000000CE
:10284000D114000000000000D114000000000000BE
:10285000D114000000000000D114000000000000AE
:10286000D114000000000000D1140000000000009E
:10287000D114000000000000D1140000000000008E
:10288000D114000000000000D1140000000000007E
:10289000D114000000000000D11400002C2C000016
:1028A0001D0B0000000000002C2C0000110C00008B
:1028B00000000000C42A00004F0D000000000000CE
:1028C000CF2A00004F0D000000000000DA2A0000AF
:1028D000690E0000000000002C2C00001117000001
:1028E0000000000054300000DD1800004C300000F3
:1028F000A32A0000451D0000703000005365637579
:10290000726520426F6F743A20636F6E66696775F7
:10291000726520666C6173680A0053656375726541
:1029200020426F6F743A205350553A2073657420DB
:10293000726567696F6E202575206173205365632A
:102940007572650A0053656375726520426F6F7416
:102950003A205350553A2073657420466C61736871
:1029600020726567696F6E202575206173204E6F38
:102970006E2D5365637572650A00536563757265E4
:1029800020426F6F743A20636F6E66696775726577
:10299000205352414D0A0053656375726520426FA2
:1029A0006F743A205350553A207365742053524146
:1029B0004D20726567696F6E202575206173205305
:1029C00065637572650A0053656375726520426FB1
:1029D0006F743A205350553A207365742053524116
:1029E0004D20726567696F6E202575206173204EDA
:1029F0006F6E2D5365637572650A0053656375725A
:102A00006520426F6F743A20636F6E6669677572F6
:102A100065207065726970686572616C730A005335
:102A2000656375726520426F6F743A204D53505F35
:102A30004E532025780A0053656375726520426FF6
:102A40006F743A207072657061726520746F206ACD
:102A5000756D7020746F204E6F6E2D5365637572A7
:102A60006520696D6167650A0000000002000000D2
:102A7000742A000000000000942A000006000000F4
:102A8000E0FF0F00000000209C2A00002100000051
:102A9000E0FF0020464C4153485F30005352414D07
:102AA0005F3000554152545F300000008D0C000033
:102AB0000000000000000000650D00002D0C00006B
:102AC00000000000636C6B5F6B33327372630063F2
:102AD0006C6B5F6D3136737263007379735F636C17
:102AE0006F636B002A2A2A2A2A2042555320464126
:102AF000554C54202A2A2A2A2A0A0020205072657E
:102B00006369736520646174612062757320657206
:102B1000726F720A00202042464152204164647262
:102B20006573733A20307825780A002020496D704B
:102B300072656369736520646174612062757320D6
:102B40006572726F720A002020496E737472756329
:102B500074696F6E20627573206572726F720A00FD
:102B60005265736572766564204578636570746933
:102B70006F6E20280053707572696F757320696ECF
:102B8000746572727570742028495251200020209B
:102B90005320696E737472756374696F6E2061641B
:102BA00064726573733A2020307825780A005245A4
:102BB00054544F4241534520646F6573206E6F74C7
:102BC000206D61746368204558435F5245545552E7
:102BD0004E0A002A2A2A2A2A2048415244204641E5
:102BE000554C54202A2A2A2A2A0A0020204275738A
:102BF000206661756C74206F6E20766563746F72E9
:102C0000207461626C6520726561640A0020204650
:102C100061756C7420657363616C6174696F6E209B
:102C2000287365652062656C6F77290A002A2A2A55
:102C30002A2A204465627567206D6F6E69746F7211
:102C400020657863657074696F6E20286E6F7420DC
:102C5000696D706C656D656E74656429202A2A2A19
:102C60002A2A0A002A2A2A2A2A20257320256429AA
:102C7000202A2A2A2A2A0A002A2A2A2A2A204D50C9
:102C800055204641554C54202A2A2A2A2A0A002037
:102C900020537461636B696E67206572726F720A8C
:102CA000002020556E737461636B696E67206572D6
:102CB000726F720A00202044617461204163636571
:102CC00073732056696F6C6174696F6E0A002020FF
:102CD0004D4D46415220416464726573733A203011
:102CE0007825780A002020496E73747275637469C0
:102CF0006F6E204163636573732056696F6C6174F6
:102D0000696F6E0A002020466C6F6174696E672DD2
:102D1000706F696E74206C617A7920737461746568
:102D200020707265736572766174696F6E2065726A
:102D3000726F720A002A2A2A2A2A205345435552C2
:102D400045204641554C54202A2A2A2A2A0A002086
:102D500020416464726573733A20307825780A00E4
:102D60002020496E76616C696420656E74727920EA
:102D7000706F696E740A002020496E76616C696418
:102D800020696E74656772697479207369676E6112
:102D9000747572650A002020496E76616C69642042
:102DA000657863657074696F6E2072657475726E94
:102DB0000A0020204174747269627574696F6E2014
:102DC000756E69742076696F6C6174696F6E0A0044
:102DD0002020496E76616C6964207472616E73693B
:102DE00074696F6E0A0020204C617A7920737461D7
:102DF000746520707265736572766174696F6E0AAE
:102E00000020204C617A79207374617465206572AA
:102E1000726F720A002A2A2A2A2A205553414745EE
:102E2000204641554C54202A2A2A2A2A0A002020CA
:102E30004469766973696F6E206279207A65726F72
:102E40000A002020556E616C69676E6564206D65AF
:102E50006D6F7279206163636573730A002020537C
:102E60007461636B206F766572666C6F770A002001
:102E7000204E6F20636F70726F636573736F722083
:102E8000696E737472756374696F6E730A002020C3
:102E9000496C6C6567616C206C6F6164206F6620A3
:102EA0004558435F52455455524E20696E746F2009
:102EB00050430A002020496C6C6567616C20757373
:102EC00065206F662074686520455053520A0020C3
:102ED00020417474656D707420746F20657865632B
:102EE00075746520756E646566696E656420696ECB
:102EF000737472756374696F6E0A002A2A2A2A2A0B
:102F000020486172647761726520657863657074CA
:102F1000696F6E202A2A2A2A2A0A002A2A2A2A20A7
:102F20004B65726E656C20416C6C6F636174696F88
:102F30006E204661696C75726521202A2A2A2A0A48
:102F4000002A2A2A2A2A204B65726E656C204F4F70
:102F5000505321202A2A2A2A2A0A002A2A2A2A2ADF
:102F6000204B65726E656C2050616E696321202A6A
:102F70002A2A2A2A0A002A2A2A2A20556E6B6E6FCC
:102F8000776E20466174616C204572726F722025E5
:102F90006421202A2A2A2A0A0043757272656E74F7
:102FA00020746872656164204944203D2025700AC0
:102FB0004661756C74696E6720696E7374727563AF
:102FC00074696F6E2061646472657373203D203094
:102FD0007825780A0049535200657373656E7469E9
:102FE000616C2074687265616400466174616C2074
:102FF0006661756C7420696E202573212053706999
:103000006E6E696E672E2E2E0A00466174616C200A
:103010006661756C7420696E2074687265616420E5
:103020002570212041626F7274696E672E0A00005C
:103030002D1B0000331800006718000099180000CD
:10304000971C0000551C0000000000000025845063
:10305000000000004750494F5F300000D71C0000BF
:10306000FB1C00002D1D00000000000000000000FF
:1030700000800050A80E0020F00E0020FC0E002062
:10308000080F0020080F0020F5FFFFFF6D61696E3B
:103090000069646C65000000340000202A2A2A2A96
:1030A0002A20426F6F74696E67205A657068797262
:1030B000204F532076312E31332E39392D6E6373E4
:1030C000312D313832332D67373135643264663310
:1030D0006464202A2A2A2A2A0A000000C507000060
:1030E0000090D003A00E0020A00E00209C2800001D
:1030F0000000000000000000D828000000000000D0
:1031000000000000B4280000AC2A0000000000000D
:10311000C0280000B82A000000000000F0280000CD
:103120005C30000030000020A828000000000000F3
:1031300000000000CC28000000000000000000009B
:10314000E42800003030000010000020080F0020AC
:10315000080F002000000000000000000F00000029
:020000040004F6
:1000000090C70220B9490400554A04001948040069
:10001000194804001948040019480400194804004C
:10002000194804001948040019480400D943040081
:1000300019480400194804009543040019480400B5
:100040007949040079490400794904007949040098
:100050007949040079490400794904007949040088
:100060007949040079490400794904007949040078
:100070007949040079490400794904007949040068
:100080007949040079490400794904007949040058
:100090007949040079490400794904007949040048
:1000A0007949040079490400794904007949040038
:1000B000F1BC040013BD040079490400794904002F
:1000C0007949040079490400794904007949040018
:1000D0007949040079490400794904007949040008
:1000E000794904007949040035BD040079490400C8
:1000F00079490400794904007949040079490400E8
:1001000079490400794904007949040079490400D7
:1001100079490400794904007949040079490400C7
:1001200079490400794904007949040079490400B7
:1001300079490400794904007949040079490400A7
:100140007949040081F0004102E000BF83F00043E0
:1001500030B54FEA41044FEA430594EA050F08BF62
:1001600090EA020F1FBF54EA000C55EA020C7FEA26
:10017000645C7FEA655C00F0E2804FEA5454D4EBA3
:100180005555B8BF6D420CDD2C4480EA020281EA6D
:10019000030382EA000083EA010180EA020281EAA5
:1001A0000303362D88BF30BD11F0004F4FEA0131F7
:1001B0004FF4801C4CEA113102D0404261EB410106
:1001C00013F0004F4FEA03334CEA133302D052428C
:1001D00063EB430394EA050F00F0A780A4F1010448
:1001E000D5F1200E0DDB02FA0EFC22FA05F2801882
:1001F00041F1000103FA0EF2801843FA05F3594168
:100200000EE0A5F120050EF1200E012A03FA0EFCE6
:1002100028BF4CF0020C43FA05F3C01851EBE37110
:1002200001F0004507D54FF0000EDCF1000C7EEB2D
:1002300000006EEB0101B1F5801F1BD3B1F5001F6B
:100240000CD349085FEA30004FEA3C0C04F101048A
:100250004FEA445212F5800F80F09A80BCF1004FB3
:1002600008BF5FEA500C50F1000041EB045141EA35
:10027000050130BD5FEA4C0C404141EB010111F436
:10028000801FA4F10104E9D191F0000F04BF0146E1
:100290000020B1FA81F308BF2033A3F10B03B3F1BF
:1002A00020020CDA0C3208DD02F1140CC2F10C024F
:1002B00001FA0CF021FA02F10CE002F11402D8BFAD
:1002C000C2F1200C01FA02F120FA0CFCDCBF41EA79
:1002D0000C019040E41AA2BF01EB0451294330BD48
:1002E0006FEA04041F3C1CDA0C340EDC04F1140425
:1002F000C4F1200220FA04F001FA02F340EA0300FC
:1003000021FA04F345EA030130BDC4F10C04C4F141
:10031000200220FA02F001FA04F340EA0300294621
:1003200030BD21FA04F0294630BD94F0000F83F46B
:10033000801306BF81F480110134013D4EE77FEA4E
:10034000645C18BF7FEA655C29D094EA050F08BF9A
:1003500090EA020F05D054EA000C04BF194610467B
:1003600030BD91EA030F1EBF0021002030BD5FEABF
:10037000545C05D14000494128BF41F0004130BDE7
:1003800014F580043CBF01F5801130BD01F000453B
:1003900045F0FE4141F470014FF0000030BD7FEAAE
:1003A000645C1ABF194610467FEA655C1CBF0B46A9
:1003B000024650EA013406BF52EA033591EA030FC0
:1003C00041F4002130BD00BF90F0000F04BF0021B8
:1003D000704730B54FF4806404F132044FF00005EB
:1003E0004FF0000150E700BF90F0000F04BF002164
:1003F000704730B54FF4806404F1320410F00045CA
:1004000048BF40424FF000013EE700BF42004FEAC4
:10041000E2014FEA31014FEA02701FBF12F07F4341
:1004200093F07F4F81F06051704732F07F4208BFF8
:10043000704793F07F4F04BF41F40021704730B5FF
:100440004FF4607401F0004521F000411CE700BF4B
:1004500050EA010208BF704730B54FF000050AE0CE
:1004600050EA010208BF704730B511F0004502D5CF
:10047000404261EB41014FF4806404F132045FEAD1
:10048000915C3FF4D8AE4FF003025FEADC0C18BF7A
:1004900003325FEADC0C18BF033202EBDC02C2F16C
:1004A000200300FA03FC20FA02F001FA03FE40EAFE
:1004B0000E0021FA02F11444BDE600BF70B54FF002
:1004C000FF0C4CF4E06C1CEA11541DBF1CEA1355E0
:1004D00094EA0C0F95EA0C0F00F0DEF82C4481EA48
:1004E000030621EA4C5123EA4C5350EA013518BF68
:1004F00052EA033541F4801143F4801338D0A0FB55
:1005000002CE4FF00005E1FB02E506F00042E0FB01
:1005100003E54FF00006E1FB03569CF0000F18BF07
:100520004EF0010EA4F1FF04B6F5007F64F54074AF
:1005300004D25FEA4E0E6D4146EB060642EAC62142
:1005400041EA55514FEAC52040EA5E504FEACE2EAF
:10055000B4F1FD0C88BFBCF5E06F1ED8BEF1004FB2
:1005600008BF5FEA500E50F1000041EB045170BD2E
:1005700006F0004646EA010140EA020081EA030172
:10058000B4EB5C04C2BFD4EB0C0541EA045170BD6E
:1005900041F480114FF0000E013C00F3AB8014F1E8
:1005A000360FDEBF002001F0004170BDC4F1000431
:1005B000203C35DA0C341BDC04F11404C4F12005B2
:1005C00000FA05F320FA04F001FA05F240EA02000D
:1005D00001F0004221F0004110EBD37021FA04F643
:1005E00042EB06015EEA430E08BF20EAD37070BDFD
:1005F000C4F10C04C4F1200500FA04F320FA05F05C
:1006000001FA04F240EA020001F0004110EBD3705D
:1006100041F100015EEA430E08BF20EAD37070BDCD
:10062000C4F1200500FA05F24EEA020E20FA04F3A6
:1006300001FA05F243EA020321FA04F001F0004155
:1006400021FA04F220EA020000EBD3705EEA430EC6
:1006500008BF20EAD37070BD94F0000F0FD101F0F5
:100660000046400041EB010111F4801F08BF013C2E
:10067000F7D041EA060195F0000F18BF704703F06C
:100680000046520043EB030313F4801F08BF013DF3
:10069000F7D043EA0603704794EA0C0F0CEA1355AF
:1006A00018BF95EA0C0F0CD050EA410618BF52EA69
:1006B0004306D1D181EA030101F000414FF000006F
:1006C00070BD50EA410606BF1046194652EA43067D
:1006D00019D094EA0C0F02D150EA013613D195EAF1
:1006E0000C0F05D152EA03361CBF104619460AD139
:1006F00081EA030101F0004141F0FE4141F4700143
:100700004FF0000070BD41F0FE4141F4780170BD32
:1007100070B54FF0FF0C4CF4E06C1CEA11541DBF97
:100720001CEA135594EA0C0F95EA0C0F00F0A7F899
:10073000A4EB050481EA030E52EA03354FEA0131C6
:1007400000F088804FEA03334FF0805545EA1313D9
:1007500043EA12634FEA022245EA111545EA1065A1
:100760004FEA00260EF000419D4208BF964244F138
:10077000FD0404F5407402D25B084FEA3202B61A57
:1007800065EB03055B084FEA32024FF480104FF42B
:10079000002CB6EB020E75EB030E22BFB61A75469F
:1007A00040EA0C005B084FEA3202B6EB020E75EB32
:1007B000030E22BFB61A754640EA5C005B084FEA9A
:1007C0003202B6EB020E75EB030E22BFB61A754667
:1007D00040EA9C005B084FEA3202B6EB020E75EB72
:1007E000030E22BFB61A754640EADC0055EA060E33
:1007F00018D04FEA051545EA16754FEA06164FEA76
:10080000C30343EA52734FEAC2025FEA1C1CC0D121
:1008100011F4801F0BD141EA00014FF000004FF0AE
:10082000004CB6E711F4801F04BF01430020B4F16F
:10083000FD0C88BFBCF5E06F3FF6AFAEB5EB030C27
:1008400004BFB6EB020C5FEA500C50F1000041EB24
:10085000045170BD0EF0004E4EEA113114EB5C04F1
:10086000C2BFD4EB0C0541EA045170BD41F48011C4
:100870004FF0000E013C90E645EA060E8DE60CEACC
:10088000135594EA0C0F08BF95EA0C0F3FF43BAFE9
:1008900094EA0C0F0AD150EA01347FF434AF95EAA0
:1008A0000C0F7FF425AF104619462CE795EA0C0F84
:1008B00006D152EA03353FF4FDAE1046194622E751
:1008C00050EA410618BF52EA43067FF4C5AE50EA2B
:1008D00041047FF40DAF52EA43057FF4EBAE12E71B
:1008E0004FF0FF3C06E000BF4FF0010C02E000BFFC
:1008F0004FF0010C4DF804CD4FEA410C7FEA6C5CDF
:100900004FEA430C18BF7FEA6C5C1BD001B050EA81
:10091000410C0CBF52EA430C91EA030F02BF90EA6C
:10092000020F0020704710F1000F91EA030F58BF2B
:10093000994208BF90422CBFD8176FEAE37040F08D
:10094000010070474FEA410C7FEA6C5C02D150EA2B
:10095000013C07D14FEA430C7FEA6C5CD6D152EAE6
:10096000033CD3D05DF8040B704700BF84461046AB
:1009700062468C461946634600E000BF01B5FFF7AA
:10098000B7FF002848BF10F1000F01BD4DF808ED7A
:10099000FFF7F4FF0CBF012000205DF808FB00BF4B
:1009A0004DF808EDFFF7EAFF34BF012000205DF8A5
:1009B00008FB00BF4DF808EDFFF7E0FF94BF0120F2
:1009C00000205DF808FB00BF4DF808EDFFF7CEFFF3
:1009D00094BF012000205DF808FB00BF4DF808ED32
:1009E000FFF7C4FF34BF012000205DF808FB00BF03
:1009F0004FEA410212F5001215D211D56FF4787347
:100A0000B3EB625212D94FEAC12343F0004343EAE9
:100A1000505311F0004F23FA02F018BF40427047C4
:100A20004FF00000704750EA013005D111F000404E
:100A300008BF6FF0004070474FF00000704700BFE4
:100A40007BB972B90029BEBF00204FF0004106E01B
:100A500008BF00281CBF6FF000414FF0FF3000F0CE
:100A6000C7B9ADF1080C6DE904CE002909DB002BF4
:100A70001ADB00F04DF8DDF804E0DDE9022304B0F4
:100A80007047404261EB4101002B1BDB00F040F856
:100A9000DDF804E0DDE9022304B0404261EB4101EE
:100AA000524263EB43037047524263EB430300F04F
:100AB0002FF8DDF804E0DDE9022304B0404261EBE9
:100AC00041017047524263EB430300F021F8DDF827
:100AD00004E0DDE9022304B0524263EB43037047B4
:100AE00053B94AB9002908BF00281CBF4FF0FF3195
:100AF0004FF0FF3000F07CB9ADF1080C6DE904CE89
:100B000000F006F8DDF804E0DDE9022304B07047E8
:100B10002DE9F0478C46089D04468A46002B4AD1B1
:100B20008A42174662D9B2FA82F64EB1C6F1200E59
:100B300001FA06F3B740B44020FA0EFE4EEA030A6B
:100B40004FEA1748230C1FFA87F9BAFBF8FE08FB97
:100B50001EAA0EFB09F243EA0A439A420BD9FB187C
:100B60000EF1FF312CBF012000209A4202D900284B
:100B700000F02A818E469A1AA3B2B2FBF8F008FB65
:100B8000102200FB09F943EA0244A14507D93C19A8
:100B900000F1FF3302D2A14500F210811846A4EB08
:100BA000090440EA0E4000211DB1F4400023C5E9CC
:100BB0000043BDE8F0878B4208D9002D00F0F28099
:100BC0000021C5E9000C0846BDE8F087B3FA83F1BF
:100BD00000294ED16345C0F0E880824240F2E580B2
:100BE0000846002DE5D0C5E9004AE2E702B9FFDE7C
:100BF000B2FA82F6002E40F099808B1A4FEA124E1C
:100C00001FFA82F801214FEA144CB3FBFEF20EFBEF
:100C1000123008FB02F94CEA004CE14508D917EB09
:100C20000C0C02F1FF3302D2E14500F2CA801A46F1
:100C3000ACEB090CA3B2BCFBFEF00EFB10CC08FB26
:100C400000F843EA0C44A0450ED93C1900F1FF33EB
:100C50002CBF4FF0010C4FF0000CA04503D9BCF1A4
:100C6000000F00F0A8801846A4EB080440EA0240F8
:100C70009AE7C1F120048B4002FA01FE0CFA01F65A
:100C8000E24020FA04F72CFA04FC00FA01F81343BE
:100C90003E431F0C320C1FFA83F9BCFBF7F007FB35
:100CA00010CC00FB09FA42EA0C4CE24508D913EBE0
:100CB0000C0C00F1FF3202D2E24500F289801046AE
:100CC000ACEB0A0CB6B2BCFBF7FA07FB1ACC0AFB7A
:100CD00009F946EA0C42914506D99A180AF1FF36FD
:100CE00001D291457AD8B2464AEA0040A2EB090205
:100CF000A0FB0E67BA42B446B94602D307D1B0454D
:100D000005D2B6EB0E0C67EB030301389946002DB4
:100D10006BD0B8EB0C0362EB090202FA04F4CB408F
:100D2000CA4000211C43C5E9004242E7B740C6F172
:100D3000200201FA06F3B44021FA02FC4FEA174EF2
:100D400020FA02F21FFA87F8BCFBFEF11A430EFBF1
:100D500011CC01FB08F0130C43EA0C4C604507D999
:100D600017EB0C0C01F1FF3301D2604533D8194663
:100D7000ACEB000C92B2BCFBFEF00EFB10CC00FB07
:100D800008F342EA0C4C634507D917EB0C0C00F151
:100D9000FF3201D2634525D81046ACEB030340EA8D
:100DA000014130E72946284603E7841A6CEB030328
:100DB00001209A4615E702383C4455E702383C4486
:100DC000EDE6023ABC4433E7AEF1020E3B44D2E614
:100DD00002389C4474E70239BC44C9E7AAF1020A0C
:100DE0001A4481E70238BC44D7E72946E1E600BF50
:100DF000704700BF844641EA000313F0030349D162
:100E0000403A23D30B6803604B6843608B68836070
:100E1000CB68C3600B6903614B6943618B69836174
:100E2000CB69C3610B6A03624B6A43628B6A83625C
:100E3000CB6AC3620B6B03634B6B43638B6B836344
:100E4000CB6BC36340304031403ADBD230320BD3FE
:100E50000B6803604B6843608B688360CB68C3603A
:100E600010301031103AF3D20C3205D351F8043B54
:100E700040F8043B043AF9D2043208D0D2071CBF30
:100E800011F8013B00F8013B01D30B880380604659
:100E9000704700BF082A13D38B07B1D010F00303AB
:100EA000AED0C3F10403D21ADB071CBF11F8013B1B
:100EB00000F8013BA4D331F8023B20F8023B9FE746
:100EC000043AD9D3013A11F8013B00F8013BF9D2B9
:100ED0000B7803704B7843708B7883706046704753
:100EE00080EA010C1CF0030F37D110F0030C20F046
:100EF000030021F0030150F8042B08BF51F8043B14
:100F00000ED08CF0030C6FF07F434FEACC0C23FA29
:100F10000CFC51F8043B42EA0C0243EA0C0300BF0C
:100F2000A2F1013C9A4201BF2CEA020C1CF0803F66
:100F300050F8042B51F8043BF2D04FEA02604FEA1C
:100F40001222012828BFB0EB036F08BF1B0AF4D0A0
:100F500003F0FF03000EC01A704710F0030F0AD011
:100F600010F8012B11F8013B012A28BF9A42F4D056
:100F7000A2EB030070474DF8045D50F8042B01F01C
:100F8000030521F0030151F8043B022D26D04DD872
:100F900022F07F45B5EB132FA2F1013C2CEA020CA5
:100FA0000DD11CF0803C08BF51F8043B0AD185EA02
:100FB0000205B5EB036F0CD150F8042BE8E74FEABC
:100FC00013235BE03CF07F4C54D10B784FEA126561
:100FD00054E04FEA126503F0FF034FE04FEA024589
:100FE000A2F1013C4FEA15452CEA020CB5EB134F78
:100FF00018D11CF0803C08BF51F8043B07D185EAAA
:101000000205B5EB034F09D150F8042BE6E75FEA80
:101010000C4C2FD10B884FEA12452FE04FEA0343C7
:101020004FEA12454FEA134328E000BF02F0FF05E4
:10103000B5EB136FA2F1013C2CEA020C0DD11CF0B0
:10104000803C08BF51F8043B0AD185EA0205B5EBA4
:10105000032F0AD150F8042BE8E74FEA13630DE0A1
:1010600012F0FF0F06D051F8043B4FEA122523F08F
:101070007F4303E04FF0000020BC704705F0FF0203
:1010800003F0FF00012828BF904204BF2D0A1B0A6D
:10109000F4D0A2EB000020BC704700BF30B44FF08A
:1010A000000310F8014B11F8015B013A84EA0504D2
:1010B00043EA0403F5D1A3F101034FEAD37030BC36
:1010C00070474FF0000310F8012B013943EA020387
:1010D000F9D1A3F101034FEAD37070472DE9F0076E
:1010E00091E8F807B2E802105B1854EB0C04B2E880
:1010F00002104D4156EB0C06B2E802104F4158EB7E
:101100000C08B2E8021059EB01095AEB0C0A8941AC
:10111000B3F1FF3374F1FF3475F1FF3576F100065A
:1011200077F1000778F1000879F101097AF1FF3AC7
:1011300051F100014A425B184C414D4156F1000605
:1011400057F1000758F1000859EB02095AEB010A60
:1011500080E8F807BDE8F00770472DE9F00791E84F
:10116000F807B2E802105B1A74EB0C04B2E8021044
:101170008D4176EB0C06B2E802108F4178EB0C083B
:10118000B2E8021079EB01097AEB0C0A89414A4274
:101190005B184C414D4156F1000657F1000758F1DC
:1011A000000859EB02095AEB010A80E8F807BDE88C
:1011B000F00770470A462DE9F04F92E8F00F2DE94D
:1011C000F30F87B091E839000999A0FB01784FF03F
:1011D0000009E3FB01894FF0000AE4FB019A4FF09C
:1011E000000BE5FB01AB0D994FF0000CE0FB01BCDF
:1011F0004FF0000EE3FB01CE4FF00002E4FB01E2F2
:101200004FF00006E5FB012600970A994FF0000712
:10121000E0FB018719EB07094FF0000747EB0707D1
:10122000E3FB01971AEB070A4FF0000747EB0707AC
:10123000E4FB01A71BEB070B4FF0000747EB070789
:10124000E5FB01B70E991CEB070C4FF0000747EBCD
:101250000707E0FB01C71EEB070E4FF0000747EB47
:101260000707E3FB01E7D2194FF0000747EB070739
:10127000E4FB0127F6194FF0000747EB0707E5FBF2
:101280000167CDF804800B994FF00008E0FB01984E
:101290001AEB080A4FF0000848EB0808E3FB01A826
:1012A0001BEB080B4FF0000848EB0808E4FB01B803
:1012B0001CEB080C4FF0000848EB0808E5FB01C8E0
:1012C0000F991EEB080E4FF0000848EB0808E0FBF2
:1012D00001E812EB08024FF0000848EB0808E3FBB6
:1012E000012816EB08064FF0000848EB0808E4FB5D
:1012F000016817EB08074FF0000848EB0808E5FB0A
:101300000178CDF808900C994FF00009E0FB01A995
:101310001BEB090B4FF0000949EB0909E3FB01B98D
:101320001CEB090C4FF0000949EB0909E4FB01C96A
:101330001EEB090E4FF0000949EB0909E5FB01E935
:10134000109912EB09024FF0000949EB0909E0FB83
:10135000012916EB09064FF0000949EB0909E3FBE7
:10136000016917EB09074FF0000949EB0909E4FB94
:10137000017918EB09084FF0000949EB0909E5FB71
:101380000189CDF80CA0089901F1100191E839000C
:1013900009994FF0000AE0FB01BA1CEB0A0C4FF070
:1013A000000A4AEB0A0AE3FB01CA1EEB0A0E4FF0E1
:1013B000000A4AEB0A0AE4FB01EA12EB0A024FF0C8
:1013C000000A4AEB0A0AE5FB012A0D9916EB0A0608
:1013D0004FF0000A4AEB0A0AE0FB016A17EB0A0722
:1013E0004FF0000A4AEB0A0AE3FB017A18EB0A08FD
:1013F0004FF0000A4AEB0A0AE4FB018A19EB0A09DA
:101400004FF0000A4AEB0A0AE5FB019ACDF810B04A
:101410000A994FF0000BE0FB01CB1EEB0B0E4FF0D7
:10142000000B4BEB0B0BE3FB01EB12EB0B024FF052
:10143000000B4BEB0B0BE4FB012B16EB0B064FF0F9
:10144000000B4BEB0B0BE5FB016B0E9917EB0B073E
:101450004FF0000B4BEB0B0BE0FB017B18EB0B0889
:101460004FF0000B4BEB0B0BE3FB018B19EB0B0964
:101470004FF0000B4BEB0B0BE4FB019B1AEB0B0A41
:101480004FF0000B4BEB0B0BE5FB01ABCDF814C0A1
:101490000B994FF0000CE0FB01EC12EB0C024FF04B
:1014A000000C4CEB0C0CE3FB012C16EB0C064FF084
:1014B000000C4CEB0C0CE4FB016C17EB0C074FF031
:1014C000000C4CEB0C0CE5FB017C0F9918EB0C08A5
:1014D0004FF0000C4CEB0C0CE0FB018C19EB0C09F1
:1014E0004FF0000C4CEB0C0CE3FB019C1AEB0C0ACC
:1014F0004FF0000C4CEB0C0CE4FB01AC1BEB0C0BA9
:101500004FF0000C4CEB0C0CE5FB01BCCDF818E0E7
:101510000C994FF0000EE0FB012E16EB0E064FF07B
:10152000000E4EEB0E0EE3FB016E17EB0E074FF0B5
:10153000000E4EEB0E0EE4FB017E18EB0E084FF092
:10154000000E4EEB0E0EE5FB018E109919EB0E0905
:101550004FF0000E4EEB0E0EE0FB019E1AEB0E0A52
:101560004FF0000E4EEB0E0EE3FB01AE1BEB0E0B2D
:101570004FF0000E4EEB0E0EE4FB01BE1CEB0E0C0A
:101580004FF0000E4EEB0E0EE5FB01CEDDE904340C
:10159000069913EB0A0354EB0B0451EB0C0152EBCD
:1015A0000E02002040F1000013EB0B0354EB0C047F
:1015B00051EB0E0152EB0E0246410020474158EB21
:1015C000000859EB0A0940F10000B3EB0E0374F177
:1015D000000471F1000172EB0A0276EB0B0677EB67
:1015E0000C0778EB0A0879EB0C0960F10000B2EB0C
:1015F0000B0276EB0C0677EB0E0778EB0B0879EB1A
:101600000E0960F100005FEAE07C7FEA0C0CDCF17F
:10161000000EB3EB0C0374EB0C0471EB0C0172F1D4
:10162000000276F1000677F1000778EB0E0879EBFF
:101630000C0960F100005FEAE07CDCF1000E13EBC6
:101640000C0354EB0C0451EB0C0152F1000256F167
:10165000000657F1000758EB0E0859EB0C0940F152
:1016600000005FEAE07CDCF1000E13EB0C0354EBAE
:101670000C0451EB0C0152F1000256F1000657F137
:10168000000758EB0E0859EB0C09DDE900ABDDE96A
:1016900002CE1AEB060A5BEB070B5CEB080C5EEB69
:1016A000090E002040F100001AEB070A5BEB080B63
:1016B0005CEB090C5EEB090E4341002044414141C3
:1016C000724140F10000BAEB090A7BF1000B7CF19A
:1016D000000C7EEB060EBB4174EB0804B14172EBCB
:1016E000080260F10000BEEB070E73EB080374EB19
:1016F0000904B94172EB090260F100005FEAE07889
:101700007FEA0808D8F10009BAEB080A7BEB080B5E
:101710007CEB080C7EF1000E73F1000374F1000401
:1017200071EB090172EB080260F100005FEAE078FA
:10173000D8F100091AEB080A5BEB080B5CEB080C0C
:101740005EF1000E53F1000354F1000451EB090166
:1017500052EB080240F100005FEAE078D8F100099E
:101760001AEB080A5BEB080B5CEB080C5EF1000E51
:1017700053F1000354F1000451EB090152EB08024C
:101780000798A0E8005C18C080E8060011B0BDE82A
:10179000F08F00BF70B491E87800B2E802105B18D7
:1017A00054EB0C04B2E802104D4156EB0C0680E8F5
:1017B00078008041013070BC70472DE9F00791E856
:1017C000F807B2E802105B1854EB0C04B2E8021000
:1017D0004D4156EB0C06B2E802104F4158EB0C0895
:1017E000B2E8021059EB01095AEB0C0A80E8F8073D
:1017F00080410130BDE8F00770472DE9F00791E81E
:10180000F807B2E802105B1A74EB0C04B2E802109D
:101810008D4176EB0C06B2E802108F4178EB0C0894
:10182000B2E8021079EB01097AEB0C0A80E8F807BC
:1018300080414042BDE8F00770472DE9F007524271
:1018400090E87800B1E880071740DB1918EA020831
:1018500054EB080419EA020955EB09051AEA020AD1
:1018600056EB0A0678C090E87800B1E88007174088
:101870007B4118EA020854EB080419EA020955EB07
:1018800009051AEA020A56EB0A0678C080410130BF
:10189000BDE8F00770472DE9F007524290E8780064
:1018A000B1E880071740DB1B18EA020874EB080454
:1018B00019EA020975EB09051AEA020A76EB0A062B
:1018C00078C090E87800B1E880071740BB4118EA7B
:1018D000020874EB080419EA020975EB09051AEA13
:1018E000020A76EB0A0678C080414042BDE8F00764
:1018F000704790E8300091E8C000A31B1340E41A41
:10190000F618EB1B1340ED1AFF1830C0C0C170472A
:10191000F0B55242FFF7EDFFFFF7EBFFFFF7E9FFEE
:10192000FFF7E7FFF0BD2DE9F0073AC91668A1FB04
:10193000069A4FF0000CE3FB06AC4FF00007E4FB07
:1019400006C74FF00008E5FB067840F8049B566890
:101950004FF00009E1FB06A91CEB090C4FF0000950
:1019600049EB0909E3FB06C917EB09074FF000092A
:1019700049EB0909E4FB067918EB09084FF0000967
:1019800049EB0909E5FB068940F804AB96684FF07E
:10199000000AE1FB06CA17EB0A074FF0000A4AEB00
:1019A0000A0AE3FB067A18EB0A084FF0000A4AEB32
:1019B0000A0AE4FB068A19EB0A094FF0000A4AEB0F
:1019C0000A0AE5FB069A40F804CBD6684FF0000CF3
:1019D000E1FB067C18EB0C084FF0000C4CEB0C0CF8
:1019E000E3FB068C19EB0C094FF0000C4CEB0C0CD4
:1019F000E4FB069C1AEB0C0A4FF0000C4CEB0C0CB1
:101A0000E5FB06AC80E88017BDE8F00770470A46A2
:101A10002DE9F04F92E8F00F2DE9F30F87B091E830
:101A200039000999A0FB01784FF00009E3FB018917
:101A30004FF0000AE4FB019A4FF0000BE5FB01AB0D
:101A40000D994FF0000CE0FB01BC4FF0000EE3FBE2
:101A500001CE4FF00002E4FB01E24FF00006E5FB8F
:101A6000012600970A994FF00007E0FB018719EB68
:101A700007094FF0000747EB0707E3FB01971AEB55
:101A8000070A4FF0000747EB0707E4FB01A71BEB32
:101A9000070B4FF0000747EB0707E5FB01B70E996F
:101AA0001CEB070C4FF0000747EB0707E0FB01C7F3
:101AB0001EEB070E4FF0000747EB0707E3FB01E7BC
:101AC000D2194FF0000747EB0707E4FB0127F6198F
:101AD0004FF0000747EB0707E5FB0167CDF80480EF
:101AE0000B994FF00008E0FB01981AEB080A4FF041
:101AF000000848EB0808E3FB01A81BEB080B4FF0BC
:101B0000000848EB0808E4FB01B81CEB080C4FF098
:101B1000000848EB0808E5FB01C80F991EEB080E0A
:101B20004FF0000848EB0808E0FB01E812EB080260
:101B30004FF0000848EB0808E3FB012816EB080605
:101B40004FF0000848EB0808E4FB016817EB0807B2
:101B50004FF0000848EB0808E5FB0178CDF8089045
:101B60000C994FF00009E0FB01A91BEB090B4FF0AA
:101B7000000949EB0909E3FB01B91CEB090C4FF023
:101B8000000949EB0909E4FB01C91EEB090E4FF0FE
:101B9000000949EB0909E5FB01E9109912EB09027B
:101BA0004FF0000949EB0909E0FB012916EB090692
:101BB0004FF0000949EB0909E3FB016917EB09073D
:101BC0004FF0000949EB0909E4FB017918EB09081A
:101BD0004FF0000949EB0909E5FB0189CDF80CA09C
:101BE000089901F1100191E8390009994FF0000AB4
:101BF000E0FB01BA1CEB0A0C4FF0000A4AEB0A0AA0
:101C0000E3FB01CA1EEB0A0E4FF0000A4AEB0A0A78
:101C1000E4FB01EA12EB0A024FF0000A4AEB0A0A5F
:101C2000E5FB012A0D9916EB0A064FF0000A4AEB74
:101C30000A0AE0FB016A17EB0A074FF0000A4AEBB9
:101C40000A0AE3FB017A18EB0A084FF0000A4AEB94
:101C50000A0AE4FB018A19EB0A094FF0000A4AEB71
:101C60000A0AE5FB019ACDF810B00A994FF0000B73
:101C7000E0FB01CB1EEB0B0E4FF0000B4BEB0B0B05
:101C8000E3FB01EB12EB0B024FF0000B4BEB0B0BEA
:101C9000E4FB012B16EB0B064FF0000B4BEB0B0B91
:101CA000E5FB016B0E9917EB0B074FF0000B4BEBAD
:101CB0000B0BE0FB017B18EB0B084FF0000B4BEB21
:101CC0000B0BE3FB018B19EB0B094FF0000B4BEBFC
:101CD0000B0BE4FB019B1AEB0B0A4FF0000B4BEBD9
:101CE0000B0BE5FB01ABCDF814C00B994FF0000CCA
:101CF000E0FB01EC12EB0C024FF0000C4CEB0C0C77
:101D0000E3FB012C16EB0C064FF0000C4CEB0C0C1B
:101D1000E4FB016C17EB0C074FF0000C4CEB0C0CC8
:101D2000E5FB017C0F9918EB0C084FF0000C4CEB15
:101D30000C0CE0FB018C19EB0C094FF0000C4CEB88
:101D40000C0CE3FB019C1AEB0C0A4FF0000C4CEB63
:101D50000C0CE4FB01AC1BEB0C0B4FF0000C4CEB40
:101D60000C0CE5FB01BCCDF818E00C994FF0000E0F
:101D7000E0FB012E16EB0E064FF0000E4EEB0E0EA2
:101D8000E3FB016E17EB0E074FF0000E4EEB0E0E4D
:101D9000E4FB017E18EB0E084FF0000E4EEB0E0E2A
:101DA000E5FB018E109919EB0E094FF0000E4EEB7A
:101DB0000E0EE0FB019E1AEB0E0A4FF0000E4EEBEA
:101DC0000E0EE3FB01AE1BEB0E0B4FF0000E4EEBC5
:101DD0000E0EE4FB01BE1CEB0E0C4FF0000E4EEBA2
:101DE0000E0EE5FB01CE079800F11C0181E8C45FEF
:101DF000BDE8F80380E8F8030AB0BDE8F08F00BF43
:101E00004FEA410C7FEA6C5C02D150EA013C0AD1F6
:101E10004FEA430C7FEA6C5C02D152EA033C02D1E8
:101E20004FF0000070474FF001007047704700000E
:101E300038B5124A124D134B107829781B8820F0C0
:101E40000C041C4381F00101297064B243F30723A1
:101E5000154679B11C43E4B2844203D020460AF00F
:101E60008FFF2C704FF4FA72BDE8384006490748DE
:101E70000FF00EBC24EA0304EDE700BF14000220BB
:101E800039000220943902203C000220C87B022045
:101E900010B590B90EF03AFE0DF08AFD044650B12F
:101EA000084909486823094A00F040FF21460848CC
:101EB00000F03CFFFEE717F019FABDE810400120E2
:101EC00000F05EBFD0520600D9520600C252060092
:101ED000F852060001460020FFF7DABF0D4A10B5A0
:101EE0001278B2B90C4AD2E8AF2F92B10378012B25
:101EF0000CD10CF01BF9044658B10146074800F01C
:101F000015FF2046BDE81040FFF7E4BF0CF0ECF8E9
:101F1000F1E710BDAE000220B00002202D540600F3
:101F2000334B70B51B78002B40D0324C324D2368B8
:101F30002A68934212DA314A08401688B6F5406F93
:101F400004BF40F604061680C20714D503215A1CAC
:101F500022602B4A2B48D15400F0E8FE22682B68FF
:101F60009A4233D1BDE870404FF40062234B2648BB
:101F70001A800FF011B9860706D504215A1C226079
:101F80001F4A2248D154E7E7480706D501215A1CC9
:101F900022601B4A1E48D154DEE70A0716D50221EB
:101FA0005A1C2260164A1B48D154D5E74B070DD561
:101FB000194C204600F098FA40B9184D227E297835
:101FC000914203D0012A02D0022A0BD070BD144ADC
:101FD000144B9A60062213485A60FFF77FFF237E56
:101FE0002B70F3E7104A0F4B9A600B22F3E700BF08
:101FF000AE000220000002200400022094390220DA
:10200000D800022038500600E400022042500600AA
:102010004C50060056500600B8000220380002203E
:1020200060500600180002206750060073B5044691
:1020300001A968460AF010FE009911F008051BD1AD
:102040000E4BD3E8AF3FBBB1636820465B6898474F
:102050000B4E636832469B68294620469847094BD9
:1020600096F8512007485A60DA689E60013208BF2E
:102070000122DA60FFF732FF02B070BDB00002202B
:102080005C0002202800022073B501780446042970
:102090004CD008D802292BD046D8012923D080481B
:1020A00000F044FE22E0072900F0D98003D805297A
:1020B000F5D17C4818E0082900F0D380FF29EED143
:1020C0004168794800F032FE0022784BD3E8EF1FD8
:1020D000C3E8E02F0028F9D10F22754B60681A8001
:1020E000FFF7F8FE02E0734800F020FE02B070BD7A
:1020F000714E724800F01AFE3578002DF6D101229B
:1021000029466F480FF01AF84FF44062684B6D484B
:102110001A80012333706C4BE2681D606B4B1A60B0
:1021200000F004FE6A48DFE76A48DDE76A4800F02D
:10213000FDFD08225E4B0DEB02041A80012304F81A
:10214000083D20460BF0B6FF054630B10146634816
:1021500000F0ECFD2846FFF7BDFE002320468DF879
:1021600000300BF0A7FF044630B101465B4800F099
:10217000DDFD2046FFF7AEFE59480EF001F80023C2
:10218000ADF80430012304468DF8043008BB5449EF
:10219000544800F0CBFD54480DF0F2FF04460028EF
:1021A00047D151494F4800F0C1FD00224F4B5049E3
:1021B0001A700122996091F85110DA6059604D4B04
:1021C0001A703A4BD3E8EF1FC3E8E02F00288DD0F8
:1021D000F8E7494800F0AAFD636801A91B68474A6F
:1021E00020469847014608B14548D2E76368204633
:1021F0005B689847014650B1424840F26B23424A1F
:10220000424900F093FD424800F090FDFEE763680C
:10221000374A9B68204698470028BCD0394840F28E
:102220006E23394A394900F081FD3A4800F07EFDBD
:10223000FEE70023ADF8043001238DF80430436835
:102240005B6843B101A9344A9847014628B9204642
:1022500000F0A0F9A9E76FF085012948A3E72F480E
:1022600042E72F4800F062FD0023104AD2E8EF1F3A
:10227000C2E8E03F0028F9D10D4A2A491380D1E88D
:10228000EF3F43F00102C1E8E02F0028F7D1DB0760
:102290003FF52CAF083924480EF03EFB26E700BF7F
:1022A000AD520600285206008C520600B0000220F3
:1022B0009439022091500600AE000220B45006006E
:1022C000E4000220DC50060000000220040002208E
:1022D0000751060027510600465106005B510600D3
:1022E0007F510600875106001D520600280002207B
:1022F0005C00022018000220A05106002D200400DE
:10230000B2510600D9520600C2520600D052060051
:10231000D9510600FA5106002D1E0400475206004E
:102320006652060010000220C87B0220002310B570
:1023300088B08DF800308DF8043001238DF8053019
:102340008DF8083002234FF480628DF8103001AB15
:10235000059302AB069304AB0793094B06A8CDF88F
:102360000CD01A800BF070FE044630B101460548CF
:1023700000F0DCFC2046FFF7ADFD08B010BD00BF4B
:102380009439022073500600012000F0F9BC0120AE
:1023900000F0F6BC8FB53D4800F0C8FC3C480AF0A0
:1023A0006BFC014610B13B4800F0C0FC0AF002FC97
:1023B000014610B1384800F0B9FC0F2100200AF0A6
:1023C000D5FC014610B1354800F0B0FC3449354821
:1023D0000FF00CF90022344B34491A60C3E90112A2
:1023E00033484FF4FA722F490FF052F9314B04ACD5
:1023F00044F80C3D20460BF007FE50B12E4840F249
:1024000083132E4A2E4900F091FC2E4800F08EFCDA
:10241000FEE72D4800F08AFC4FF480622B4B1A80B7
:102420000DF072FA50B1244840F24B23234A24495C
:1024300000F07CFC264800F079FCFEE7254EFFF713
:1024400075FF3746DFF89C800BF098FE3378CBB1F0
:10245000002140460EF0C8FEA0B91F4B8DF80400C5
:102460001B68204602931D4B03930BF0F9FD0546B4
:1024700030B101461A4800F059FC2846FFF72AFD02
:1024800000233B7002F0C2F9DEE700BF14530600E0
:10249000211F040029530600555306007E530600F1
:1024A000311E04003C000220080002202D230400FD
:1024B000C87B022089200400D9520600C2520600BF
:1024C000D0520600A6530600D253060094390220CB
:1024D000E5530600AE00022004000220D8000220CE
:1024E00008540600E4000220F0B5254E0546306889
:1024F00087B0436803219B689847044628B1214868
:1025000000F014FC204607B0F0BD30686A4643680E
:102510000321DB689847044608B11B48F0E705989B
:10252000FDF762FF14A3D3E90023FEF7F1F8064696
:1025300004980F46FDF758FF02460B4630463946D1
:10254000FDF706FE06460F460022C5E904670F4B5D
:10255000FEF73AFA58B90E4B002230463946FEF7DC
:1025600029FA002814BF022303232B76CAE701238C
:10257000FBE700BFAFF300800000000080842E4125
:10258000FC0002204A5406006654060000001C406D
:1025900000001CC0014B1860704700BFFC00022007
:1025A00008B50446084611461A46A0470EF0C0FD7D
:1025B00002F0AAF970B50C254D43C66890F90B00DE
:1025C00074198842A8BF21464FF0200492FBF4F40E
:1025D000B8BF715902F01F0001EB8401196070BD92
:1025E00007B501ABFFF7E6FF0123019A03FA00F0FC
:1025F00013680343136003B05DF804FB07B501AB38
:10260000FFF7D8FF0123019A03FA00F0136823EAC9
:102610000003136003B05DF804FB10F0010005D067
:102620004FF02003EFF3118083F3118870472DE9F9
:10263000F8430446FF2200214FF00C0E4368058941
:1026400000685D4394F80AC02844E2728C4505DCBA
:1026500000252389AB4222DCBDE8F883B5FBF3F209
:102660000EFB01F7D4F80C801F2A08EB0706C8BF41
:102670001F324FEA930306F10409C8BF520903F160
:102680000303C6E9019923F00303D4BFE17248F8BC
:10269000070001F10101C8BF00EB8200D6E76268C4
:1026A000E3686A4320681E1D811886509A68204698
:1026B0004A609A68116099602A460021FFF790FFEE
:1026C0000135C6E72DE9F04F8BB0867A00AFC7E938
:1026D0000232B3000A3303F4FF63ADEB030DE946A6
:1026E000436804464846033323F0030340F80439A3
:1026F0004FF0FF3500234FF00C0C5A1E9E427A62B9
:102700000ADD2BB102689208033222F00302426014
:1027100050F8042F8A420BD27B6A013313D1002375
:102720006FF00B003A6D13602C37BD46BDE8F08F9B
:10273000E2680CFB032202F1040E5268724518BFD6
:102740001D460133D9E76E1CE9D0207CFFF765FFF9
:102750000C236B431A1DE368386213441E68B342AE
:1027600077D0D6E900131960316859F825204B60FD
:1027700023682946F31A93FBF2F22046FFF73EFF47
:10278000A9EB890305F1010B3B6109EB85057A6A29
:102790000BF1FF339A4216DC237CD90702D53B6A42
:1027A00083F31188FB6800201A467B6A13607A6AFB
:1027B000236859F82220F31A93FBF2F3BA681360E6
:1027C0003B6D1E60B0E7236855F8042BF31A93FBAA
:1027D000F2F34FF0010A9B003A69BB6105EB450338
:1027E00013447B61D5F8008059460AFB08F3FB616E
:1027F000F3187B60BB6920460AEB0302FFF7F0FE8B
:102800007B68226808F1FF389844A8EB0208218908
:1028100062684A4390450AD2E2687969F8690A44D5
:10282000111D31509168596091680B6093600AF1F5
:10283000010ABAF1040FD5D1237CD80702D53B6A2F
:1028400083F31188207CFFF7E8FE0BF1010B38625F
:102850009DE7013D6A1CA6F10C037FF47FAF0026C3
:102860009AE700002DE9F04F87B0837A00AF9B0014
:102870000A3303F4FF63ADEB030DE94643680446F6
:102880004D460120033323F00303C9F80030814291
:1028900021D2207C0D461646FFF7BFFE804659F830
:1028A00025302089FB60FA68236802FB06FB013AA9
:1028B00002EB0B01BA60626803EB0B0A42439142E0
:1028C00012D33D48A2233D4A3D4900F02FFA3D482E
:1028D00000F02CFAFEE72B6801309B08033323F04D
:1028E000030345F8043FD2E73246294620467B6081
:1028F000FFF776FE0C23E26803FB05227B68111DBF
:1029000043F80B109368CAF804309368C3F800A02A
:10291000C2F808A0237CDA0701D588F31188207C4F
:10292000FFF77BFE8046002D3DD007F114033246B1
:1029300029462046FFF73EFE042390FBF3F07A6918
:1029400083001068D84000F00F000F282BD14FF003
:10295000000A26F00303F96803EB0A0201FB02FBFD
:10296000B968B4F808C00BEB0100616801FB0CF119
:1029700088420FD2294620467B60FFF73FFE22683F
:102980007B6802EB0B0152F80B004968086052F8B3
:102990000B2051600AF1010ABAF1040FDBD1013DAD
:1029A00096FBFAF67BE7237CDB0701D588F31188D9
:1029B0001C37BD46BDE8F08FD95206008154060091
:1029C000B5540600F7520600002070470B6801332B
:1029D0000B60014B1B681847D0D402202DE9F04F43
:1029E00085B00E9C9B46012CB8BF0124012B0CBF67
:1029F0003023202315468046894601260A270022D7
:102A0000DFF870A0019402930AF101040AB9AA4503
:102A10001ED2B5FBF4F049463030C04701220136E2
:102A2000B5FBF4F10A23013F012F04FB1155BAFB5A
:102A3000F3FAE9D1494605F13000C047BBF1030F75
:102A400003D1019B9C1B002C0FDC05B0BDE8F08F6F
:102A5000019BBB42E4DBBBF1020FE1D8494602987F
:102A600003920136C047039ADAE749462020C0475F
:102A7000013CE8E7FFC99A3B30B58A680C68551CF1
:102A800014B14B68934201DC8D6030BD013B934231
:102A900008BF00228D600CBFE254A054F5E700008F
:102AA000014B1860704700BFD0D402202DE9F04FD1
:102AB0004FF0000A06460F464FF0FF39D04689B066
:102AC0001C46531E0493002505E06DB9252800F02F
:102AD00011813946B047049B13F8010F0493002875
:102AE000F3D109B0BDE8F08F642861D019D8392836
:102AF0000AD8312850D22D283CD030283DD0252866
:102B000008D13946B047DEE7582800F088806328AE
:102B100000F0EA8039462520B047049B39461878F2
:102B2000F0E7702871D006D8692841D06C283CD0D5
:102B30006828D0D0EEE7752857D017D87328E9D188
:102B4000236804F1040B1C46254615F8010B0028E8
:102B500040F0BF80B8F1030F40F0D580E41AA9EB34
:102B60000404002C00F3BB805C46ACE7782856D008
:102B70007A28DEE74FF00308ADE7B9F1000F0EDA6F
:102B8000B8F1000F00F0BC80A0F13009B8F1000FDF
:102B900008BF4FF002089EE7B9F1000FF4DB0A23EB
:102BA00003FB0909A9F13009F0E70AF1010A92E7EC
:102BB000BAF1010FC5BF073424F0070325681D686B
:102BC000D4BF043403F10804002D05DA39462D2062
:102BD000B0476D4209F1FF3943462A46CDF80090CF
:102BE00039463046FFF7FAFE6DE7BAF1010FC5BF6F
:102BF000073424F0070322681A68CCBF03F10804E5
:102C00000434CDF800904346EAE739463020B04717
:102C100039467820B0474FF008094FF001080822E4
:102C2000BAF1010FC5BF073424F00703236803F18D
:102C30000804CABF1B68059305934FF00003934631
:102C4000D8BF0434039307930BF1FF3B059B4FEA76
:102C50008B0023FA00F010F00F0009D1079B13B985
:102C6000BBF1000F24D14FF0300C07E0069AEBE7E0
:102C700009288CBF4FF0570C4FF0300C3946604498
:102C80000692B047039B079501330393BBF1000FF6
:102C9000ECD1B8F1030F7FF416AF039BC3EB4905EA
:102CA000002D7FF710AF39462020B047013DF7E7F0
:102CB000531E91450693E9DBB8F1010F03D1394664
:102CC0003020B047E2E7B8F1020FDFD139462020CB
:102CD000F7E7394603932C46B047039B34E7394660
:102CE0002020B047013C3CE72068251D3946B0470D
:102CF0002C46E8E6AA46A8464FF0FF390125EAE649
:102D00004FF00108E7E65C460546E4E6002313B50C
:102D100002AC44F8043D02460B4603482146FFF747
:102D2000C5FE02B010BD00BFCD2904000FB407B529
:102D300004A951F8040B0191FFF7E8FF03B05DF817
:102D400004EB04B0704700000CB430B5002585B02A
:102D500008AB53F8042BCDE90101044601A907484B
:102D600000930395FFF7A2FEDDE902309842B8BF59
:102D7000255405B0BDE8304002B07047792A040000
:102D800008B504464FF02002EFF3118382F3118857
:102D900001F003FA204601F04BFE0348FFF7C6FF9F
:102DA00001F034FDFCE700BFCF540600704700007F
:102DB00010B54FF02003EFF3118483F3118800F076
:102DC00011F80122054BC3F840254FF0FF32044BA8
:102DD0009A62DA6284F31188002010BD00900340EB
:102DE00000ED00E0074AD2F8883043F47003C2F8DF
:102DF0008830BFF34F8FBFF36F8F034B034A1A60C6
:102E0000704700BF00ED00E0D4D402200090D00352
:102E100008B5034A034B4FF4E871034810F07EFAFB
:102E20002F55060066550600745506002DE9F84337
:102E30000646914629B9494B494AB321494810F001
:102E40006DFA04792420484D00FB045090F82000CE
:102E5000002840F081800868421C0DD01F2801D94D
:102E6000FFF7D6FF01234FF0030C404F8340BB60B8
:102E700000F1800347F823C04F687B1C09D01F2F47
:102E8000EED84FF0000EDFF8E4C007F180034CF8F5
:102E900023E091F814E091F815C033688A694EEA8E
:102EA0000C0CBEF1010FC3F82425C3F86CC5C3F8A0
:102EB0000C05C3F8147523D18F68781C09D01F2F17
:102EC000CED84FF0000EDFF8A4C007F180004CF818
:102ED00020E0C868421C0FD01F28C1D84FF0010C59
:102EE0004FF00308DFF884E00CFA00FCCEF808C0CD
:102EF00000F1800C4EF82C80C3F80805C3F810755B
:102F0000242363430969E818C0F80490E950B9F133
:102F1000000F10D000233068C0F81031C0F8203105
:102F2000C0F82431C0F84431114BC0F8043340F3E9
:102F3000073001F0B3FB082233680E48C3F80025C0
:102F40002423002203FB0453C3E906225A61012211
:102F500083F82020BDE8F8830748FBE7B555060055
:102F600048550600BE550600000102200025844099
:102F7000100302000000AD0B0500AD0BF8B52423D3
:102F8000284C0579274603FB054393F82060012E62
:102F900006D04FF48271244B244A254810F0BEF924
:102FA00021B9244B214A40F20511F6E722B9224B00
:102FB0001E4A4FF48371F0E715B9B2F5803F04D390
:102FC0001E4B1A4A40F20711E7E701F06043B3F1E4
:102FD000005F20D1656905BB03686261C3F82051B9
:102FE000C3F85851C3F84415C3F848256268A16076
:102FF0009E60A2B9D3F82011D3F8582129B9002A2C
:10300000F8D00F4800237B61F8BD0D480D4B002A16
:1030100008BF1846F6E70C48F6E70C48F4E70948FD
:10302000F2E700BF000102200956060058550600CD
:10303000BE550600335606003A56060045560600B1
:103040000800AD0B0000AD0B0A00AD0B0B00AD0B83
:103050000023C0E900337047036823B901600023EF
:1030600041600B60704743681960F8E7006870477B
:1030700003680BB11A680260184670470020704759
:1030800007B5002202A941F8042D08480DF09EF969
:1030900010B100F085FA0190019818B10123436046
:1030A0000023038103B05DF804FB00BF603A0220F7
:1030B00001F02AB908B5034A034B4FF405710348E0
:1030C00010F02CF9BF560600D6560600F35606003F
:1030D00030B56FF0010300240A4D87B0CDE90243FB
:1030E0004FF44072084BCDE90444CDE90044074950
:1030F00028460EF041F9284605490EF00BF9204606
:1031000007B030BD98390220E9330400A07E0220C8
:10311000CE56060008B500F02FFABDE80840014879
:10312000FFF796BF300102202DE9F0471F4D204EDA
:10313000761B3609092E06D91E4B1F4A4FF489719A
:103140001E4810F0EBF81E4BD3E8EF4F621CC3E8AB
:10315000E12F0029F8D1A4B90423342219491A48CF
:103160000DF022F9194B1A4A4FF400401A60A1469B
:1031700000F022FE4FF001082346DFF858A0B342CA
:1031800001D1BDE8F0876F685C1C3C712B7B4BB1B3
:103190002B689B6803B19847C7F8009087F80580B3
:1031A0008AF8008023461035E9E700BFF44F060097
:1031B000045006002B570600B6560600F3560600CC
:1031C0002C010220D07D0220443A0220D8D40220D3
:1031D000B1300400240102202DE9F843254B0446B8
:1031E0001878F0B14FF02003EFF3118683F31188C4
:1031F0002148FFF73DFF054686F3118858B11F4B64
:10320000D3E8EF2F013AC3E8E12F0029F8D154B1F8
:10321000284600F043FA1848FFF728FF003018BF8F
:103220000120BDE8F883164A164B90469946164E83
:10323000164FB61AFF1A3609FF08B442E8DA210120
:1032400008EB010043685B7993B16B899B09BB4232
:1032500001D3FFF72FFFAA7A09EBC3031B7902F012
:1032600007029A4204D858F8013029461B6898474B
:103270000134E2E72401022030010220280102206B
:10328000F44F0600E44E060004500600F44F06001A
:10329000164B70B51B68418105469847144CE86091
:1032A000D4E8EF3F0133C4E8E23F002AF8D14FF001
:1032B0002003EFF3118683F311880E482946FFF7A8
:1032C000CBFE86F311880C4B1B7823B1BDE8704010
:1032D0000020FFF781BF23680A2B06D1074B18682F
:1032E00018B1BDE870400DF0FDBE70BDD8D402200D
:1032F0002801022030010220380102203C01022076
:1033000070B504460E461546FFF7BAFE58B10122C5
:103310000461447A466162F3071444722946BDE8A9
:103320007040FFF7B5BF70BD2DE9F04105468846F6
:1033300017461E46FFF7A4FE60B102230561457AD9
:10334000C0E9058763F3071545723146BDE8F041D2
:10335000FFF79EBFBDE8F0812DE9F8430546894699
:1033600090461F46BDF82060FFF78AFE68B1032330
:103370000561457AC0E9059863F307154572C76191
:103380003146BDE8F843FFF783BFBDE8F88310B5C9
:103390001C4600F095F920B12146BDE81040FFF72A
:1033A00077BF10BDF8B50D4F3C7864B90C4E0D4D8C
:1033B000AD1B2D09AC4207DB01233B700020FFF75A
:1033C0000BFF0028FAD1F8BD2301F01842685279AA
:1033D00012B1F3585B6898470134EBE738010220DB
:1033E000F44F06000450060008B5FFF79DFE0DF0EF
:1033F0009FFE094A106028B1084B1B68092B01DDAC
:103400000DF070FE0020FFF7E7FE0028FAD14FF420
:103410007A700DF0F9FDF5E73C0102202801022049
:10342000044A054B9B1AB1EBD30F34BF52F831005D
:1034300000207047E44E0600F44F060073B50022EA
:10344000064601A90F480CF0C1FF0546B8B9012294
:10345000019BD3E8EF1FC3E8E02F0028F9D1019CBE
:103460002D22231D1846314610F068FD7E220346AA
:1034700084F8312084F83250184602B070BD024BF7
:10348000FAE700BF443A02205E570600054B984217
:1034900005D39C3398428CBF002001207047002048
:1034A000704700BFD47D022007B504380190D0E8F2
:1034B000EF3F5A1EC0E8E12F0029F8D1012B03D1BC
:1034C00001A903480CF0AAFF03B05DF804FB00BF9C
:1034D000443A02202DE9F8431C4603890E46DB08D6
:1034E000A3429DF8207003D800231360BDE8F88341
:1034F00011682144994284BF191B11600C2BD2F82A
:10350000009028D9072CD0F814802BD80823183025
:103510004B4528BF4B4620441D461A46FFB1314655
:10352000FDF768FCA9EB05092E44B9F1000FDDD0C9
:10353000C4F11C054D4528BF4D46201D40442A4678
:10354000BFB13146FDF756FCA9EB0509D8F800805C
:103550002E440024E9E714304FF00008D8E7014674
:103560003046DDE7083C1B2CDFD9D8F800801C3C36
:10357000F9E701463046E5E7202302491A460248AA
:103580000CF012BFA0810220603A02200430D0E883
:10359000EF3F0133C0E8E23F002AF8D17047000056
:1035A000002373B5094E02AC44F8043D0120FFF737
:1035B00013FE00220546214630460CF007FF08B1F5
:1035C000002DF3D1019802B070BD00BF603A022017
:1035D00007B5002202A941F8042D05480CF0F6FEBB
:1035E00010B1FFF7DDFF0190019803B05DF804FB17
:1035F000603A0220407A00097047437A1B098B42E7
:1036000016D9032B03D800EB8101486970470129C3
:1036100003D800EB810188697047436902390629A4
:1036200003D803EB81014868704707391B68F6E748
:10363000002070477FB5047A457A14F001040190A8
:103640004FEA151510D0019B1A7A920706D55B69CF
:1036500004AC114D44F8043D039BB3B901A90E48D5
:103660000CF0DCFE04B070BD002DECD0AC42019833
:10367000E9D22146FFF7C1FF0646FFF707FF10B169
:103680003046FFF711FF0134F0E71E682146284657
:103690000CF0C4FE0396DFE7603A02200346021DE9
:1036A000D2E8EF1F0139C2E8EC1FBCF1000FF7D1DF
:1036B0005B680BB9FFF7BEBF704700697047000039
:1036C0002DE9F74F0E2A00900D46164609D92F48CE
:1036D000D0232F4A2F49FFF729FB2F48FFF726FB5E
:1036E000FEE7FFF775FF044658B300274FF00002CE
:1036F00067F3071201234272A6F1020A022200F1C7
:10370000140B5946D146436002724761BAF1000F6B
:103710000DDC009B032E2361637A66F3071363724B
:1037200019D8B20029465846FDF764FB09E001911B
:10373000FFF74EFF0199804638B92046FFF77AFF20
:103740004446204603B0BDE8F08F0860AAF1070A9E
:1037500007600146DAE74E462B68D4F81480A3616F
:103760006B680835E361072E374628BF07274FEA05
:103770008709294608F104004A46FDF73BFBF61B82
:103780004D44D8F80080EED1DBE700BFD9520600E7
:1037900075570600AC570600F752060013B5002413
:1037A0000094FFF797FE02B010BD00000EB403B501
:1037B00003AB53F8042B014604480193FFF776F955
:1037C000002002B05DF804EB03B07047B13A04008A
:1037D0002DE9F0478EB00EAF81460D46FFF76DFF25
:1037E00006464846FFF706FF4FF000088246830072
:1037F0000E3323F00703ADEB030D0EACD04516D10D
:103800004846FFF7F7FE0F281ED8DFE810F0190032
:10381000200026002D00360041004E005D006E00A5
:1038200081009600AD00C600E100FE001D0141468A
:103830004846FFF7E2FE44F8280008F10108DDE7FA
:1038400031462846FFF7B2FFBD46BDE8F087226843
:1038500031462846FFF7AAFFF6E7D4E900233146B0
:103860002846FFF7A3FFEFE7A36831460093D4E9AA
:1038700000232846FFF79AFFE6E7E3683146019305
:10388000A36828460093D4E90023FFF78FFFDBE706
:10389000236931460293E36828460193A3680093A5
:1038A000D4E90023FFF782FFCEE763693146039333
:1038B000236928460293E3680193A3680093D4E93F
:1038C0000023FFF773FFBFE7A369314604936369E1
:1038D0002846039323690293E3680193A368009346
:1038E000D4E90023FFF762FFAEE7E36931460593B1
:1038F000A369284604936369039323690293E368E9
:103900000193A3680093D4E90023FFF74FFF9BE7DF
:10391000236A31460693E36928460593A369049315
:103920006369039323690293E3680193A368009397
:10393000D4E90023FFF73AFF86E7636A314607932D
:10394000236A28460693E3690593A3690493636990
:10395000039323690293E3680193A3680093D4E976
:103960000023FFF723FF6FE7A36A31460893636ADA
:1039700028460793236A0693E3690593A369049392
:103980006369039323690293E3680193A368009337
:10399000D4E90023FFF70AFF56E7E36A31460993AB
:1039A000A36A28460893636A0793236A0693E36928
:1039B0000593A36904936369039323690293E368FE
:1039C0000193A3680093D4E90023FFF7EFFE3BE7E0
:1039D000236B31460A93E36A28460993A36A089346
:1039E000636A0793236A0693E3690593A3690493C3
:1039F0006369039323690293E3680193A3680093C7
:103A0000D4E90023FFF7D2FE1EE7636B31460B9328
:103A1000236B28460A93E36A0993A36A0893636AAF
:103A20000793236A0693E3690593A3690493636983
:103A3000039323690293E3680193A3680093D4E995
:103A40000023FFF7B3FEFFE6A36B31460C93636BD5
:103A500028460B93236B0A93E36A0993A36A08939E
:103A6000636A0793236A0693E3690593A369049342
:103A70006369039323690293E3680193A368009346
:103A8000D4E90023FFF792FEDEE670B50546002676
:103A900043681C68D5E90120214630442B685268F0
:103AA0009847241A0644F5D16B681C6070BD00006D
:103AB00008B5D1E901321B68D0544A681368013354
:103AC0001360CA68934205D9054B064A3921064856
:103AD0000FF024FC02D10846FFF7D7FF002008BDF5
:103AE00041580600B7570600715806002DE9F04FFF
:103AF0000B7A8BB003F00503052B04460D461646E2
:103B000000F08F8012F0020702F0010902F00808AD
:103B100006D07707CA6859D49249FFF747FE07468F
:103B2000B9F1000F0AD0AB7A8F4A03F0070352F8BD
:103B300023201AB18D492046FFF738FEAB7AB5F83D
:103B40000A90C3F3C20A4FEA9919B8F1000F09D0DD
:103B5000874A03F0070352F8232086492046FFF7DF
:103B600025FE804649465046FFF75AFC82490246E8
:103B70002046FFF71BFE804447442B7AD90752D4D6
:103B800021462846FFF724FE2B7A03F00503052B78
:103B900016D0F1070BD5AB7A734A03F0070352F83E
:103BA000233023B1754A71492046FFF7FFFDF20625
:103BB00006D4B3064CBF724972492046FFF7F6FDA2
:103BC0002046FFF762FF0BB0BDE8F08F6E4B1F6819
:103BD000002FA5D06D4B4FF4616E19684FF47A7CBD
:103BE000B2FBF1F1B1FBF7F3B3FBFEF20EFB123EB9
:103BF00007FB13130CFB03F1B1FBF7FB4FF03C0A7F
:103C000007FB1B11BEFBFAF30CFB01F1B1FBF7F74D
:103C10000AFB13E1CDE901B700915D49FFF7C6FD4D
:103C20007DE70027A9E72B7A0DF1200803F00503B3
:103C3000052B2CD1E36833B9564B574A4FF4B37177
:103C400056480FF06BFB0027B946E36842460893DD
:103C5000A1684B462846FFF7A1FD089A63681A60E1
:103C60003AB1A368134413F8017CA7F10A02574242
:103C700057412046FFF709FF089B9944002BE4D1E8
:103C8000002F81D046492046FFF790FD7CE728466B
:103C9000FFF713FD354902462046FFF787FD4FF039
:103CA0000009DFF810A108230AAA42F80C3D41469A
:103CB0004B462846FFF772FD079B002B3AD0F306D0
:103CC00006D4B0064CBF2E492E492046FFF76EFDA4
:103CD0004FF0000B5F4533DC4FF0000B079B9B451B
:103CE00035D218F80B202F492046FFF75FFD0BF166
:103CF000010BBBF1080FF1D12B492046FFF756FD10
:103D00004FF0000B079A934526D218F80B20059226
:103D10000FF044FB059A10444178204611F0970FAC
:103D200008BF2E222149FFF741FD0BF1010BBBF12A
:103D3000080FE7D1079B072B7FF626AF9944B2E720
:103D400051462046FFF732FD0BF1010BC2E718493F
:103D50002046FFF72BFDCAE751462046FFF726FD18
:103D6000E3E700BFE8570600D4570600F7720600E5
:103D7000AC5806000D580600135806003C580600C3
:103D80002B5806002A580600400102204401022058
:103D9000F157060017580600C05706007158060074
:103DA000285806002D5806003758060039580600D6
:103DB000335806003558060001230021074A10B584
:103DC000074C1360A04204D801B11360054B186082
:103DD00010BD40085B000121F4E700BF4401022050
:103DE00040420F0040010220F8B50D461646044639
:103DF0004718A74201D12846F8BD736814F8011B83
:103E00005B6830469847F4E77047000010B50C46F1
:103E10000846FFF7BBFB214604480F22FFF766FE6A
:103E20002046BDE81040FFF739BC00BF50590600DE
:103E300008B506480CF0A4F928B9054B054A382105
:103E400005480FF06BFA054B586008BD0459060091
:103E50000B590600E05806000F59060054010220D5
:103E600008B548B90C4811230C4A0D49FEF75EFF0E
:103E70000C48FEF75BFFFEE70B4B1A684AB1064899
:103E80001223064A0949FEF751FF0648FEF74EFF86
:103E9000FEE7186008BD00BFD95206007159060040
:103EA000FD700600F75206007C3A0220B759060062
:103EB00008B500F029FA064BD3E8EF2F0549511851
:103EC000C3E8EC1FBCF1000FF6D1104408BD00BFE1
:103ED0005C0102200DCA9A3B43685B6818470020CA
:103EE000704700000A4B70B5C6B204461B683046E6
:103EF000984701280AD00A2C064D03D10D212868C5
:103F0000FFF7EAFF31462868FFF7E6FF204670BD5D
:103F1000DCD402206001022010B5044C204600F0E1
:103F200005FE2046BDE81040FEF7BABDE53E0400A0
:103F300008B504480CF024F9034B1860FFF7ECFFB8
:103F4000002008BD045906006001022010B54FF0A2
:103F50002003EFF3118283F31188114C237823B9E6
:103F600082F311886FF0770010BD013BDBB2237044
:103F700023B182F311886FF00F00F5E7094B01219F
:103F8000187828B1217082F311886FF00A00EBE7EE
:103F9000197082F31188044A11601870E4E700BFB9
:103FA00066010220650102200450004010B54FF068
:103FB0002003EFF3118283F311880F4C207880B136
:103FC00082F311880D4AD2F81C34D2F8182403F079
:103FD000030343F48033934314BF6FF07600002053
:103FE00010BD0123237082F31188044AC2F8040132
:103FF000C2F818159360E5E7640102200050004004
:1040000008B500220121052000F06CFB052000F01E
:1040100045FB002008BD00002DE9F0414FF02003D2
:10402000EFF3118283F311882E4B18781F46441C3E
:104030001C7070B182F311883B78002B45D12A485F
:1040400068232A4A2A49FEF771FE2A48FEF76EFEC7
:10405000FEE7294D95F80080B8F1000F06D01870E2
:1040600082F311886FF00A00BDE8F08101262E70FE
:1040700082F31188214C21B3052000F01FFBC4F806
:104080000081D4F80433C4F804632660D4F8002116
:104090009AB10022DB0758BF0123C4F800214FF07A
:1040A000200258BFC4F80833154B0520C3F88021FF
:1040B00000F0F4FA00232B70BEE720BF40BF20BF02
:1040C000E4E7C4F800112660F4E70C4BD3F80C3495
:1040D00003F00113B3F1011F0CBF00206FF0760055
:1040E000C2E700BF66010220D9520600FC59060053
:1040F000435A0600F75206006501022000500040B6
:1041000000E100E038B51F4BD3F80851D3F8042381
:10411000D3F8000102F00102D3F80443D3F80411EC
:10412000EDB970B10020C3F8000132BB41B10022EB
:10413000144BC3F80421A20702D50222C3F80823B6
:1041400038BD9AB90029F2D10F4840F245130F4A01
:104150000F49FEF7EBFD0F48FEF7E8FDFEE70025EF
:10416000C3F808510028DDD1002ADFD0D3F80C3481
:1041700003F00113B3F1011FD8D10122014BC3F8A1
:104180000823D3E700500040D9520600FC5906002E
:104190004E5A0600F7520600704770474FF0200352
:1041A000EFF3118083F311887047000000230D4A5C
:1041B00010B5C2F84031FFF7F1FFD2F8043540F2F4
:1041C000471209490C681B1B23F07F43B3FBF2F332
:1041D00002FB03420A6080F311881846BDE81040D4
:1041E0000DF076BB005001406801022038B51B4835
:1041F0000BF0C6FF70B3436801211B689847002489
:1042000040F24713164D4FF40012C5F80845C5F8A3
:1042100040354FF48033C5F84433C5F80433114BAF
:1042200001211C60104B1520C3F88021224600F0AC
:1042300059FA152000F032FA012320460B4A136088
:104240002B60D5F8043503F2471323F07F43C5F8FC
:10425000403538BD4FF0FF30FBE700BF6D5A060018
:10426000005001404051014000E100E00850014091
:1042700070B54CF66905B0F1FF3F14BF02462A46FF
:10428000FFF78CFF124B134C1E68531EAB42A8BFA6
:104290002B4640F24715D4F8041523EAE3738A1B32
:1042A00022F07F4202F5A37205FB0323B3FBF5F373
:1042B00005FB0363591A21F07F411F2998BF5B1941
:1042C00023F07F43C4F8403580F3118870BD00BFF0
:1042D000680102200050014008B5FFF75FFF084B5E
:1042E000084AD3F8043512689B1A40F2471223F0AB
:1042F0007F43B3FBF2F380F31188184608BD00BF7B
:10430000005001406801022008B5FFF747FF064B47
:10431000064AD3F80435126880F31188981A20F001
:104320007F40104408BD00BF0050014068010220DA
:1043300004488168406A884203D003494FF08052A4
:104340000A607047987B022004ED00E000232021E2
:104350000348C2180133412B82F80013F9D170478A
:1043600000E100E0084A09499368096858669966BF
:1043700007494B6843F080534B60002383F3118857
:104380009368986E704700BF987B0220007D0600FE
:1043900000ED00E0202080F311880D498A684FF07D
:1043A00028001044EFF3098C80E8F01F094F4FF00C
:1043B00000664A6A8A603E60506E0023536680F34E
:1043C000118802F1280090E8F01F8CF309887047EB
:1043D000987B022004ED00E01EF0040F0CBFEFF309
:1043E0000880EFF30980816931F8021C11F0FF01A8
:1043F0000229FFD000B500F057FA00BD38B5194CBE
:1044000005461948FEF792FCA36AD90602D517485B
:10441000FEF78CFCA36A1A0702D51548FEF786FC46
:10442000A36A9B070ED51348FEF780FC616BA36A55
:10443000180607D51048FEF779FC1DB1A36A23F0D2
:104440008003A362074CA26AD20702D50B48FEF78D
:104450006DFCA36A9B0602D50948FEF767FC0020A5
:1044600038BD00BF00ED00E0DC5B0600F35B06003A
:10447000055C0600195C0600325C0600495C06001B
:10448000695C060038B51E4C05461E48FEF74EFC1A
:10449000A36AD80409D51C48FEF748FC184A002036
:1044A000936A43F47F43936238BDA36A190501D52B
:1044B0001648F1E7A36A9A0514D51548FEF736FCAD
:1044C000A16BA36A1B0407D51248FEF72FFC1DB190
:1044D000A36A23F40043A362094B9B6A5805DDD508
:1044E0000D48D9E7A36A5905FAD4A36ADA0501D5BC
:1044F0000A48D1E7A36A9B04D0D50948CCE700BF9E
:1045000000ED00E08D5A0600F35B0600055C060036
:10451000A45A0600BE5A0600D45A0600F05A0600F5
:10452000695C060010B51C4C1C48FEF7FFFBA36A33
:104530009A0102D51A48FEF7F9FBA36ADB0102D5FE
:104540001848FEF7F3FBA36ADC0202D51648FEF713
:10455000EDFB114CA36A180302D51448FEF7E6FBE5
:10456000A36A590302D51248FEF7E0FBA36A9A0337
:1045700002D51048FEF7DAFB074CA36ADB0302D52D
:104580000D48FEF7D3FBA36A00206FEA03436FEAEE
:104590001343A36210BD00BF00ED00E0995C06006C
:1045A000B25C0600C65C0600E15C0600F35C060037
:1045B000125D0600385D0600535D060070B5284D9B
:1045C00006466C68FEF7EEFEC4F30804E31E092BF2
:1045D0003AD8DFE803F0053335303939393939371E
:1045E0002048FEF7A3FBEB6A9A0703D51E48FEF7A7
:1045F0009DFB02E0EB6A5B0005D400203146BDE87C
:10460000704000F01DB91948FEF790FB184B1B785D
:104610002BB10120FFF7F2FE0628EFD170BD154B3C
:104620001B781BB10120FFF72DFFF5E7124B1B880C
:104630009BB2002BE1D0FFF775FFEDE70020E9E723
:104640000020F0E70D48D2E70D4B0E49A4F110020F
:104650000F2CC8BF19460C48FEF768FBCDE700BF1A
:1046600000ED00E0375B06004F5B0600715B060063
:1046700028ED00E029ED00E02AED00E0915B060066
:104680001E5B0600095B0600C85B0600024A536910
:1046900043F010035361704700ED00E043B2002B7C
:1046A00008DB012200F01F0002FA00F0024A5B0959
:1046B00042F82300704700BF00E100E043B2002B46
:1046C0000DDB012200F01F0002FA00F05B09044A32
:1046D000203342F82300BFF34F8FBFF36F8F704733
:1046E00000E100E04B1C072B10B50C460BD90F4A1C
:1046F0000F4910487223FEF719FB072221460E4886
:10470000FEF714FBFEE742B2002AA8BF02F16042A6
:104710004FEA4313B8BF094ADBB2ABBF02F56142AF
:1047200000F00F0082F80033135410BD7F5D0600C7
:10473000B85D0600D9520600CF5D060014ED00E01A
:1047400000F06AB808B572B6044B186A18B10022B6
:104750001A620BF041FD62B608BD00BF987B0220D3
:10476000704700002DE9F041099F05460F2F0C46C8
:104770001646984625D11C4B984526D10A9B042203
:10478000394628460CF0D0FE0023A6F16801174AEE
:10479000214421F0070122F00102C5E91333C5E9E4
:1047A00016468A61069AC1F800804A60079A8A60B4
:1047B000089ACA604FF08072CA61A9646B66BDE84E
:1047C000F08107F110031E2BD8D93C23084A094970
:1047D0000948FEF7ABFA6FF00F030E22394607487F
:1047E000FEF7A4FAFEE700BFDD010500A1250400E5
:1047F000015E0600365E0600D9520600D25E060053
:10480000014910220A60704710ED00E0404080F33B
:10481000118830BF704700BF404080F31188DFF837
:104820001CC0DCF800C01CF4006C0CBFEFF3088067
:10483000EFF3098000B5FFF7C1FE00BD04ED00E015
:1048400038B504460D46FEF7ADFD052C1AD8DFE855
:1048500004F00319191315170D48FEF767FA0CF049
:1048600067FCAA6901460B48FEF760FA2946204614
:10487000BDE8384000F01CB80748EEE70748ECE711
:104880000748EAE721460748FEF750FAE7E700BF86
:10489000015F06009F5F0600215F0600475F06007C
:1048A000615F06007C5F060001460068FFF7C8BF35
:1048B000052810B50CD00CF015FD60B10CF012FD00
:1048C0000C490D4B002808BF19460C48FEF72EFA7C
:1048D000FFF79CFFFCE70CF015FD0028EED1084C1B
:1048E0000848A168FEF722FAA068BDE8104000F071
:1048F0000BB800BFDB5F0600DF5F0600F05F06005D
:10490000987B02201060060038B505464FF0200362
:10491000EFF3118483F31188037BDB0709D510487B
:104920002523104A1049FEF701FA1048FEF7FEF958
:10493000FEE70CF061FD0E4B9B68AB420BD10D4BBB
:104940005A68C2F3080212B92046FFF70BFD5A68F5
:1049500042F080525A602046BDE838400CF0BEB8A4
:10496000D952060035600600706006009E600600A1
:10497000987B022000ED00E000B572B60B4A106A89
:1049800000281EBF002111620BF026FC62B6EFF377
:104990000580A0F110004FEAC0000549014409C993
:1049A00098475DF804EB034800470000987B02201D
:1049B000104C060031430400202080F31188064883
:1049C0004FF40061401880F30988022080F31488B6
:1049D000BFF36F8F00F006F8D0C8022030BFFFF79A
:1049E000FDBF00BF104A08B5104B22F07F029A604D
:1049F000BFF34F8FBFF36F8FD3F8882042F470025C
:104A0000C3F888204FF00042C3F83422BFF36F8F01
:104A1000B0EE400ABFF36F8F0BF0F8FB0BF000FC19
:104A2000FFF794FC0BF020FC0000040000ED00E018
:104A3000BFF34F8F0549064BCA6802F4E062134387
:104A4000CB60BFF34F8F00BFFDE700BF00ED00E07C
:104A50000400FA0508B5FFF7C1FFBDE80840FFF7FD
:104A600067BC00000522034B5A60BFF34F8FBFF3B2
:104A70006F8F704790ED00E0BFF35F8F0022014B16
:104A80005A60704790ED00E070B51F4D1F492B68CC
:104A90000C68C3F307239C4228460ED91C4A1D49C3
:104AA0001D4840F25513FEF741F92A682146C2F32A
:104AB00007221A48FEF73AF9FEE7FFF7DDFF4FF647
:104AC000AA734A6800212B638C4202F1100603D1BD
:104AD000FFF7C8FF002070BD157A56F8103C05F0AE
:104AE0001F0223F01F031A4356F8043C6D0923F0FC
:104AF0001F0343F0010343EA45038160C2600131B3
:104B000003613246E0E700BF90ED00E0F854060094
:104B1000BB60060032800600D9520600FE60060027
:104B20004FF0FF307047002070470000014B1860C5
:104B3000704700BFE4D40220F8B506460D460024B5
:104B4000064FAC4208DA3B6898470A28305504F112
:104B5000010401D00D28F4D12046F8BDE0D4022094
:104B60002DE9F04106460D4604460A4FA31B9D421F
:104B700002DC2846BDE8F0812378A0460A2B02D14A
:104B80003B680D2098473B6898F80000013498472F
:104B9000ECE700BFE4D4022008461146FFF7CCBF83
:104BA00008461146FFF7DCBF4FF0FF30704700208A
:104BB00070470120704700207047002070474FF475
:104BC000005300204B60704708B505210148FFF7EE
:104BD000C7FFFEE730610600074910B50B68C4182F
:104BE0000648C0F1005202F5802294423ABFC01834
:104BF0000C604FF0FF3010BD6C01022010E5022068
:104C00000BF0E4BA704700008279044B03EB4213C7
:104C1000DB69C01A024BC01058437047D0E4022031
:104C2000ABAAAAAA10B5094B827903EB42139B6980
:104C30000A685C6823689A4294BF0A600B60FFF7B9
:104C4000E3FFD4E9002302FB003010BDD0E40220D2
:104C50002DE9F3410546019116460CF0B3FE0746D7
:104C60004FF02003EFF3118883F311886B8A002B38
:104C70003DD02A8A9A422AD9002128460BF056FEB6
:104C8000044620B388F31188019B002B3CD0731C91
:104C9000012B06D90CF096FEC01BB04294BF361A09
:104CA000B61BA3791E4F324607EB43139B6901A93C
:104CB0001B6820461B6898470546206128BBA079E1
:104CC000214607EB40100BF02CFE2C4618E06B8AB7
:104CD0005A1E6A8288F3118818222C8AE41AEB691A
:104CE00002FB04340E4BED1A6D11A571CCE788F36D
:104CF0001188314628460BF019FE04460028C3D11E
:104D0000204602B0BDE8F081236100230122236028
:104D1000A280A381019A2369E281A360F0E700BF2A
:104D2000D0E4022083690A465B681968FFF790BFE8
:104D30008368194401607047F8B504460026144D95
:104D400004B9F8BD23792768013BDBB22371002B3E
:104D5000F7D1216959B163799B0707D4A37920461C
:104D600005EB43139B691B689B6898472661A079F4
:104D7000A66005EB40135B6926601BB1204698478F
:104D80003C46DDE7214605EB40100BF0CAFDF7E796
:104D9000D0E40220036803B970471846FAE70268B6
:104DA00010B51AB10B461C6814B91A60016010BD29
:104DB0002346F8E710B5044628B908460B790133B5
:104DC0000B7110BD18460368002BFBD1FFF7E7FFFE
:104DD0002046F6E710B508B10B68036000230C68A5
:104DE00008460B60FFF7A8FF204610BD83880268C5
:104DF00019448180D018704710B503688488234413
:104E0000144484801846FBF7F5FF10BD02688068E3
:104E1000101A704702688168C388521A80889B1AEA
:104E2000181A70472DE9F84F81460F4690469A466A
:104E300004460A9E2568EDB908342046FFF7EAFFCC
:104E4000B84294BF1FFA80FB1FFA87FB41465A46BF
:104E50002046FFF7D1FFB7EB0B075D44D8440BD0DA
:104E60000B995046B047044630B101464846FFF71B
:104E7000A1FFE1E72C46DDE72846BDE8F88F0000FA
:104E80004FF0FF32012101480CF058B970010220A7
:104E900002684AB943683BB982682AB9C06800F120
:104EA0007F435842584170470020704738B54369E6
:104EB00004460D463BB159B163699B681B7803F00A
:104EC000F003602B0DD02046BDE8384001F0F4BB64
:104ED0000146006A01F0F6F90128EDD00028F2D170
:104EE00038BD0A2294F84430294662F3C60384F898
:104EF0004430204602F06CFFF0E708B501F075FE83
:104F0000FFF7BEFF02F0F8FC03F0C8F805F024FD3F
:104F100005F056FC05F02AFA01F09EFA01F080FE39
:104F200001F04CFB002008BD2DE9F041044690B093
:104F3000002800F08A804269002A00F08680036A17
:104F4000002B00F0858090F84430C3F3C3030A2B94
:104F500071D1956802F09EFE183501461022284650
:104F60000EF042FD20B96FF07C0010B0BDE8F0817A
:104F700063699D6818352846FFF78AFF01460028B7
:104F800047D00CAE354663699A6802F108031832BF
:104F9000374618685968083303C793423E46F7D12D
:104FA00095E80F006E4686E80F0008AFBC466369BF
:104FB0009B6803F1180203F12808BE461068516887
:104FC0000832AEE8030042457746F6D1674608331B
:104FD0003A4603CAAA4218605960174603F108030B
:104FE000F6D1636904AD9F6896E80F0085E80F006D
:104FF00007F118032A4603CA62451860596015462E
:1050000003F10803F6D120460121FFF74FFF0020EE
:10501000ABE7284600F0C4F90028B2D1636998686C
:10502000037EFF2B02D1437E012BECD00830FFF72B
:105030002FFF002897D12146206A01F05BF9022852
:105040000CBF6FF0040000208FE76FF03C008CE78E
:105050006FF0150089E7002210B503680BB91846F8
:105060000BE08B421C680FD142B942680460934246
:1050700000D14460002201201A6010BD1460416814
:105080008B4208BF4260F5E71A462346E6E790F8F0
:1050900038306FF3000380F838307047D0E8AF0F36
:1050A000084100F00100704730B40D46114630B1A0
:1050B000446B24B12A46A44630BC0368604730BC28
:1050C0007047802AF8B507460E46144601D90020DD
:1050D000F8BDD5082A460EF087FC0028F7D1C4F1A8
:1050E000800414F007040FD0735D7A5DC4F10801E9
:1050F0005A40FF238B4083F0FF0303FA04F422425B
:105100000CBF01200020E3E70120E1E708B51022F1
:105110000EF06AFCB0FA80F0400908BD0A4601466C
:1051200001480CF0B5BA00BFC87B022000231A4624
:1051300005F0CAB82DE9F84F0CF044FC314B82461B
:105140001C68002C53D0B4F1140552D0246804B16B
:10515000143C4FF000084FF0FF364FF0FF37DFF8F8
:10516000A8B0DFF8A0907DB9B8F1000F48D00023B7
:10517000254ABB4208BFB24238BF164623483146D3
:10518000BDE8F84FFFF7CABF296AC1B9AB69EA6940
:10519000A3EB0A031344002B2FDC0223E96185F8FB
:1051A000453005F114014846FFF755FFA542DBD015
:1051B0000CB3636903B1143B25461C46D3E7DA45BB
:1051C00005D10CF0FFFB2B6AA861013B2B622B6A17
:1051D000002B0ADCEA690023BB4208BFB2423EBF93
:1051E00016461F464FF00108E0E75A46F3E725460A
:1051F000AFE72C46ADE72346DEE7DA45EAD1E0E744
:10520000BDE8F88F880102209BFFFF7F98010220F4
:1052100038B500230C4681F84530054680B9012396
:105220004FF00002114963F30202114B60F3C50213
:105230005B1ADB0863F38F120E490F48FEF760F824
:10524000286800210C30FFF729FF70B101232146A7
:1052500084F84630284604F00BFB30B904F12400F2
:105260006421BDE83840FFF759BF38BDE44E060061
:10527000344F06005D6106004F6406002DE9F04FD3
:10528000064680B3051D00204FF0480A844648F2C8
:10529000FE0B0AFB0C635B6C1C4C23F07D4303F09C
:1052A000FF23A3421BD135F8043C0A2B17D12B88CE
:1052B0005B4514D0002301F1FF3905F1FF3819F8DF
:1052C00001EF18F8014F03F10807A64510D1FBB212
:1052D000802BF4D114789C429CBF2846137048352B
:1052E000BCF1000F01D0BDE8F08F4FF0010CD0E70A
:1052F0008EEA0404FFB214F0800FEBD10133DBB26D
:105300006400BB42E4B2F6D1E4E700BF0001000252
:1053100043685BB109B9002070470B60FBE742604E
:10532000C2F858010029F6D00A60F4E7034AD2F81F
:105330005831002BF3D06FF002007047B801022003
:1053400010B5446854B104F0C2FC38B904F5947047
:105350004FF47A71BDE81040FFF7E0BE10BD0000C9
:1053600010B4A0F5947292F856310B480133DBB2B9
:105370000A4982F85631884202D15DF8044B7047E1
:105380004468944201D02030F5E7022BF5D85DF84F
:10539000044BFFF7D5BF00BF10E5022010E5022047
:1053A0002DE9F04106460F46174DDFF86080454570
:1053B00001D1002021E06C681CB394F847309A07B3
:1053C00008D523880A2B05D18022211D3046FFF7FE
:1053D00078FEA0B994F88F309B0712D5B4F8483006
:1053E0000A2B0ED1802204F14C013046FFF769FEF2
:1053F00038B1482007B13D602044BDE8F08100206D
:10540000F8E72035D3E700BF10E5022010E50220C1
:10541000002337B502A941F8043D0123A0F120047F
:1054200080F82130A0F124052046FFF7B9FF85421E
:1054300007D101990448FFF779FE2146019803F04E
:10544000D5F803B030BD00BF0D0060F038B544683A
:105450000D4604B394F847309A0708D523880A2BE1
:1054600005D18022211D2846FFF72BFE88B994F82C
:105470008F309B070FD5B4F848300A2B0BD1802210
:1054800004F14C012846FFF71CFE20B148202044BF
:1054900038BD0020FBE70020FAE70000F8B5012343
:1054A000044680F8453000234FF47A7063611E4B48
:1054B000A1FB0067596804F1140271BBC3E9002223
:1054C0000CF080FA194AA061002330463946FBF7F8
:1054D00007FB164B206203FB1060E06114480CF0E0
:1054E00047F94FF47A716422002380FB0101FBF736
:1054F000F7FA054620B1236AA3B9E369834211DABA
:105500000C480CF07CF8236A002B09DD45B90749EB
:105510000848BDE8F840FFF701BE0A605A60CFE7CF
:10552000E169F5E7F8BD00BF880102209BFFFF7F1E
:10553000A4010220980102202DE9F04F8FB0884687
:1055400005A9074693461C46FFF7E2FE002803DA4A
:1055500000200FB0BDE8F08F7E6896F847309807BE
:1055600000F1EF8096F88F30990700F1F380DDF8B5
:1055700014A09AF84750C5F3400525B19AF88F302A
:105580009A07E5D4012548266E430AEB060999F8E7
:1055900047300DF1180C43F0020389F847300A2315
:1055A0002AF806306346424689F844B008F11008EC
:1055B000E646106851680832AEE803004245F446FA
:1055C000F6D11A4609F1040C0DF12808134603CB55
:1055D0004345CCF80000CCF804101A460CF1080C36
:1055E000F4D106F12400644950440BF0FFFF482336
:1055F00003FB05A393F84720002C00F0B8806FF35D
:10560000000283F8472021464846FFF747FF3B68E2
:10561000DDF814A05B681C6914B13846A047044645
:10562000E30740F1828040F2FF23ADF828304FF0CD
:105630000009ADF82A90ADF82C90ADF82E90ADF899
:105640003090ADF83290ADF834904FF48073ADF8EF
:1056500036304146384604F06DFD031E1EDA13F164
:10566000780F03931AD001224FF0000B434962F3E5
:10567000020B434A69F3C50B521AD20841460A206D
:1056800062F38F1B01F024FCFDF7D8FEADF800B0EB
:105690000246039B3B493C48FDF75EFE14F00204C2
:1056A00043D140F2FF230A93ADF82C40ADF82E40D1
:1056B000ADF830404FF48073ADF83230FF238DF8F1
:1056C0003430482303FB05A56B7CB2449AF81320C1
:1056D0008DF835309AF8123043EA0223ADF83630AF
:1056E0004146384604F026FDB0F100091DDA19F1F3
:1056F000780F1AD001234FF00005214A63F3020509
:105700001E4B4146D21AD20864F3C5050A2062F343
:105710008F1501F0DDFBFDF791FEADF8005002465C
:105720004B461A491A48FDF717FE05993846314489
:10573000FFF76EFD17483946FFF7F8FC059830442F
:1057400007E7311D4046FFF7E1FC00283FF40AAFB0
:10575000002008E006F14C014046FFF7D7FC002886
:105760003FF405AF0120482303FB0060F1E642F05F
:10577000010283F847204AE711540400E44E060072
:10578000344F060086610600FA6206009A61060040
:1057900024630600010060F0102270B5044688B052
:1057A00000210DEB02000EF0AFF903A92046FFF730
:1057B000AFFD002812DA02234FF000024B4963F3D9
:1057C00002024B4B6FF3C5025B1ADB0863F38F12C7
:1057D00048494948FDF794FD08B070BD039B002B74
:1057E000FAD048F2FE032268049300230593117D4A
:1057F000062956D0082972D0022912D1517D0129DB
:105800000FD10693FF218DF81B10FE218DF81D305E
:1058100013698DF81C101A788DF81E205B788DF8AE
:105820001F300023012204A92046FFF785FE05460C
:10583000D0B901234FF000062C4A63F302062C4B2B
:1058400004A99B1ADB0860F3C5060A2063F38F16D0
:1058500001F03EFBFDF7F2FDADF800600246234685
:1058600024492648FDF778FD039991F847309A07B7
:1058700007D50B880A2B04D1A94202D02046FFF796
:10588000C7FC039991F88F309B07A5D5B1F8483034
:105890000A2BA1D14831A9429ED02046FFF7B8FC7F
:1058A0009AE71369997818888DF81A10FF218DF8F6
:1058B0001B10FE21ADF818008DF81C1033F8031FE3
:1058C000ADF81D109B788DF81F30537D032BA8D1A8
:1058D0009DF8183083F002038DF81830A1E71269A3
:1058E00006AB1068516803C3F2E700BFE44E060040
:1058F000344F0600B261060098630600C4630600D8
:1059000073B50D4601A90646FFF702FD002835DBF9
:105910002B78FF2B32D1019B93F8A40010F00100EB
:1059200008D093F8BC20D10726D593F8D420D2070D
:1059300024D4022018244443191991F8A42042F0D9
:10594000010281F8A4200A22A1F89020294604F13E
:105950009402134405F1100251F8040B914243F8EC
:10596000040BF9D106483146FFF7E0FB019B04F137
:105970009000184402B070BD0120DBE70020F9E779
:10598000030060F02DE9F84F47688046894607B369
:1059900000254FF0180A07F1940B0AFB05F03C189C
:1059A00094F8A430A034DB0710D549465844FFF7DB
:1059B000ADFB064650B1237941466FF300032371D6
:1059C0000548FFF7B3FB3046BDE8F88F0135032DDE
:1059D000E3D10026F7E700BF040060F02DE9FF41A6
:1059E000074644680E4681B901234FF0000263F375
:1059F000020261F3C502354B354936485B1ADB08B4
:105A000063F38F123449FDF77BFC002C5CD094F8D3
:105A10004730990707D494F88F309A070BD40020A9
:105A200004B0BDE8F0813146201DFFF76FFB002870
:105A3000F1D0002507E0314604F14C00FFF766FB8A
:105A40000028ECD0012548216943631893F84730BA
:105A5000DB070CD4DFF88C80143121444046FFF77B
:105A6000FAFAD8F8003013B91C480BF0C8FD4820EA
:105A700000FB054494F847306FF3410384F8473046
:105A800040F2FF2300930023ADF80430ADF8063058
:105A9000ADF808304FF48073ADF80A30FF238DF86D
:105AA0000C30737BF27B8DF80D30B37B43EA02231D
:105AB000ADF80E3069463846FFF764FF08483946AE
:105AC000FFF734FB0120ABE72046A9E7344F06007F
:105AD000E44E060051630600DA61060098010220D8
:105AE000020060F08801022030B50D4685B004AB9D
:105AF00043F8040D19462846FFF752FCE0B901238C
:105B00004FF00004124A63F30204124B29469B1A19
:105B1000DB0860F3C5040A2063F38F1401F0D8F9A1
:105B2000FDF78CFCADF800400246039B0A490B4888
:105B3000FDF712FC05B030BD24300BF060FD039979
:105B40000748FFF7F3FA29460398FFF747FFF1E705
:105B5000E44E0600344F0600C36106006D63060084
:105B60000E0060F02DE9F0411F4691F847301646CF
:105B70009A0705460C4612D50B880A2B0FD191F8CF
:105B80004430012B0BD101F104083A46414630461E
:105B9000FFF797FA18B141462846FFF71FFF94F820
:105BA0008F309B0714D5B4F848300A2B10D194F8E5
:105BB0008C30012B0CD14C343A4621463046FFF74D
:105BC00080FA28B121462846BDE8F041FFF706BF1C
:105BD000BDE8F0812DE9F74F0BF0F4FE304B804625
:105BE0001C68002C40D04FF0FF364FF0FF374FF0CD
:105BF000000A2568DFF8AC90DFF8B0B0D4E90213F2
:105C0000002B36D16268A2EB08020A44002A44DC69
:105C100094F8252001A963F3410284F82520206A25
:105C2000FFF776FB00280BDB0199206A94F82430FB
:105C300004F11002FFF796FF216A5846FFF776FA43
:105C4000AC4203D03DB32B682C4685B9BAF1000FA6
:105C50000AD00023134ABB4208BFB24238BF1646DF
:105C600011483146FFF75AFA03B0BDE8F08F1D46E0
:105C7000C4E7C84501D1013BE360E368002BC8BF1E
:105C800049460023BB4208BFB1423EBF0E461F46F5
:105C90004FF0010AD4E72B46D6E7C845F1D1EAE731
:105CA000900102209BFFFF7F24030220060060F08A
:105CB0002DE9F84F82460F464FF0180B184D194B3F
:105CC0009D4201D1002021E01FB13B680BB1AB42E6
:105CD00023D16C680CB34FF0000804F194090BFB5E
:105CE00008F6A21992F8A410CB0711D5B2F89020AB
:105CF0000A2A0DD1802209EB06015046FFF7E1F98F
:105D000030B107B13D6006F190002044BDE8F88F46
:105D100008F10108B8F1030FE1D12035CFE700BF4A
:105D200010E5022010E50220F8B50A4B05461B6875
:105D30000E46174663B11C685A68AA4204D19B6894
:105D40003A4631462846984714B123462468F3E77B
:105D5000F8BD00BF1C0302202DE9F04387B00D46BB
:105D600001A9064690461F46FFF7D2FA002803DA3B
:105D7000002007B0BDE8F08374680CB394F8473096
:105D8000990709D504F1E8012846FFF7BFF918B1D2
:105D900094F8FC30434511D094F88F309A070FD512
:105DA00004F588712846FFF7B1F948B194F8243119
:105DB000434505D12820D8302044DAE70020FAE70F
:105DC000DDF804C0BCF1000FD2D09CF8FD30C3F365
:105DD000400323B19CF825319B07C9D40123282215
:105DE0005A4302F1D804624492F8FD1082F8FC8014
:105DF00041F0020182F8FD10C2F8F8602A4602ADB7
:105E0000AE4602F11009A846106851680832A8E8A9
:105E100003004A454546F6D10CEB040210320DF161
:105E20001808754603CD454510605160AE4602F135
:105E30000802F6D1282202FB03C393F8FD200137A4
:105E40000CBF42F001026FF30002044883F8FD200A
:105E50003146FFF76BF90198AEE700BF050060F02F
:105E600070B544680D4616460CB9002070BD94F814
:105E7000FD30980711D494F825319B07F5D53246AB
:105E8000294604F58870FFF71CF90028EDD00120A1
:105E9000282303FB0040D830E8E704F1E800FFF7CF
:105EA00010F90028E7D00020F2E700002DE9F041CA
:105EB00006460F46174DDFF86080454501D10020AA
:105EC00023E01EB133680BB1AB4211D16C687CB1D9
:105ED00094F8FD309A070DD494F825319B0707D527
:105EE00094F82421394604F58870FFF7EAF850B990
:105EF0002035E2E794F8FC20394604F1E800FFF78A
:105F0000E0F80028E8D016B90120BDE8F08135603E
:105F1000FAE700BF10E5022010E50220F8B54B1C9F
:105F200004463CD000234FF47A7603601C4BA1FB5F
:105F300006675A6872BBC3E900000BF043FD194ABB
:105F40000023606039463046FAF7CAFD1549E06023
:105F500001FB1060A06014480BF00AFC4FF47A714A
:105F60006422002380FB0101FAF7BAFD054620B147
:105F7000E368A3B9A368834211DA0C480BF03FFB36
:105F8000E368002B09DD45B906490848BDE8F8403B
:105F9000FFF7C4B810605860CFE7A168F5E7F8BD17
:105FA000900102209BFFFF7F300302202403022088
:105FB00090F8253001469B0705D50023C0E9023340
:105FC0000148FFF748B87047900102202DE9F041E1
:105FD0004468064688461746CCB394F8FD309A07C5
:105FE00008D504F1E800FFF791F818B194F8FC30F7
:105FF000BB4229D094F825319B0728D5414604F5AA
:106000008870FFF783F810B394F82431BB421ED197
:1060100001252820D8302044FFF7CAFF282303FB9E
:10602000054595F8FD3042466FF3410385F8FD3094
:1060300021463B463046FFF795FD06483146FFF7BF
:1060400075F80120BDE8F08100252846E2E7002030
:10605000F8E700BF060060F0F8B505460E460023DD
:106060000D4C04F1240794F83820208C02F0010232
:10607000616B13B100231846F8BD002AFBD00A2833
:10608000F9D1A942F7D131463846FFF73FF801234D
:106090000028E8D0004BEEE7440302200B4B30B55C
:1060A00093F838201D8CC2F3400112F001025C6BA2
:1060B00008D039B10A2D05D130B184420CBF184641
:1060C000002030BD0020FCE71846FAE74403022018
:1060D0004FF47A735943FFF721B80000F0B5234C11
:1060E000164694F8383085B0DA0705463CD443F0BC
:1060F000010384F838306F460A233A4623840B465E
:10610000606301F1100EBC46186859680833ACE8AA
:10611000030073456746F6D10FCA154F87E80F0095
:1061200094F83830C6B143F002036FF3820311498B
:10613000A7F1240084F838300BF058FA4FF47A7144
:10614000A7F124007143FEF7E9FF0B482946FEF74B
:10615000EDFF064805B0F0BD66F34103DBB243F046
:10616000040384F83830F0E70020F3E7440302200A
:10617000680302208F500400090060F00C4A10B53B
:1061800092F83830044613F001030FD090420DD13D
:106190000BF035FA94F8383006486FF3000384F8B2
:1061A0003830616BFEF7C2FF012010BD0020FCE714
:1061B000440302200A0060F0436810B56BB393F803
:1061C000472094070FD5481C09D11A880A2A0AD1FA
:1061D00048F2FE029C88181D944204D110BD93F928
:1061E00045208A42F1D093F88F00C0F34000002888
:1061F000F4D04A1C03D093F98D208A420DD1B3F814
:1062000048200A2A09D103F14C00B3F84C2048F287
:10621000FE039A4218BF0020E0E70020DEE70000FE
:1062200048F2FE03F7B500240A880E469A428DF81C
:10623000074030D00B78194DFF2B13D1184E10B3F7
:106240000121FFF7B9FF15E068680DF1070231463B
:10625000FFF714F8002818BF04462035BD42F3D1DB
:10626000B4B912E00E4F0028F8D00DF107024068D3
:10627000FFF704F80446F3E701212846FFF79CFFE7
:10628000044628B92035B542F6D101F003FD044695
:10629000204603B0F0BD014DD0E700BF10E502205D
:1062A00010E5022038B5D0F84841FDF701FE650839
:1062B00004EB4404C5EB5404B0FBF4F303FB1400FB
:1062C000284438BD03685B681B681847F8B5084B5D
:1062D00005461B680E4617464BB11C685B683A467C
:1062E00031462846984714B123462468F6E7F8BD9E
:1062F000140302202DE9F041D1E906780546006833
:106300000C460C300021FEF7C9FEF0B902224FF016
:106310000003284962F30203274A60F3C503521AB7
:10632000D20862F38F1325492A462548FCF7FCFF63
:106330006FF072069FBB636B2BB1324604F13401E0
:106340002846FFF7C3FF02231AE0286801210C301A
:10635000FEF7A4FE40B9E36A33B9236A1B681A69E1
:10636000E2621B7D84F8303094F84430C3F3C303F9
:106370000A2B08D1204603F089FA014620B90123EF
:106380001846BDE8F08121462B6828465B685B68AB
:10639000984703464FB10228F2D16FF00406324607
:1063A00041463846FEF780FEC5E70228E8D16FF087
:1063B0000406C0E7E44E0600344F0600756106008F
:1063C0003A640600012070470120704710B504466A
:1063D000006800210C30FEF761FE58BB23685B6843
:1063E000DB684BBB23681B6983B901214FF00002B6
:1063F00061F3020263F3C5021249134B13485B1A9F
:10640000DB0863F38F121249FCF77AFF23680C3321
:10641000D3E8EF2F42F00102C3E8E12F0029F7D1C2
:106420002046FFF7B9F92046FEF78AFF21460948C2
:10643000FEF77CFE002004E001212046984700285A
:10644000D0DA10BDE44E0600344F0600F9630600B2
:10645000EE610600020001D02DE9F04F464F002505
:10646000BA4687B000F0C2FB444945480BF0BEF87D
:10647000444945480BF0BAF8444C454BE41A454BA7
:10648000C4F3C904DA1B03924FEA521B0493039A24
:10649000EB19954212D1049B534537D101234FF09C
:1064A000000263F302026FF3C5023B493B4864F309
:1064B0008F1207B0BDE8F04FFCF722BF5AF8052055
:1064C000126856680EB132686AB9012262F3020896
:1064D0006FF3C50864F38F1842463149314805937C
:1064E000FCF70EFF059B18463268904773685BB94E
:1064F000012262F3020963F3C50964F38F194A4666
:1065000027492948FCF7FCFE2035C0E7BBF1010F05
:106510001CDD02254FF0000365F302036FF3C50392
:1065200064F38F13ADF8003001221B491F485B460E
:10653000FCF712FF4FF0000265F302026FF3C50291
:1065400064F38F1214491A48FCF7DAFE4023194C01
:1065500084F8543147F230532046C4F84831FFF7ED
:10656000A1FE1549C4F84C0104F5947007B0BDE8CC
:10657000F04F0BF03BB800BF10E50220355104008E
:1065800098010220D55B040024030220344F06004A
:10659000E44E060010E50220F86106004D62060098
:1065A0006A610600046206002C6206007D62060035
:1065B000BE620600B80102206153040070B50025D8
:1065C000064E074CA41B24F01F042034A8192035C4
:1065D000A54200D170BDFFF7F9FEF7E710E50220F4
:1065E00010E5022073B504460D4616460AF07AFE01
:1065F00098B1002201A9204609F0E8FE78B90146C9
:106600004C2201980DF080FA0123019880F8405047
:1066100080F84330046102B070BD3246EAE70020E2
:10662000F9E770B504460D4616460AF05BFE58B110
:1066300000212046FEF776FB044618B129460830B3
:10664000FEF776FB204670BD3146F2E70A4601466A
:106650000148FFF7C7BF00BF54E402200A460146C5
:106660000148FFF7DEBF00BFD0E402200A46014622
:106670000148FFF7D6BF00BFF0E4022003461A69C5
:10668000044B90F840009A4201D1FFF7E7BFFFF7B3
:10669000EDBF00BF38E402200B4601461846FFF765
:1066A000EDBF20B190F84330013380F8433070479C
:1066B00008B1FEF741BB704707B5019080B190F873
:1066C00043306BB1013BDBB280F8433043B94069E2
:1066D00008B1FFF7EDFF019B01A9186909F09EFEC3
:1066E00003B05DF804FB10B50446084661699142A9
:1066F00004D118B9FEF76EFB606110BD1146BDE80C
:106700001040FEF767BB436910B50C460BB94161F9
:1067100010BD1846FEF73EFB2146BDE81040FEF7CF
:106720003EBB38B50546FFF7A9FF044618B1014640
:106730002846FFF7E8FF204638BD38B5044608462E
:106740000D46FEF727FB63690360656138BD0000F5
:106750002DE9F04F87B004930F4604990390164635
:106760004569FFF78BFF044610B300F10808404667
:10677000FEF750FBB0421FD201234FF00005344A10
:1067800063F30205334B6FF3C5059B1ADB084046E4
:1067900063F38F15FEF73EFBADF80050034632461B
:1067A0002D492E48FCF7D8FD2046FFF781FF002435
:1067B000204607B0BDE8F08F31464046FEF716FB95
:1067C000AE89002EF4D0A346D5F80890002FEFD064
:1067D0000BF1080318460593FEF71CFBBE42B246B8
:1067E00028BFBA46AAEB0002002A8046059B1DDBA3
:1067F00001463F1A1846FEF7F9FA42464946FAF7AB
:10680000F9FA059B1846FEF705FB58B9DDE90301C7
:10681000FFF734FF82460028C6D001465846FEF7EF
:10682000C9FAD346A6EB0806C144CFE7514618463D
:10683000FEF7DCFA52464946FAF7DCFA2D68002DDD
:10684000B6D0A7EB0A07AE89D5F80890BEE700BF1F
:10685000E44E0600944F060073640600D8640600F8
:106860002DE9F04107464FF000084469002C35D06F
:10687000236863B304F1080630469D89FEF7CAFA1F
:10688000A84203D23046FEF7C5FA0546A368A089A0
:1068900021682A4618448968FAF7ACFA2946304636
:1068A000FEF7A4FA236898689A894119521B0DF0E3
:1068B000C9F82268304693895D1B9581FEF7AAFAD4
:1068C00078B1226821463846FFF70DFFCEE7A3894D
:1068D0003BB9224641463846FFF705FF0120BDE897
:1068E000F081A0462468C1E72DE9F3410D46174623
:1068F0009846044618B9002002B0BDE8F081002A8D
:10690000F9D00029F7D0436943B94146FFF7B6FEF5
:1069100001460028EFD02046FFF7F5FE22690E4B16
:106920009A4217D0A6691EB1A38F9D4228BF1D466B
:106930006069FEF72FFA094B019400933A464346EB
:106940002946FEF76FFA80B2002ED5D0A38F1B1A0E
:10695000A387D1E70026EBE738E40220996604001C
:10696000F8B51446069D00283AD082898A4207D994
:10697000002296462180591E89B203B120B9F8BD84
:10698000891A89B20068EEE7B4F800C00CF101037F
:106990009BB255B3D54218BF876802F1010618BFF4
:1069A00017F80C70B6B218BFAF54238082899A4290
:1069B00022D832460068A4F800E0F0B9E9B101231A
:1069C0004FF000020E4963F302020E4B60F3C50262
:1069D0005B1ADB0863F38F120B490C48FCF790FC41
:1069E0004FF6FF7300202380C9E7238086899E42EB
:1069F00003D825800068E0E732460B46BBE700BFBE
:106A0000E44E0600944F060080640600BC64060055
:106A10001FB51C4603AB00930223FFF7A1FF9DF8AF
:106A20000C209DF80D3043EA0223238004B010BDF2
:106A30001FB51C4603AB00930423FFF791FF039B94
:106A40001BBA236004B010BD2DE9F84FDDF82C907F
:106A50000C4615469A46BDF828800746002860D1A6
:106A600001234FF00002454963F30202444B60F3F7
:106A7000C5025B1ADB0863F38F1242494248FCF7F8
:106A80003FFC4FF6FF730024AAF8003032E048D2F2
:106A900004F1080B5846ED1AFEF7BCF9ADB286B208
:106AA000B5422AD229465846FEF7A0F9A58904F135
:106AB000080B5846E689FEF7A9F9361A761BB6B2D6
:106AC000464528BF4646A068494628443246FAF75C
:106AD00091F9A1893544691A002902DD5846FEF76B
:106AE00085F9A8EB06081FFA88F8B8F1000F35D130
:106AF000AAF800502046BDE8F88F04D181B258466C
:106B0000FEF774F91FE00CD981B25846FEF76EF912
:106B10002468AD1BADB224B90C993846FFF701FECD
:106B2000044634B90C993846FFF7FBFD04460028AB
:106B3000A7D0A389AB42BAD8A9D104F10800FEF7C7
:106B400069F90028B3D1246834B90C993846FFF7A5
:106B5000E8FD0446002894D00025A8E72468B14445
:106B6000002CF9D10C993846FFF788FD044600281F
:106B700087D001463846FFF7C6FDEDE7E44E060034
:106B8000944F06008E64060000650600002307B5DA
:106B900000934069FFF7E4FE03B05DF804FB07B51E
:106BA000B0F8463090F841100DF10602194489B250
:106BB000FFF7ECFF18B1BDF806308068184403B049
:106BC0005DF804FB07B5B0F8463090F841100DF1C0
:106BD0000602194489B2FFF7D9FF18B1BDF8063093
:106BE0008068184403B05DF804FB7047072310B5B4
:106BF000084C0949C4F8C03020466FF008034FF430
:106C000096620AF0CFFC04F110000449BDE8104080
:106C10000AF080BB44040220009B02202465060089
:106C2000072310B5084C0949C4F8C03020466FF05E
:106C3000080340F2DC520AF0B5FC04F110000449EC
:106C4000BDE810400AF066BB80030220B09F02201E
:106C50001B65060010B5013A0A44914209D307D1D9
:106C60000B781B02184480B2834284BF013080B28B
:106C700010BD0C784B78023103EB04239BB218440F
:106C800080B2834284BF013080B2E6E730B50C09A0
:106C9000ABB1092C86BFA2F10A0564193034431C3C
:106CA000047001F00F01092984BF0A3A89184FF0D6
:106CB000000298BF303119705A70581C30BD002C3A
:106CC000E7D10346EDE72DE9F843164603EBC3028F
:106CD00003EB4203082903EBC3030D46074650FAB2
:106CE00083F480460CBF0D46062530464FF03A0926
:106CF000A0450FD0012318F8011B4122FFF7C6FF62
:106D0000034683F80090A8EB0703DBB29D4200F135
:106D10000100EDD80023B04216BF00F8013C184630
:106D20003046BDE8F883000000232DE9F04F0A2823
:106D300087B082468B469146CDE904333FD103911B
:106D400004A9DCB2002207E00878013201300870A3
:106D5000A018C0B2072804D898183BF810000028E3
:106D6000F2D00133082B01F10101EAD100234FF0E9
:106D7000FF374FF0010804AAD25C424588BF5FB2DA
:106D800003F1010388BF9046082BF4D10293B8F1B8
:106D9000010F4FF03A0308BF4FF0FF370193002275
:106DA0004C461646029B9E421ADB4C4509D00023F6
:106DB000BAF1020F0CBF04F8013C237003E0022873
:106DC00005D04FF00009484607B0BDE8F08F2E23EC
:106DD00004264FF0FF37CDE901364FF00108DEE71A
:106DE000029B042B2DD11BF8061049B930232046F5
:106DF00000F8023B019B63700136F6B20446D1E70E
:106E0000234609204FF0000EDFF8C0C0B1FBFCF5AF
:106E100086450CFB151100DC1DB1864630351D7012
:106E200001330A250138BCFBF5FC451CEED14FF0BF
:106E3000000119701B1BDBB20199E0180130E1540D
:106E4000DAE7B7420ED102B91FB93A23013404F888
:106E5000013C3A23237008F1FF331E44601CF6B254
:106E60000022C9E71AB13A23013404F8013C039B1C
:106E700033F816301D0245EA13252DB2C5F307235A
:106E8000EDB2ABB10F2BD9B20BD900236122204652
:106E9000FFF7FCFE012361222946FFF7F7FE0122DE
:106EA000AAE7092994BF30315731601C2170F1E7FE
:106EB0000F2D03D9612229462046EEE7092D94BF04
:106EC00030355735601C2570E9E700BF00CA9A3B92
:106ED000094B10B41A68094C01321A60032392FB63
:106EE000F3F303EB4303D21A282303FB02425DF8BA
:106EF000044BFFF719BF00BF8005022008050220E0
:106F0000F0B590F8443085B0C3F3C3030A2B0646AE
:106F10005BD14769B0F84650BC682022A3881802AC
:106F200040EA13204B1B184404F1080180B2FFF71C
:106F300091FE96F8411000262944044600963346F7
:106F40000DF10E0289B23846FFF70AFD054610B969
:106F50004FF6FF7037E08289BDF80E309A4210D2AA
:106F600001234FF000021A4963F30202194B66F342
:106F7000C5025B1ADB0863F38F1217491748FCF749
:106F8000BFF9BDF80E30A968AA891944D21A12B205
:106F900096B220463246FFF75DFE2D68044675B175
:106FA000F307A968AA89F2D50B78013A1C44A4B268
:106FB000A34284BF0134A4B212B20131E8E7002831
:106FC000C6D040BA80B205B0F0BD0020FBE700BFDC
:106FD000E44E0600BC4F060034650600446506001A
:106FE00010B559B14469A3688B4207D2A0891144F6
:106FF000184481428CBF0020012010BD0020FCE716
:10700000034B1A6802605A68186002B958607047EA
:1070100084050220002170B5B0F8463086B09A1C75
:1070200090F841300091134404460DF116029BB2D2
:107030004069ADF81210FFF793FCBDF81620054625
:1070400022B118B96FF0150006B070BD4FF47A7315
:10705000029302230DF11206009301960DF116031F
:1070600029462046ADF81420FFF7EEFCBDF8163097
:107070000BB10028E6D03A212046FFF741FF4FF43C
:107080007A73C043CDE901630223ADF81200009387
:10709000BDF8142005AB29462046FFF7D5FCBDF806
:1070A00014301BB10028CDD00020CDE71846CBE727
:1070B0001FB5B0F8463090F8414000911C440DF1E6
:1070C0000E020423A1B24069FFF74AFCBDF80E305E
:1070D000ABB1A0B901234FF000020A4963F30202E9
:1070E000094B60F3C5025B1ADB08084863F38F1293
:1070F0000749FCF705F96FF0150004B010BD00203A
:10710000FBE700BFE44E06002C4F06000D660600AC
:107110007965060010B5B0F8463090F8412086B089
:107120001A444FF47A73CDE901130423009392B209
:107130000DF116034169FFF787FCBDF81630ABB1BE
:10714000A0B901234FF00002094963F30202094B81
:1071500060F3C5025B1ADB08074863F38F12074927
:10716000FCF7CEF86FF0150006B010BD0020FBE76D
:10717000E44E06002C4F06009A6606008C65060059
:107180002DE9F041436996B09B6805469A88130241
:1071900043EA1223B0F84620C2F57F42FC32134482
:1071A0001BB2032B01DC0220A8E0076A4FF47A71BE
:1071B0000020FFF74BFA04460028F4D000216E6946
:1071C000002E40F09E804FF47A7332462846FFF737
:1071D000BFFA8046002800F0DC8001462046FFF719
:1071E00092FA0A2294F84430276262F3C60384F8C4
:1071F00044303B6808F108005B7D84F831303B681F
:107200005B7D84F83930FDF701FE282384F84000C7
:1072100084F84130B5F84630002B76D0A4F84630DB
:1072200063699A6860231370002353709370D3705E
:107230007B680BB193F85431D3716B699E68137EF0
:10724000FF2B06F1080306F1180661D10DF1080EB7
:10725000F446F046186859680833A8E80300B342BA
:10726000C646F6D1183206AE634603CBB342106071
:1072700051609C4602F10802F6D163693846D3F8A2
:1072800008806B69374699681831FEF7C9FF0346D5
:1072900000F1100C3A4618685968083303C2634578
:1072A0001746F7D108F108030AAF324603CABA42BB
:1072B00018605960164603F10803F6D100266B6B7F
:1072C00001A9E36295F83830204684F830306663CF
:1072D000FFF7EEFEB0425CDB812301A9204601935B
:1072E000FFF718FF2046FFF795FE2046FDF71CFE2E
:1072F000B0424EDB2846FFF7DFF9304616B0BDE856
:10730000F081B389366819445AE7A4F8466087E7E4
:107310000AAF3A46BC46186859680833ACE803001F
:10732000B3426746F6D10FCA06AF87E80F000DF1EA
:10733000380EF4466A69636996689B6806F118021C
:107340002836F046106851680832A8E80300B242B7
:10735000C646F6D1083312AE624603CAB24218607E
:107360005960944603F10803F6D16369D3F808C065
:1073700097E80F0016AF86E80F000CF118033246AD
:1073800003CABA4218605960164603F10803F6D1E1
:1073900094E72046FFF790F905E700001FB5B0F825
:1073A00046400DF10E02231D90F8414000911C440F
:1073B000A1B214234069FFF7D3FABDF80E30ABB188
:1073C000A0B901234FF00002094963F30202094BFF
:1073D00060F3C5025B1ADB08074863F38F120749A5
:1073E000FBF78EFF6FF0150004B010BD0020FBE727
:1073F000E44E06002C4F0600526606009F6506000C
:1074000030B50024B0F846200C704C708C70CC70F5
:10741000131D90F8412087B01A444FF47A73CDE9D8
:1074200001131423009392B20DF116034169FFF783
:107430000BFBBDF81630ABB1B0B901234FF0000221
:107440000A4963F302020A4B60F3C5025B1ADB08C8
:10745000084863F38F120849FBF752FF6FF01500DD
:1074600007B030BD1846FBE72046F9E7E44E0600BA
:107470002C4F0600DF660600B56506001FB5B0F8A4
:10748000463090F841400433234490F84A4000913C
:107490001C440DF10E020223A1B24069FFF760FA0D
:1074A000BDF80E3033B1002814BF00206FF0150076
:1074B00004B010BD1846FBE71FB5B0F846400DF10B
:1074C0000E02231D90F8414000911C44A1B21423E8
:1074D0004069FFF745FABDF80E30ABB1A0B9012302
:1074E0004FF00002094963F30202094B60F3C50241
:1074F0005B1ADB08074863F38F120749FBF700FFAD
:107500006FF0150004B010BD0020FBE7E44E06004C
:107510002C4F06002E660600CB65060030B5002411
:10752000A1F80140CC70B0F8462087B0131D90F848
:1075300041201A444FF47A73CDE9011314230093C8
:1075400092B20DF116034169FFF77EFAA0B901234B
:107550004FF00002094963F30202094B60F3C502D0
:107560005B1ADB08074863F38F120749FBF7C8FE75
:107570006FF0150007B030BD2046FBE7E44E060073
:107580002C4F0600BB660600E16506001FB5B0F88B
:1075900046400DF10E02231D90F8414000911C441D
:1075A000A1B20C234069FFF7DBF9BDF80E30ABB197
:1075B000A0B901234FF00002094963F30202094B0D
:1075C00060F3C5025B1ADB08074863F38F120749B3
:1075D000FBF796FE6FF0150004B010BD0020FBE72E
:1075E000E44E06002C4F060076660600F76506009E
:1075F0002DE9F04F984643699BB09B6806469B79FE
:1076000089463A2B9246076A0DD116A9FFF750FD1D
:1076100018B19DF95930002B05DB6FF01505284690
:107620001BB0BDE8F08F4FF47A710020FFF70EF821
:107630000446002800F04481736999688A79112A08
:1076400000F0F280062A00F0F1802C2A40F0DF8062
:1076500000259A891B681544002BFAD14FF47A73E0
:10766000302229463046FFF773F88346002800F0A1
:10767000248101462046FFF746F80A2294F8443058
:10768000276262F3C60384F844303B680BF10800BC
:107690005B7D84F831303B685B7D84F83930FDF7E1
:1076A000B5FB002384F840007868A4F8463008B1A0
:1076B00090F854010022616916928B68ADB25A703D
:1076C0009A70DA703A2208354FF0600C6DBA9D80DE
:1076D0009A714FF47A758DF817A028224FF0010A9D
:1076E000D8718DF8169083F800C00DF1160384F858
:1076F0004120204602950193CDF800A012ABFFF780
:10770000A3F90DF117030146BDF848200295CDE914
:1077100000A3204612ABFFF797F90423029516AD9C
:1077200000930146BDF84820019512AB2046FFF7B3
:107730008BF9B9F1040F0CD12046FFF730FA4FEA6C
:1077400018431A0A4371C8F307230271837180F842
:10775000078073699A68137EFF2B02F1080302F118
:10776000180267D10DF1180EF44661698D68F04674
:10777000186859680833A8E803009342C646F6D152
:1077800005F118030AAD624603CAAA42186059609F
:10779000944603F10803F6D163693846D3F80880AC
:1077A00073692F4699681831FEF73AFD034600F1D8
:1077B000100C3A4618685968083303C263451746E7
:1077C000F7D108F108030EAF2A4603CABA4218607F
:1077D0005960154603F10803F6D1736B2046E36246
:1077E00096F8383084F83030F36A636396F83030B6
:1077F00084F83830FFF70EFC051E04DB2046FDF749
:1078000093FB00285FDA2046FEF756FF07E73B6848
:1078100018315B6838469B689847C0F180002F2874
:1078200006D9A0F1300519E7302517E73C2515E703
:10783000002513E70EAFBC46BE46186859680833EA
:10784000AEE8030093427746F6D19CE80F000AAFFA
:1078500087E80F0063690DF148089A6873699968B1
:1078600001F1180301F1280CC6461868596808335D
:10787000AEE803006345F046F6D112AB08329C46F1
:10788000BCE80300AC4510605160634602F1080299
:10789000F5D16369D3F808C097E80F001AAF85E8FF
:1078A0000F000CF118032A4603CABA421860596047
:1078B000154603F10803F6D18FE76FF00B05A2E739
:1078C0006FF00B05ABE60025A9E6000010B4094BEC
:1078D0001B685BB11C7A8C42FAD15C7A944201D06D
:1078E000002CF5D15B685DF8044B184702205DF869
:1078F000044B7047840502200148FFF781BB00BF9D
:10790000E8D40220072938B504460D4610DD0123CE
:107910004FF000020A4963F302020A4B6FF3C502FB
:107920005B1ADB0863F38F1207490848FBF7E8FC92
:107930006088A3881844143005FB004038BD00BFA0
:10794000E44E06008C4F06000E67060038670600FE
:107950000378013BDBB2037013B9036903B1184725
:10796000704738B5054600242B89A34201DC00206E
:107970000AE021462868FFF7C5FF03782BB900F11C
:107980001403C3600123037038BD0134ECE7000029
:107990002DE9F74F43788146FF2B884692464CD11C
:1079A000DFF8A4B04FF0FF3500245F460BF102036F
:1079B000E60031190BEB0102681C127A17D1002A7C
:1079C00039D019449AF80420DAF8000001930CF039
:1079D0000BF8019B68B926443E44337A0133337275
:1079E00089F80140C9F8088003B0BDE8F08F002A8B
:1079F000E7D10134082CDBD16B1C21D0EE007019CB
:107A00003B181A7A01321A7289F80150DAF800101C
:107A10009AF8042031B1062A04D802305A7038444A
:107A2000F9F7E8F99AF804302E443E4473700020C8
:107A3000C9F80880D8E72546DBE76FF07700D3E781
:107A40006FF00100D0E700BF8C05022038B5437805
:107A50000546FF2B3FD0072B10D901234FF0000222
:107A60001E4963F302021E4B6FF3C5025B1ADB086B
:107A700063F38F121B491C48FBF742FC6B781B4CCD
:107A800003EBC30323441B7A83B901214FF00002A7
:107A900061F3020263F3C5021049114B14485B1AEB
:107AA000DB0863F38F120F49FBF72AFC687800EBC1
:107AB000C00121440B7A013BDBB20B7233B90221C6
:107AC000092212FB0012A118A3508B80FF23002073
:107AD0006B70A86038BD6FF07700FBE7E44E0600DE
:107AE0008C4F060016670600BF6706008C05022053
:107AF000FF670600072813B5044614D901234FF089
:107B000000020C4963F302020B4B6FF3C5025B1AD0
:107B1000DB0863F38F12ADF8002008230246074903
:107B20000748FBF719FC074804EBC404204402B0E3
:107B300010BD00BFE44E06008C4F0600256706000E
:107B4000736706008C05022002684AB943683BB996
:107B500082682AB9C06800F17F4358425841704793
:107B6000002070472DE9FF47934280461D46084696
:107B70000E9F03DD022300203B704CE003AE009615
:107B800001230DF10E02BDF83010FEF7E9FE28B911
:107B90004FF6FF73BDF80E209A42EBD09DF80C30E3
:107BA00053B10DF10D030093BDF80E1001230DF13B
:107BB0000E02FEF7D5FEF8B102244FF6FF790DF163
:107BC0000D0A00B3A5421ED99DF80C3033B3012B2A
:107BD00045D003F0C003802B54D0C02B4BD0402B9A
:107BE000C8D0B8F1000FC5D09DF80D309A1C1444D0
:107BF000A4B2BDF80E203AE04FF6FF73BDF80E2098
:107C00009A42B7D00224A542B4D10D9BBDF80E20F4
:107C10001A8001233B7004B0BDE8F0870134A4B2A0
:107C2000A542F0D9BDF80E10009601230DF10E0209
:107C3000FEF796FE18B9BDF80E304B459AD09DF868
:107C40000C30002BBDD0BDF80E10CDF800A00123E4
:107C50000DF10E02FEF784FE0028B2D18AE79DF8EE
:107C60000D309A1C1444BDF80E20A4B20232134405
:107C7000ADF80E30D4E7D8F814309B681B7EFF2B8C
:107C80003FF478AF2346022204214046FFF7B0FCC0
:107C900070E70000004870475C6806002DE9F0417D
:107CA0000D4688B03221044616469846FEF7E6FC9B
:107CB0000746002864D001462046FEF73EFD6022BC
:107CC00063699B681A7000225A709A719A70DA7010
:107CD00094F84520DA712AB9D8F8041009B191F85E
:107CE0005421DA7132466E46B44602F11008B646A7
:107CF000106851680832AEE8030042457646F6D176
:107D0000183304AA664603CE964218605960B446FA
:107D100003F10803F6D1636994469E682B4605F18A
:107D2000100E654618685968083303C57345AC469C
:107D3000F7D1134606F1080208AE1D4603CDB54241
:107D4000106051602B4602F10802F6D10023A4F81E
:107D5000463063699DF838209B6828219A710A2271
:107D600094F8443084F8411062F3C60384F8443038
:107D700007F10800FDF73AF8204608B0BDE8F081A9
:107D80000446F9E770B505460E46FEF769FD6A69D7
:107D9000002314465CB99268283B5BBA112E93808D
:107DA0000ED1286AFEF70EFB28B9002070BDA1890C
:107DB00024680B44EEE76969284602F0D9FDF4E730
:107DC0003A2EF2D12846FFF725F900EAE070EDE7F8
:107DD0002DE9F04F4669044633460027B56889B05F
:107DE0009A891B681744002BFAD1AA88130243EA28
:107DF00012239BB22833BB423AD151B905F1180086
:107E0000FFF7A2FE002833D105F10800FFF79CFE22
:107E100070BB2B7AFF2B2BD02A7EFF2A01D16B7EE1
:107E200033B3002940F0F080974BB5F81AC058885A
:107E3000844516D1B5F81CC09888844511D1B5F891
:107E40001EC0D88884450CD1D5F81CC0586884451C
:107E500007D1286A844504D1696ADB68CB1A594284
:107E60005941FF2A40F0D0806B7E012B40F0C58045
:107E7000022005E1A36A1E783A2E00F0B580112E8B
:107E800000F0B280062E4FF0000800F0AF8095F8A9
:107E900006A02823564645460DF120096069ADF835
:107EA000188029F80A3D0DF1150B18BB112EA4F806
:107EB000465084F8426000F09B803A2ED8D107A942
:107EC0002046FFF7F5F80028D2DB2046BDF81E500B
:107ED000FFF7A0F807A92046FFF7EAF8BDF81E3023
:107EE000AB42C5D19DF81D209DF81C102046FFF720
:107EF000EDFCC5E03A2ED9D0112ED7D0062ED5D024
:107F0000BDF81610CDF800B001234A46FEF728FD53
:107F10000028ADD000233B2E8DF81C30A8D03C2E7D
:107F200016D0002E57D118F0010F39D001234FF091
:107F30000002564963F30202554B66F3C5025B1A11
:107F4000DB0863F38F1253495348FBF7D9F98FE7E6
:107F500006ABBDF8161000934A460123FEF700FD5C
:107F60000146002884D0BDF8183048F03C080133A1
:107F7000DB009BB21D44ADF81830ADB207AACDE9C5
:107F80000192BDF81620204600923A46FFF7EAFD1E
:107F90009DF81C30022B3FF46BAF9DF8156084E711
:107FA00006ABBDF8161000934A460123FEF7D8FC35
:107FB000014600283FF45CAFBDF818300133DB0008
:107FC0009BB21D44ADF81830ADB2BAF1000F02D12A
:107FD00048F00108D2E7BDF816300122013B042128
:107FE0002046FFF705FB43E700255FE745465DE7D1
:107FF0002146304602F016FC42E029B1052B3FF441
:1080000037AF082B3FF434AFAB1DA3620021282308
:10801000A4F8461084F84130B36805F11808DB79FC
:10802000404684F84530FDF7BBF9014600287FF44F
:1080300021AF4046FDF73CFE00287FF41BAF2B7EAE
:10804000FF2B3FF417AF07AB06AA4146206A02F0A8
:1080500037FB00283FF40CAF069B4BB1DB681A6876
:108060002362527D84F831201B685B7D84F83930AF
:108070000799204602F046FB0028FFF6F9AE0020E3
:1080800009B0BDE8F08F00BF5C680600E44E060052
:108090003C4F0600446806006C68060008B501F015
:1080A00019FEBDE8084002F07BB80346002003B982
:1080B00070479A891B681044F9E7026842B943681F
:1080C00033B9826822B9C068B0FA80F040097047BD
:1080D0000020704703685B689B681847C36893F883
:1080E00030208A4203D0052A18BF83F83010704729
:1080F00070470022002310B50446C0E90A23006837
:1081000018B1FEF7D9FA0023236010BD38B5044634
:10811000C068FFF7EEFF002500210020E368C3E9F7
:1081200006011D622046FFF713FC29462046BDE8E4
:108130003840FFF78BBC08B50C3009F019FB4FF441
:108140007A716422002380FB0101F8F7C9FC08BDA5
:108150000A460146014809F09BBA00BFC87B0220CD
:108160002DE9F34D09F03AFC0026CDE90001224F3C
:10817000DFF888B0F35D13B307EB060ADAF80C807A
:10818000B8F1000F1BD0D8E90A1251EA020316D049
:1081900011F57A7442F10005DDE90023A21A65EBBE
:1081A00003031D46012A75F1000314460EDB5846F1
:1081B000FFF7C1FF18B921465846FFF7C9FF4C36F3
:1081C000B6F5187FD6D102B0BDE8F08D00230024AB
:1081D000D8F80000C8E90A340028F0D0FEF76CFA9D
:1081E000D8F80000FEF768FA0020C8F800005046F2
:1081F000FFF7AEFBE3E700BF0CD502200C06022020
:10820000F8B5054640690E4608302C211746FCF7A4
:10821000EDFD60226B6900249B68311D1A703A22C3
:108220009A71FF22080240EA11215C709C70DC7098
:108230009980DA712846FEF7B2FC07702846FEF7EF
:10824000AEFC4470F8BD10B54369044690F8402078
:1082500098680021801A0BF057FC0023E36284F831
:10826000303010BD08B503681A7D062A14D0082ADC
:1082700014D001214FF00003094861F302030949BA
:108280006FF3C503091AC90861F38F13064807493C
:10829000FBF74AF8002008BD0820FCE71020FAE7A9
:1082A000E44E06004C4F0600B26906000169060064
:1082B00010B540B139B1062A08D842700230F8F73B
:1082C00099FD002010BD6FF01500FBE76FF07900FD
:1082D000F8E700002DE9F8430F4E074688460024D2
:1082E000B146A35D3BB94C34B4F5187FF9D10025F4
:1082F0002846BDE8F8831FB133199B689F42F2D12D
:1083000009EB0405E8681022414604300BF06CFBD1
:108310000028E8D1ECE700BF0CD502202DE9F84F8A
:108320000646006AFFF7D6FE96F84030834218D022
:108330000025A9462C46AB46D6F8148086F84000A6
:10834000B8F80C707561C4B932213046FEF796F961
:10835000054648B93046FEF7AFF94046FEF7A8F9A2
:108360002E463046BDE8F88F01463046FEF7CBF981
:1083700005F10800FCF74EFD84B2BC4205F108008F
:1083800019D33946FCF732FDD8F808103A4649446B
:10839000F8F730FDD8F800A04046C8F800B0FEF766
:1083A00087F9BAF1000FDCD0E41BA4B2BAF80C7064
:1083B0004FF000090FE02146FCF718FDD8F808102F
:1083C000224649443F1BA144F8F714FDC24600244D
:1083D000BFB21FFA89F9D046B5E770B50C4606461C
:1083E00015460B70D3084B7002790168A01CF8F792
:1083F00001FD307900212A1A02302044023ABDE8FA
:1084000070400BF081BB00007FB501A9FFF754F865
:10841000002814DA01234FF000020B4963F3020233
:108420000A4B6FF3C5025B1ADB08094863F38F122E
:108430000849FAF765FF002007B05DF804FB9DF8D6
:108440000400C0F38010F7E7E44E06004C4F06002E
:10845000C76B06009C6806007FB501A9FFF72CF8E2
:10846000002814DA01234FF000020B4963F30202E3
:108470000A4B6FF3C5025B1ADB08094863F38F12DE
:108480000849FAF73DFF002007B05DF804FB9DF8AE
:108490000400C0F34010F7E7E44E06004C4F06001E
:1084A000C76B0600BB6806007FB501A9FFF704F89B
:1084B000002814DA01234FF000020B4963F3020293
:1084C0000A4B6FF3C5025B1ADB08094863F38F128E
:1084D0000849FAF715FF002007B05DF804FB9DF886
:1084E0000400C009F8E700BFE44E06004C4F060048
:1084F000C76B0600AD68060048F2FE030A8810B597
:108500009A424FF0010411D14FF0000209490A4B81
:1085100064F302025B1ADB086FF3C502074863F3DA
:108520008F120749FAF7ECFE002010BDFDF7DCFAC8
:108530002046FAE7E44E06004C4F06008E6906001E
:10854000DC6806002DE9FF4106461C480C469046B3
:10855000FFF707FA054660B3FF23437023466C46D6
:1085600027468660C66803F1100C224618685968D1
:10857000083303C263451446F7D1331D04AA3C46B1
:1085800003CC944218605960274603F10803F6D1E2
:1085900041462846FFF7A2FD0122EB68002000219A
:1085A00083F835200022C3E90A01C3E906011A60F5
:1085B0001A62284604B0BDE8F08100BF00D5022051
:1085C000704700007FB518234178064A0230FEF755
:1085D0007AFB054A034618216846FAF7B5FB07B04F
:1085E0005DF804FBD4050220F772060070B505465D
:1085F0000E46FFF76FFE044668B13146284601F08B
:10860000C1FF2046FFF782FD002303481A46294692
:1086100001F05AFE012070BD100060F0FFF75ABE55
:108620002DE9F0470F4692B0114615461E4680468A
:10863000FFF750FD6421FEF709F8044638B16421C4
:10864000FEF71CF8814628B92046FEF735F86FF092
:108650000B058FE001462046FEF755F80A22D8F8B0
:108660000030C4F820805B7D204684F83130D8F893
:1086700000305B7D84F8393094F8443062F3C603EF
:1086800084F84430282384F84130FFF7DCFD40466D
:10869000FFF7E8FD002300F1140AA4F84630882211
:1086A0005FFA8AF180462046FFF7AAFD09F108002B
:1086B0005146FCF79BFB63699A683B4601AFBC4699
:1086C00003F11009BE46186859680833AEE8030084
:1086D0004B457746F6D1083205AB674603CF9F423C
:1086E00010605160BC4602F10802F6D162699C46F6
:1086F00097682A4605F1100E6546106851680832E1
:1087000003C57245AC46F7D107F1180509AA1F4603
:1087100003CF9742286069603B4605F10805F6D112
:108720003346164603F11007354618685968083372
:1087300003C5BB422E46F7D10FCA12AD05E90F00A3
:10874000236A20461D68FEF72AFA103500F1180149
:10875000022328464246FFF740FE9DF8683012A9E2
:1087600001F8143D2046FEF7D9FE051E06DA204624
:10877000FDF7A2FF284612B0BDE8F087636908F153
:108780004008A3F80C802046FEF744FC051E204656
:10879000EEDBFCF7C9FB002805DA2046FDF78CFF6D
:1087A0006FF01505E6E70025E4E70000436870B5C3
:1087B0000D4613B1D3F84C418CB901234FF00002A0
:1087C000104963F30202104B6FF3C5025B1ADB081A
:1087D00063F38F120D490E48FAF792FD0024EE68FC
:1087E00009F0FCF8EB68C6E906011C620948FFF7CE
:1087F000A2FC28B92146BDE870400648FFF7A8BC96
:1088000070BD00BFE44E06004C4F060038690600FC
:108810006A6B0600EC0502202DE9F04104468CB09D
:108820004069FFF742FC07A985B22046FEF744FEE7
:10883000002811DA01234FF00002B64963F3020267
:10884000B54B6FF3C5025B1ADB08B449B44863F358
:108850008F12FAF755FD07E0412D07D805A92046EC
:10886000FEF726FC002834DA0220C7E063699B6823
:10887000DB79FF2BF2D19DF82030FF2BEED0204684
:10888000FFF7C2FD20B163699B681B7EFF2BE5D01B
:108890001423606984F84A30FFF707FC02A9A0F1AD
:1088A0002C052046FEF7EAFD002618B994F84A2068
:1088B000954213D808A9206AFCF7C8FD002839D0D2
:1088C00090F94530002BCFD108A9206AFFF714FE9C
:1088D000CAE79DF81530002BDAD0C5E79DF80930BE
:1088E000002BE7D09DF80810022907D1B4F84660A4
:1088F000B11D94F841600E441644B6B202EBC303B6
:10890000DBB2934284F84A300FD801234FF00002C3
:10891000804963F30202804B6FF3C5025B1ADB08E8
:1089200063F38F127D497F4893E702A92046FEF743
:10893000A5FDBAE7CDE9030008A9206AFFF7CAFC44
:108940000546002890D0002E5BD16B78FF2B6FD0AE
:108950006878FFF7CFF80746002885D0002E7ED034
:108960004278811C0DF10E000BF03EF810F100086A
:1089700018BF4FF00108EB6893F83030002B75D129
:10898000002E3FF471AFB8F1000F08D03846FFF762
:1089900019FE7A780DF10E013846FFF789FC204662
:1089A000FFF732FD00285CD001212846FFF796FB37
:1089B000002200200021EB6883F83420C3E906017F
:1089C0001A622946206AFFF7F1FE2046EE68FFF79B
:1089D0006BFDEB6886F835001E685EB13046FCF72B
:1089E000A3FA002880F29280E868FFF782FB304605
:1089F000FDF762FE2046FDF75FFE00200CB0BDE8EB
:108A0000F081236A0DF10E021B6831461B7D6069FF
:108A100000920DF10A028DF80D30FDF7A1FF00283C
:108A200093D14FF6FF73BDF80A209A428DD11BE710
:108A3000002E3FF419AF9DF80D300CAA8DF81830B8
:108A40000DF10E0342F81C3D216A2846FEF7A0FFF7
:108A500000283FF47DAF2846FFF758FB04E7B046F7
:108A600089E702212846FFF739FBAEE72046FFF7EA
:108A7000F3FC68B9B8F1000F0AD0EB6893F8303016
:108A8000012B7FF4F1AE02212846FFF727FBEBE62E
:108A90002046FFF7E1FC20BB2046FFF7DDFCB0B924
:108AA000AEB1B8F1000F12D12046FFF7ADFC28B3EC
:108AB00001212846FFF712FB002000210022EB686D
:108AC000C3E906011A622946206AFFF76FFEEB68C8
:108AD00093F83530002B3FF478AF2046FFF7E4FCE5
:108AE00073E7B8F1000FDFD03846FFF76BFD7A78F7
:108AF0000DF10E013846FFF7DBFBD5E7B8F1000FAB
:108B0000E5D002212846FFF7E9FAE0E70022EB680A
:108B10001A606CE7E44E06004C4F060059690600E7
:108B2000EA690600086A06002DE9F04F1E469DB06E
:108B30009DF89C3088463146154601938146DDF804
:108B400098A0FFF7C7FA6421FDF780FD044638B10D
:108B50006421FDF793FD074628B92046FDF7ACFDDB
:108B60006FF00B0B6AE001462046FDF7CCFD0A22B0
:108B7000D9F80030C4F820905B7D204684F831306D
:108B8000D9F8003008375B7D84F8393094F84430E8
:108B900062F3C60384F84430282384F8413000236C
:108BA000A4F84630FFF74FFB206AFFF75BFB00F1AC
:108BB00014018722C9B281462046FFF721FB142108
:108BC0003846FCF713F963699B68002E3AD140F2EE
:108BD000FF229A611E775E779E77DE7783F82060AA
:108BE00083F821604FF480725A84FF2283F8242096
:108BF0009AF80D2083F82520BAF80E20DA8407AA07
:108C000013460AF1100C1646DAF80000DAF80410E0
:108C10000AF1080A03C6E2453246F4D10FCB18AE7A
:108C200086E80F000DF15C0A51462046FEF7E8FB8E
:108C3000B0F1000B20DA2046FDF73EFD58461DB08E
:108C4000BDE8F08F0DF10C0C06F1100E6246306895
:108C50007168083603C276459446F7D103AE1833DF
:108C60000DF11C0C324603CA624518605960164665
:108C700003F10803F6D1C2E76369D3F808B0019B9A
:108C8000002B64D0BBF80470FFF704F80DF12C0C36
:108C90000246654600F1100AE6461068516808323F
:108CA000AEE803005245F446F6D10BF108030DF18E
:108CB0003C0C2A4603CA624518605960154603F108
:108CC0000803F6D163699A683B0243EA17239BB213
:108CD000A3EB090999FA99F9A2F804902046FEF746
:108CE00099F9B0F1000BA6DB3146206AFFF7F2FAE2
:108CF000054638B902463146206AFFF723FC05468F
:108D0000002847D0B8F1000F15D0EE683368002B6B
:108D100043D14046FDF7C5FC3060EE6808F05EFECA
:108D2000C6E90A013C48FFF706FA20B94FF47A7108
:108D30003948FFF70DFA2046FCF7F6F8002867DA05
:108D4000B8F1000F2CD0E868FFF7D3F928E06DB335
:108D50000DF13C0C624605F1100AE6462868696888
:108D60000835AEE803005545F446F6D115460BF13B
:108D700008030DF14C0C2A4603CA6245186059607D
:108D8000154603F10803F6D1636998680830FFF7C8
:108D900094F958B3B8F1000F02D04046FDF78CFCAF
:108DA0002046FDF789FC6FF0150B47E70BF1180122
:108DB000206AFDF735FA0DF14C0C0246654600F1CC
:108DC0001003E646106851680832AEE803009A4284
:108DD000F446F6D10BF108032A4603CA524518603F
:108DE0005960154603F10803F6D1CDE749463846E8
:108DF000FBF7FCFF236A20461D68FDF7D0FE103507
:108E000000F1180101234A462846FFF7E6FA65E714
:108E10004FF0000B12E700BF0C0602202DE9F341D2
:108E200006460F461546FFF755FA044678BB9DF8EF
:108E3000202039463046FFF785FB044638BB012326
:108E40004FF000062F4A63F302062F4B39469B1A58
:108E5000DB0860F3C5060A2063F38F16FEF738F8C7
:108E6000FAF7ECFA1823294A297907462868FDF70A
:108E70002AFFFAF7E3FAADF8006003463A462449C0
:108E80002448FAF769FA204602B0BDE8F0812A4684
:108E900031462046FEF77CFD78301AD1E36893F81E
:108EA0003030052B26D06078FEF724FE2A798046E4
:108EB000296802300AF098FDB8B14046FFF782FBFE
:108EC0002A7929684046FFF7F3F902212046FFF787
:108ED00005F9E36893F8303063B9CDE900731A46B9
:108EE00019463046FFF720FE04E0E36893F830307F
:108EF000002BEAD0002331461A46074801F0E4F976
:108F0000C1E700BFE44E06004C4F0600D405022026
:108F1000CB680600406B06000F0060F02DE9F04FB3
:108F200041699BB004460846FFF7BFF880B2392874
:108F300008D98B68DA79FF2A04D11A8948F2FE032E
:108F40009A420CD012A92046FEF7B2F8002802DBA4
:108F50009DF849301BB102201BB0BDE8F08FB4F87A
:108F600046101AAD2C3189B225F84A1D0DF11903AE
:108F700000932A4601236069FDF7F2FC0023BDF847
:108F80001E1000932A460123FDF7EAFC0028E2D0D8
:108F90009DF8192022B1236A5B680BB183F8542134
:108FA00007AB2A46BDF81E10FDF732FD08AB2A4676
:108FB000BDF81E10FDF73CFD09AB2A46BDF81E109A
:108FC000FDF736FD06460028C5D00BA92046FEF762
:108FD000DDFA834B834A0028A3EB0203C3F3C903E2
:108FE00003930EDA01234FF0000263F30202039BA6
:108FF0006FF3C50263F38F127B497C48FAF780F95F
:10900000A9E7089B7A4A591E914210D8226A5768EC
:10901000002F7AD0D7F84C210C99914207D00FB18C
:10902000C7F848313846FDF73DF9C7F84C01099AB1
:1090300022B1236A5B680BB1C3F850214FF0000ADC
:109040000DF11B03BDF81E1000932A460123304684
:10905000FDF786FC0DF11A030093BDF81E100123E5
:109060002A46FDF77DFC00283FF475AF9DF81B20D4
:10907000BDF81E80032A00F0BF80052A47D0012AD0
:109080009DF81A7040F0068206238DF83C308DF86A
:10909000493094F830300DF14A02052B98BF8DF815
:1090A0003C300E9200929DF83C302A464146FDF736
:1090B00057FC064610B9B8F1000F21D19DF83C309D
:1090C000C3EBC703023B13F0FF030CD00022304672
:1090D0000092BDF81E102A46FDF742FC064610B964
:1090E000BDF81E3063B963690EAA9968022308317E
:1090F0000093206A0123FFF791FE8246002E9FD144
:10910000BDF81E30002B3BD025E73A4684E700230C
:109110002A46009341460223FDF722FC0AAB2A4669
:10912000BDF81E10FDF784FC064620B9BDF81E30C0
:10913000002B7FF410AF0A9AA2F5A063B3F57B4F22
:1091400018D301214FF0000361F3020303996FF379
:10915000C50361F38F1324492648CDE912124FF459
:10916000A0614FF6FF72CDE91412042212A9FAF79A
:109170000EF9F0E6236A1B681A83002E7FF460AFB5
:109180006369206A99680831FCF766FFBDF81C2006
:109190000346002800F09681002A40F08681FCF703
:1091A000EDFFBAF1000F10D0DAF80C30186860B19A
:1091B000FBF7BAFE002804DADAF80C301868FDF77D
:1091C0007BFADAF80C00FEF794FF236A586800F582
:1091D000947008F014FA2046FDF76EFA0020BBE602
:1091E0004C4F0600E44E06007E6906008C6A0600BD
:1091F0007FEE3600A56A06009DF81A308DF84820EB
:10920000DB00023B8DF849300DF14A0300932A46FA
:1092100001234146FDF7A4FB0DF14B03BDF81E10E1
:1092200000932A460123FDF79BFB13AB2A46BDF8AA
:109230001E10FDF7FDFB14AB2A46BDF81E10FDF70E
:10924000F7FB0023BDF81E1000932A46042316AF37
:10925000FDF786FBBDF81E10009710232A46FDF788
:109260007FFB064620B9BDF81E30002B7FF448AFC7
:10927000DDE913239A42FFF441AF48F2FE03BDF843
:1092800058209A423FF43AAF9DF94B30002B38DA20
:109290009DF84A203946206AFCF7E2FD002840F09C
:1092A0008380139B6BB39DF84A203946206AFCF7F4
:1092B00053FD002878D10123BDF80820394663F317
:1092C000020293B260F3C503ADF80830BDF8082080
:1092D000039B0A2063F38F127E4BADF808200E9398
:1092E000FDF7F6FDFAF7AAF89DF84A300F901093B3
:1092F000236A042211930EA9BDF808307648FAF7C4
:1093000046F89DF84B305B067FF5F8AE139B002BBB
:109310003FF4F4AE9DF84A30402B7FF4EFAE0E22BE
:1093200000210DF13A000AF0EFFB236A1A6848F2B7
:10933000FE03ADF8383000230F93117D06294DD080
:10934000082969D0022912D1517D01290FD110932A
:10935000FF218DF84310FE218DF8453013698DF8FB
:1093600044101A788DF846205B788DF847300DF15F
:10937000380897E8030088E8030000214046FCF71E
:109380000FF8DDF84C900746002878D090F844306C
:10939000012B74D1B9F1FF3F44D190F8473043F02D
:1093A000010387F84730A9E6139951B14A1C90F898
:1093B00025300ED06FF3000380F82530FCF7AEFDAA
:1093C0009FE790F8242000F11001206AFCF7FEFDD1
:1093D00097E743F0010380F8253092E71369997805
:1093E00018888DF84210FF218DF84310FE21ADF84A
:1093F00040008DF8441033F8031FADF845109B78FA
:109400008DF84730537D032BB1D19DF8403083F068
:1094100002038DF84030AAE7126910AB106851685A
:1094200003C3F2E7B9F5E15F08D913993846FCF7B1
:1094300035F897F847306FF30003B2E7C069C8B159
:10944000264A3B6AC117C2FB0301CDE9040108F0BB
:10945000B9FABB69C01A09F05DFFDDE904BCBBEBDA
:10946000000B6CF1000C4FF47A72002358466146F1
:10947000F7F736FB4845D8D34FF4E151D6E7B9F1B9
:10948000FF3F206A0CBF00234B4601224146FCF7F8
:1094900053F833E60022FB00023B00929BB22A46BF
:1094A0004146FDF75DFA064628E6BAF1000F04D002
:1094B0000120DAF80C1081F8350011461846FCF747
:1094C00007FE6EE66369206A99680831FCF706FEBC
:1094D00067E600BF69690600D26A06009BFFFF7F4E
:1094E0002DE9F04F04469DB04069FEF7DEFD0DF119
:1094F0005C0985B249462046FDF750FF002811DA85
:1095000001234FF00002BF4963F30202BE4B6FF329
:10951000C5025B1ADB08BD49BD4863F38F12F9F73A
:10952000EFFE13E03F2D04D963699B68DB79FF2BC5
:1095300010D09DF86030FF2B0CD113A92046FDF709
:10954000B7FD002802DB9DF84D301BB102201DB095
:10955000BDE8F08F1423606984F84A30FEF7A5FD5A
:1095600002A9A0F12C082046FDF788FF01460DF165
:109570003E0619B994F84AA0C2452ED318AE31461A
:10958000206AFBF763FF82460028DFD0636900F1A1
:1095900004089D6805F108073846FEF78EFD014670
:1095A000002800F0DC8040F2FF23AA699A42CDD166
:1095B000EB69002BCAD12A6AB2F1807FC6D16A6AF0
:1095C000D2B2FF2AC2D19AF945200226002A77D1C9
:1095D0004146206AFEF790FFB8E79DF80950002D3C
:1095E000CCD09DF808B0BBF1010F48D16769B868CD
:1095F0000830FEF762FD0028A8D1022D0ED94FF0E9
:1096000000026BF3020261F3C5027F4B7D49814882
:109610005B1ADB0863F38F127C4980E7B4F84610CD
:1096200000968B1D94F841100BAA1944EB0051448D
:10963000023BDBB289B238468DF83D30FDF790F938
:1096400030B94FF6FF73BDF82C209A423FF47EAF3D
:109650009DF83D2094F830308DF850209A4288BF14
:109660008DF85030636913AA99680023083100937C
:10967000206A1396FFF7D2FB00283FF467AF94F8F7
:109680004A209DF8093002EBC303DBB29A4284F80A
:109690004A300FD301234FF000025A4963F302020C
:1096A000594B6FF3C5025B1ADB0863F38F125749FE
:1096B000594834E702A92046FDF7E0FE014658E785
:1096C0004FF0FF326E762A76AB76EB762B776B77A0
:1096D000AB77EB7785F8203085F8213085F822309C
:1096E00085F8233085F8243085F8253085F8263034
:1096F000012385F827306369206A9D6805F1180108
:10970000FCF78EFD03AA0346164600F1100E9446A0
:10971000186859680833ACE8030073456246F6D10F
:1097200005F1080307AD324603CAAA421860596022
:10973000164603F10803F6D1202362693946926880
:10974000206A009318324346FEF76AFF0546002858
:109750007FF4FCAE2046FCF7AFFF2846F7E638461C
:10976000FBF71EFE00287FF4F1AE40F2FF22636992
:109770009B68996903F1180E914209D1DA693AB9E7
:109780001A6AB2F1807F03D15A6AD2B2FF2A45D059
:109790007146206AFBF75AFE804600283FF4D6AE99
:1097A0000FAD2F4663699A6802F108031832AC4680
:1097B000186859680833ACE8030093426546F6D14F
:1097C00013AD3A4603CAAA4218605960174603F11E
:1097D0000803F6D163699F6896E80F0085E80F00DB
:1097E00007F108032A4603CA4A451860596015461E
:1097F00003F10803F6D1636908F104089F6808378C
:1098000034E000BFE44E06004C4F06000E6906002F
:10981000216A06003F6A0600736A060007AA94469A
:109820000833154618685968083303C573452A4636
:10983000F7D10BAD624603CAAA421860596094463C
:1098400003F10803F6D16369D3F808C096E80F0066
:109850000FAE85E80F000CF108032A4603CAB24296
:1098600018605960154603F10803F6D1602364E7D8
:10987000012307B501930023043100911A461946CC
:10988000FFF752F903B05DF804FB00000023F0B5C8
:1098900085B00393044608B1436983B901234FF0AF
:1098A0000002544963F30202534B6FF3C5025B1A83
:1098B000DB0863F38F1251495148F9F721FD236A00
:1098C0001B680C33D3E8AF3F990777D46369626BA9
:1098D0009B6803F1180112B91B7EFF2B08D194F885
:1098E00044305A076AD42046FEF718FD044665E066
:1098F00003A8FCF7DBFA63699D68183500284CD093
:10990000039B1A682362527D84F831201B685B7DBB
:1099100084F83930039B7BB9294603A8FCF7C6FAC3
:10992000002855D0039B1A682362527D84F83120A9
:109930001B685B7D84F8393029460398FEF7CAFC22
:109940000646002847D04078FF2844D0FEF7D2F8DA
:10995000831C6363437884F83830F36893F83030BD
:10996000022B14D130460321FEF7B8FBF76808F04C
:1099700035F8F36841F28836C7E906011E622148CE
:10998000FEF7D9FB18B931461E48FEF7E1FB94F803
:1099900044305B0712D42946A5E7294600F072FD42
:1099A000064670B100F048FE05460028B2D13046A8
:1099B00000F0C2FD2046FCF77FFE0024204605B0E3
:1099C000F0BD2946FCF76AFB88B100F12405A1E748
:1099D000236A0393B0E70026636921469A68CDE9BC
:1099E000005633460832206AFFF79EF8E5E7002D5F
:1099F000A2D1DFE7E44E06004C4F0600E768060000
:109A00009E6B0600EC0502202DE9F04F85B007F0B3
:109A1000E5FF0025804689464E4E4F4BDFF848B1A2
:109A2000F61A4E4FC6F3C90615F80B30002B3CD082
:109A30000BEB0504E168002937D0D1E90623CDE915
:109A40000223134331D0DDE90223086A121843EBE5
:109A5000E073B2EB080263EB0903012ACDE90223AC
:109A600073F1000308DB3846FEF765FBE8B902999D
:109A70003846FEF76DFB18E000230022C1E90623FB
:109A800091F83030052B10D8DFE803F0162B1A2F91
:109A90003503012363F3020A6FF3C50A66F38F1AD5
:109AA00052462F492F48F9F72BFC4C35B5F5187F56
:109AB000BAD105B0BDE8F08F91F83430022B03D94C
:109AC0002046FEF723FBF0E7013381F83430002312
:109AD0000431009101931A461946A068FFF724F853
:109AE000E3E7022381F83030DFE7042381F83030E8
:109AF000002381F8343091F83430A068022B01F152
:109B000004020BD91146FCF7A7FA0028CDD090F833
:109B100038305B07C9D4FCF731FBD1E7013381F85A
:109B200034300023CDE9002319461A46FEF7FCFF26
:109B3000E368029307F052FF029BC3E90601E36862
:109B40004FF47A7438461C62FEF7F5FA0028ACD15F
:109B500021468DE74C4F0600E44E0600EC0502203E
:109B60001E690600026B06000CD50220F0B500212C
:109B700085B00746FEF7AEFA6421FCF767FD0446A0
:109B800038B16421FCF77AFD064628B92046FCF777
:109B900093FD6FF00B0589E001462046FCF7B3FD0D
:109BA0000A223B6827625B7D204684F831303B689F
:109BB0005B7D84F8393094F8443062F3C60384F84E
:109BC0004430282384F84130FEF73DFB4FF0FF324C
:109BD000022163699B681A76597600229A76DA76B2
:109BE0001A775A779A77DA7783F8202083F821203A
:109BF00083F8222083F8232083F8242083F825206B
:109C000083F82620012283F82720636938469D685F
:109C100005F11801FCF704FB6A460346174600F1FC
:109C2000100E9446186859680833ACE80300734571
:109C30006246F6D105F1080304AD3A4603CAAA42CA
:109C400018605960174603F10803F6D163699868F4
:109C50000830FEF732FA074658BB206AFEF702FBCF
:109C60000546291DC9B2204685220836FEF7C8FAE6
:109C700004213046FBF7BAF887B929463046FBF78E
:109C8000B5F8236A20461E68FCF789FF103600F1FC
:109C9000080101232A463046FEF79FFB2046FDF7C8
:109CA000B9F9051E204606DAFCF706FD284605B080
:109CB000F0BD0025D5E7FBF737F9002805DA204687
:109CC000FCF7FAFC6FF01505F0E70025EEE7FFF76B
:109CD0004DBF000008B50948FDF792F90848FDF7A7
:109CE0008FF90849084807F081FC0848FDF788F912
:109CF000BDE808400649074807F078BC6CD7022049
:109D0000F4D40220618104000C06022078D70220DE
:109D1000099A0400EC05022003685B689B681847F9
:109D200007B502AA02F8011D32230121FCF7DCFD70
:109D3000431E5842584103B05DF804FB07B549BAC9
:109D400002AA22F8021D32230221FCF7CDFD831E58
:109D50005842584103B05DF804FB70B50D46D1B2CE
:109D600004461E46FFF7DCFF10B90024204670BDF4
:109D700000212046FFF7D4FF0028F6D031462046C8
:109D8000FFF7DCFF0028F0D02A46322310212046BE
:109D9000FCF7AAFD10280546E7D1002EE6D0FDF716
:109DA00079FF3223024629462046FCF79DFD102804
:109DB000DCD0DAE740F2FF23F0B58BB006460F4661
:109DC000ADF818300025ADF81A50ADF81C50ADF8BC
:109DD0001E50ADF82050ADF82250ADF824504FF48D
:109DE000B053ADF8263006A9FFF796FF3221FCF7F5
:109DF0002DFC0446002800F09B8006A93046FCF7A5
:109E00000FFA00950146334606AA2046FDF746FFA5
:109E100038B96FF00B052046FCF74EFC28460BB016
:109E2000F0BD0121636920469A68D1719B893A216E
:109E3000A4F84830FFF774FF0028EAD029462046EE
:109E4000FFF76EFF0028E4D040F202512046FFF7F2
:109E500075FF0028DDD029462046FFF76FFF002858
:109E6000D7D029462046FFF75BFF0028D1D02946EE
:109E70002046FFF755FF0028CBD08F212046FFF763
:109E80004FFF0028C5D029462046FFF749FF00288C
:109E9000BFD000212046FFF751FF0028B9D0002194
:109EA0002046FFF74BFF0028B3D0336826625B7D66
:109EB000394684F83130336820465B7D84F8393088
:109EC000FCF721FC00212046FDF75CFF051EA2DB0C
:109ED00008233A21A4F8463020466669FDF710F8B9
:109EE0003A2105462046FDF70BF86FEA2525C043C9
:109EF000EDB245EA002080B2030243EA10200DF1E2
:109F00001603322201930223ADF816000093029249
:109F100005AB31462046FCF797FD00283FF479AFAA
:109F20002046FBF701F8051EFFF675AF002575E723
:109F30006FF00B0572E7F8B50E460021174605468F
:109F4000FFF7EAFE3221FCF781FB0446D0B1012184
:109F5000FFF7F4FE30B96FF00B052046FCF7ACFBC1
:109F60002846F8BD01233A4631462046FFF7F5FE64
:109F70000028F0D028466169FFF71CFF0023054642
:109F80006361EAE76FF00B05EAE700002DE9F047AF
:109F90000446002547698CB0002F40F0BE80B4F81D
:109FA000461006AA0B1D94F841102046194489B2A8
:109FB000FCF7ECFD05AB0DF11A02BDF81810FCF72B
:109FC00027FD08AEBDF81A1002230DF11A02009702
:109FD000FCF7C6FCBDF81A1010230DF11A0200960A
:109FE000FCF7BEFCBDF81A1002230DF11A0200970F
:109FF000FCF7B6FC0DF116030DF11A02BDF81A10AC
:10A000006069ADB2FCF704FD28B94FF6FF73BDF8E7
:10A010001A209A427DD0BDF81630B4F846201B01B4
:10A02000443313449BB2AB4207D8B3F5A06F04D8B6
:10A0300063699B68DB79012B09D007A92046FDF7EE
:10A0400037F8002865DB9DF81D30002B61D1FDF746
:10A0500021FE10220146304609F0C6FC05460028C4
:10A0600057D1D4F82080D8F8047087B901234FF075
:10A0700000022C4963F302022B4B67F3C5025B1A03
:10A08000DB0863F38F1229492948F9F739F90021D0
:10A090004046FFF741FE3221FCF7D8FA044600287B
:10A0A00037D00021FFF73CFE80B300264FF018099F
:10A0B00007F1940A09FB06F17B1893F8A430DA073C
:10A0C00009D59B0707D50023022251442046FFF7FC
:10A0D00044FED8B101350136032EEBD1002D15DD3C
:10A0E0003223616902930DF11303019301230022CE
:10A0F0000093204607AB8DF81350FCF7A5FC28B160
:10A1000061694046FFF756FE002363612046FCF775
:10A11000D3FA02200CB0BDE8F087BB893F681D442C
:10A120003AE700BFE44E0600444F06001B6C0600F1
:10A130002B6C060073B50D4602AB43F8040D1946AF
:10A140002846FBF7B5FD0446F0B1037D9B0718D404
:10A15000022229460198FFF7EEFE061E0EDB237D44
:10A16000012243F00203237529460198FBF7DCFD29
:10A17000002301991A46094800F0A6F8304602B0BB
:10A1800070BD6FF07706F9E729460198FBF7B8FB39
:10A1900004460028DCD16FF00B06EFE7070060F003
:10A1A0000148FCF72DBF00BF84D702202DE9F84FEE
:10A1B0003F4F4FF0FF313F4807F016F84FF0FF31A7
:10A1C0003D4807F011F83D4BB3F90050002D21DB5D
:10A1D00057F83520F2B13A496A1CB1F9000012B2C1
:10A1E000A8421A8012D14FF6FF720A801A80354EAB
:10A1F0003468CCB9002347F8353007EBC5056B60F0
:10A200002D4806F0C9FF06F0B5FED2E7022AEED1CE
:10A210000022EBE74FF0FF320021264806F08EFFC8
:10A22000254806F0B9FFC4E74FF00008C346D4F84C
:10A23000009007EBC50A57F83510A06881EA0003C3
:10A2400013F0405F21D1C3F30A43F3B98BB21BB1C2
:10A2500082B20AB1184218D000016368DAF804200B
:10A2600022D5986908B182420FD1A1609A61226813
:10A27000B8F1000F10D1716832608C4200D1726069
:10A28000C4F800B0184606F087FFB9F1000FB1D04E
:10A290004C46D9F80090CEE7C8F800207268944286
:10A2A00008BFC6F80480EBE720469847A046ECE7D5
:10A2B00034060220A4E402208CE40220F8060220E6
:10A2C000480602202C060220224B70B51B6804466B
:10A2D0006FEA137202F0030212EA10720D4637D1D0
:10A2E0006FEA1342C2F30A0212EA104230D1DB4392
:10A2F0009BB203422CD14FF0FF31174806F074FF98
:10A300001649174E0B88174801331BB2022B08BFA2
:10A31000002306EBC3025560B0F9002046F8334035
:10A32000934211D15A1C92B2022A08BF002256F859
:10A33000324004B1028008480B8006F02DFFBDE8D2
:10A340007040094806F028BF002AB8BF0380F2E732
:10A3500070BD00BF440602208CE4022048060220A3
:10A3600034060220F8060220A4E4022030B50024BE
:10A37000134B144AC3E90044134B87B01C604FF6DB
:10A38000FF731380114A214613801148102209F0EF
:10A39000BBFB6FF008030F4DCDE90243CDE9044448
:10A3A000CDE900440C4B4FF400720C49284606F0EE
:10A3B000E3FF28460A4907B0BDE8304006F0AABFCF
:10A3C0002C0602204806022044060220F80602203D
:10A3D000340602204C060220ADA1040090A5022004
:10A3E000546C0600002110B50D4A13680BB91846CD
:10A3F0000BE083421C680FD141B9516814608B4255
:10A4000000D15460002201201A6010BD0C60506819
:10A41000834208BF5160F5E719462346E6E700BFCF
:10A42000FC0602207047000038B5044680B90123BD
:10A430004FF000020E4963F302020E4B60F3C502B7
:10A440005B1ADB0863F38F120B490C48F8F758FFCF
:10A45000002338210A4A01FB03F0855C1DB110443A
:10A46000C568A54203D00133082BF4D1002038BDC4
:10A47000E44E06009C4F06005D6C0600CE6C0600A4
:10A4800090D702202DE9F74F00260B46B0463546FF
:10A49000DFF8A090009018F0800F3AD13822724374
:10A4A00012F8091091B3009929B109EB02018968EA
:10A4B000009881422AD14A44D76897F82040444501
:10A4C00024D3802C22D807F1100B4FEAD40A184667
:10A4D00052465946019309F087FA019BB0B9C4F17D
:10A4E000800414F007040ED01BF80A2013F80A1099
:10A4F000C4F108005140FF22824082F0FF0202FABC
:10A5000004F4214202D13D4697F820800136082EFE
:10A51000C1D14DB12846FFF765FF054B1A682A6087
:10A520005A681D6002B95D60284603B0BDE8F08F2F
:10A53000FC06022090D7022038B50446D0B1002393
:10A54000C1681A460E48FFF7BFFE2046FFF74AFFD4
:10A550002046FFF769FF054678B164682CB1606852
:10A5600008B1FDF7F5F92468F8E72846FDF7F0F99A
:10A57000002038BD6FF01500FBE76FF00100F8E731
:10A580000C0060F02DE9F0410D46044680B901232E
:10A590004FF00002224963F30202224B60F3C5022E
:10A5A0005B1ADB0863F38F121F492048F8F7A8FEF7
:10A5B00085B901234FF00002194963F30202194BD8
:10A5C00065F3C5025B1ADB0863F38F12164918485E
:10A5D000F8F796FE29462046FEF720F800240746A5
:10A5E00026462546DFF84C8008EB0403D86840B1C6
:10A5F000436833B15A68BA420DD1FFF79DFF60B985
:10A6000001353834B4F5E07FEED10DB906EAE675D0
:10A610002846BDE8F0811B68EBE70646F1E700BF7E
:10A62000E44E06009C4F06006F6C06004F64060067
:10A63000AF6C060090D702202DE9F047A0B3446824
:10A6400094B31A4D1A4BDFF86C80ED1ADFF868905E
:10A65000DFF868A0C5F3C90563685B78FF2B0BD1F1
:10A66000012363F302066FF3C50665F38F163246C6
:10A6700041464846F8F744FE63685A78FF2A10D0EE
:10A68000D86810B10430BDE8F087012363F30207F6
:10A6900060F3C50765F38F173A4641465046F8F711
:10A6A0002FFE2468002CD7D10020ECE79C4F060039
:10A6B000E44E0600886C0600EB6C0600346D060064
:10A6C000F8B507460D4616461C46FDF7A7FF20B114
:10A6D00000233360256001200BE029463846FFF750
:10A6E000D1FE306030B1FFF7A7FF2060003018BF07
:10A6F0000120F8BD2946FBF7D1FC0028F9D0243011
:10A700002060E8E7F8B504460020FDF787FF06461D
:10A71000002847D04078FDF7EDF90546002844D0E1
:10A72000E06AB0B1AF1C6A78394609F05DF998B9B2
:10A7300001234FF000021E4963F302021D4B60F338
:10A74000C5025B1ADB0863F38F121B491B48F8F73D
:10A75000D7FD6FF0150027E094F84430204643F011
:10A76000040384F84430236A1B681A69E2625A7D44
:10A7700084F831201B7D676384F830302B7884F8AF
:10A7800039306B7884F83830B3681A682362527DA8
:10A7900084F831201B685B7D84F83930BDE8F840CF
:10A7A000FAF7C2BB6FF00100F8BD6FF00200FBE7E3
:10A7B000E44E06009C4F06009E6C0600626D06008B
:10A7C0007047026842B9436833B9826822B9C068E9
:10A7D000B0FA80F0400970470020704790F844308C
:10A7E00010B50C460988C3F3C303994216D10A2B4E
:10A7F00016D10A2914D1436999686AB10831043421
:10A800002046FFF7DEFF30B91022204609F0ECF8B1
:10A81000B0FA80F0400910BD1831F0E70020FAE7E7
:10A820000120F8E72DE9F04F112885B00C4604D13E
:10A8300002A9204600F03AF908B902205FE0C38877
:10A84000B0F8029001936369B0F8008098680378CB
:10A8500003F0F003602B06D100210830FAF7A0FDC9
:10A8600008B1C845E9D04FF0FF3A00265746384DA9
:10A87000A5F1180B95F82120D3072AD595F82010BB
:10A88000112926D135F8160CA5F1180108B140455B
:10A890001FD1688808B148451BD1900713D495F89B
:10A8A0002120510705D5002229462046FFF796FFB3
:10A8B00078B17A1C26D195F822209245BCBF0FFAB8
:10A8C00082FA374605E001222046FFF787FF00287D
:10A8D000E5D10136042E05F13C05CBD17B1C24D0FB
:10A8E000206AFBF771FDA0B93C201A4B214600FB02
:10A8F0000730D0E90C32984702289ED0002005B0DE
:10A90000BDE8F08F3C2202FB07B25288002AD2D069
:10A91000DFE76169204600F02BF86169204600F00E
:10A920008BF8019B8342DFD087E794F84430C3F370
:10A93000C3030A2B81D163699B681B7EFF2B3FF405
:10A940007CAF0023324601212046FCF751FE74E71C
:10A950001C07022004070220704710B508220C468D
:10A96000FCF73EFB002814BF2046002010BD00006D
:10A970002DE9F041002786B004460D46ADF814706D
:10A98000FCF720F9064601462046FFF7E6FF58B1DE
:10A99000B771F77111212046FCF7B2FAC043F0807D
:10A9A000284606B0BDE8F0814FF47A780227B4F863
:10A9B000462005AE931D94F8412029461A4492B2D0
:10A9C0000DF11603CDF80880019600972046FCF79C
:10A9D0003BF8112105462046FCF792FAC043BDF82A
:10A9E0001620ADF81400023A2946CDE90168009717
:10A9F0000DF1160392B22046FCF726F80546002812
:10AA0000CED101234FF00002074963F30202074B46
:10AA100060F3C5025B1ADB0863F38F120449054833
:10AA2000F8F76EFCBCE700BFE44E0600B44F06002A
:10AA3000946D0600CA6D06007FB504460E46FCF70D
:10AA4000C1F8054601462046FFF787FF10B1E888A8
:10AA500004B070BDB4F846100DF10E028B1D94F8D1
:10AA600041103046194403AB009389B20223FBF72F
:10AA700077FF80B901234FF00002084963F3020217
:10AA8000074B60F3C5025B1ADB0863F38F120549BD
:10AA90000548F8F735FCBDF80C00D9E7E44E060090
:10AAA000B44F0600A76D0600CA6D06007FB50646C6
:10AAB0000D46FCF787F8044601463046FFF74DFF88
:10AAC00000283AD1B6F8463096F841100DF10E0242
:10AAD000194489B2022300957069FBF741FFAB1C52
:10AAE000BDF80E1000930DF10E020223FBF738FFA4
:10AAF0002B1DBDF80E1000930DF10E020223FBF783
:10AB00002FFFAB1D0093BDF80E1002230DF10E02B6
:10AB1000FBF726FF044698B901234FF000020949CC
:10AB200063F30202084B60F3C5025B1ADB0863F3B0
:10AB30008F1206490648F8F7E3FB204604B070BDC3
:10AB40002C46FAE7E44E0600B44F0600BA6D060044
:10AB5000CA6D060010B50278A2F13003D9B20929F6
:10AB600005D9A2F14103052B1AD8A2F13703427887
:10AB70001B01A2F13001CCB2092C18D80B44827809
:10AB80001B01A2F13001CCB2092C1DD80B44C078B6
:10AB90001B01A0F13002D1B2092922D8D01810BD72
:10ABA000A2F16103052B29D8A2F15703DFE7A2F137
:10ABB0004101052902D8373A1344E0E7A2F16101C7
:10ABC00005291BD8573AF7E7A2F14101052902D818
:10ABD000373A1344DBE7A2F1610105290ED8573A51
:10ABE000F7E7A0F14102052A02D837381844D6E722
:10ABF000A0F16102052A01D85738F7E70020CEE717
:10AC00002DE9F84F0A780646222A01F1010934D0CD
:10AC10004FF00009624B19604846BDE8F88F5C2987
:10AC200014BF01320232013411782046222903D0A8
:10AC300011B1601CF3D100205A4A013012689047CC
:10AC40000746002800F0A98004464FF00A0A4FF09A
:10AC500009084FF00D0B99F80020222A00D07AB98C
:10AC60000022227099F800203761222A4FF0040256
:10AC700008BF09F10109F260CEE74A460024D3E794
:10AC80005C2A09F1010C03D022700134E146E2E7AD
:10AC900099F801206E2A19D007D8622A04F101031D
:10ACA0000CD0662A10D0227012E0742A12D0752AB5
:10ACB00013D0722AF7D184F800B009E0082222707C
:10ACC0001C460CF1010CE1E70C22F8E784F800A027
:10ACD0000134F6E784F80080FAE709F10200FFF793
:10ACE00039FFA0F55C42B2F5806F054609F1050C0D
:10ACF000E7D30028E5D0A0F55842B2F5806F3AD2EC
:10AD000099F806205C2ADCD199F80720752AD8D159
:10AD100009F10800FFF71EFFA0F55C43B3F5806F53
:10AD200009F10B0CCDD2204BC0F3090003EA8525B5
:10AD3000284300F58035B5F5803F23BF05F03F037C
:10AD400063F07F03E370032324BF0423AD0905F000
:10AD50003F0004F1030E60F07F000EF1FF320EF8A9
:10AD6000010CAD0905F03F0060F07F00541E02F8B1
:10AD7000010CAD0903E07F2809D8012301340B4AF7
:10AD8000D25C013B154304F8015C1C4499E7B0F523
:10AD9000006FD0D2A21C0223E4E781463CE700BF4B
:10ADA000F407022054D9022000FC0F00EE6D0600CB
:10ADB0000346184623B102780133013A1F2AF8D915
:10ADC000704710B530B103682BB18468181909F0C9
:10ADD00041F8204410BD1846FCE70000064B10B5B2
:10ADE0001B6828209847044618B12822002108F043
:10ADF0008BFE204610BD00BF54D90220F8B5054691
:10AE00000C4609B9002411E004227549204609F0D6
:10AE10004FF818B90223EB60043407E005227149AA
:10AE2000204609F045F818B9E86005342046F8BD19
:10AE300004226D49204609F03BF818B90123EB6064
:10AE40006B61E9E72378222B05D121462846BDE82E
:10AE5000F840FFF7D5BE2D2B05D0A3F13002092A0B
:10AE60001DD8012302E04FF0FF3301342278302A4D
:10AE700008BF01342278313A082A4FF0000209D87D
:10AE80000A2014F8011B303900FB021221783039F6
:10AE90000929F6D953436B610323EB60C6E75B2BAB
:10AEA00036D10523601CEB60FFF782FF0378044670
:10AEB0005D2B01D10134B9E7FFF790FF0646A8608A
:10AEC00000289FD02046FFF773FF01463046FFF76A
:10AED00095FFFFF76DFF0446002893D003782C2BD5
:10AEE00004D05D2BE6D0414B1C608BE7FFF776FF6B
:10AEF0000546002886D030604660601CFFF758FF8A
:10AF000001462846FFF77AFFFFF752FF2E46E2E799
:10AF10007B2BE8D10623601CEB60FFF749FF037829
:10AF200004467D2BC6D0FFF759FF0646A8600028CF
:10AF30003FF468AF2046FFF73BFF01463046FFF77E
:10AF40005FFEFFF735FF00283FF45CAF0024336954
:10AF50003461336203783A2B02D0244B186065E7E2
:10AF60000130FFF725FF01463046FFF747FFFFF7A7
:10AF70001FFF074600283FF445AF03782C2B03D072
:10AF80007D2B29D1441C51E7FFF728FF05460028F7
:10AF90003FF438AF30604660781CFFF709FF014688
:10AFA0002846FFF72DFEFFF703FF00283FF42AAFE6
:10AFB0002B692C612B6203783A2B02D00B4B186063
:10AFC00020E70130FFF7F4FE01462846FFF716FFA1
:10AFD000FFF7EEFE2E46CCE7044B186012E700BFE9
:10AFE000F56D0600FA6D0600006E0600F4070220FB
:10AFF000F8B5054668B30668F6B1836842685C1820
:10B00000A24201DB1E4417E0013C44EA640444EA26
:10B01000A40444EA241444EA242444EA24440E4BBD
:10B0200001341B68204698470C4F064630B93B68F0
:10B0300028689847C5E900663046F8BDD5E9001292
:10B04000F5F7D8FE3B6828689847C5E90064AB6807
:10B05000D8E70646F0E700BF54D9022050D90220B5
:10B0600070B5064608F0F6FE064B441C1B682046E9
:10B070009847054618B122463146F5F7BBFE2846EB
:10B0800070BD00BF54D90220F8B5D0E90667054667
:10B090000C460022002330463946F5F777FC80B194
:10B0A00054B102212046FFF7A3FF044610B15249D4
:10B0B00008F072FE2046F8BD504B02201B689847EE
:10B0C000F3E76869F5F790F932463B46F5F73EF845
:10B0D00041EC100B06F038FF0022494B51EC100BED
:10B0E000F5F768FC00B33CA3D3E9002330463946AA
:10B0F000F5F760FCC0B10022424B30463946F5F707
:10B1000063FC88B15CB115212046FFF771FF04464E
:10B110000028CFD06A693C4908F0A6FDCAE7374B42
:10B1200015201B689847F2E774B340212046FFF7CB
:10B130005FFF04460028BDD047EC106B06F010FFFF
:10B1400032463B4651EC100BF5F700F841EC100B82
:10B1500006F0FAFE00222A4B51EC100BF5F72AFC00
:10B16000B8B147EC106B06F0EFFE1DA3D3E9002346
:10B1700051EC100BF5F714FC58B132463B4623490D
:10B18000204608F071FD95E71C4B40201B6898474E
:10B19000CFE747EC106B06F0D7FE13A3D3E90023EB
:10B1A00051EC100BF5F7FCFB18B132463B46184941
:10B1B000E6E747EC106B06F0C7FE0DA3D3E90023CA
:10B1C00051EC100BF5F70AFC0028EED132463B4655
:10B1D0001049D5E7AFF300800000C0FFFFFFDF415B
:10B1E00044F3C2E4E4E9634C8DEDB5A0F7C6B03E8C
:10B1F0000000000065CDCD413280060054D9022008
:10B200000000B03C0000E0C111530600086E0600CB
:10B210000D6E0600106E06002DE9F0470346064647
:10B2200088460022194611F8014BCCB95ABB9C1B29
:10B23000E11CB8F1000F21D04046FFF7D9FE0546CA
:10B2400058B12227431C07703146184608F0A4FD68
:10B2500003460022234407555A702846BDE8F0876C
:10B26000631E1E2B08D9222C06D0A4F15C035C427D
:10B270005C4122430B46D5E70124FAE7414B0846DF
:10B280001B689847DBE796B9B8F1000F0AD0032195
:10B290004046FFF7ADFE05460028DED03A4908F0EB
:10B2A0007BFDDAE7374B03201B689847F3E7B1468D
:10B2B0003778DFF8D8A017B1651C1AD12C46E11CED
:10B2C000B8F1000F23D04046FFF792FE0546002854
:10B2D000C3D022235C274FF06608DFF8B490441CEB
:10B2E0000370013E16F8013FB3B922226370227049
:10B2F000B3E73946504608F0D9FC20B1A51C19F82F
:10B30000017F2C46D7E71F2F98BFA51DF7E71D4BE0
:10B3100008461B689847D9E71F2B04F1010006D99E
:10B32000222B04D05C2B02D023700446DAE727706E
:10B3300032780C2A16D009D8092A1AD00A2A15D030
:10B34000082A19D16223A01C6370EEE7222A06D0D6
:10B350005C2A04D00D2A0FD1A01C7223F4E7A01C94
:10B360006270E2E7A01C84F80180DEE7A01C6E2377
:10B37000EAE7A01C7423E7E7494608F075FCA01D26
:10B38000D3E700BF54D90220136E0600166E0600E4
:10B390001E6E06002DE9F04F80468946002685B0D6
:10B3A0001C460368019273B9AEB97CB103212046F3
:10B3B000FFF71EFE834610B1714908F0EDFC5846B8
:10B3C00005B0BDE8F08F01361B68ECE76D4B03203C
:10B3D0001B689847EEE7002C4CD0012120460293D1
:10B3E000D4F808B0FFF704FE029B10B94FF0000B31
:10B3F000E5E75B220270A2684FF02C0A0132A260DE
:10B40000019A1E46002A14BF02270127D8F80050CF
:10B4100009F1010907F101085DB902212046FFF792
:10B42000E7FD0028E2D05D234570037023689B444C
:10B43000C5E72346019A4946284600F0A7F820466A
:10B44000FFF7BFFC2B68A06073B141462046FFF7B1
:10B45000CFFD0028CAD0019B80F800A033B9431C5F
:10B460001E70A3683B44A3602D68D5E72022831C8F
:10B470004270F5E7DFF80CA1B700DAF80030384683
:10B480009847CDF808A005460028AFD04FF0050A30
:10B490003A46214608F038FBD8F80080A5F1040BA5
:10B4A00009F10109B8F1000F1BD01CB12C462F4443
:10B4B000354E59E02346019A4946404600F066F869
:10B4C0004BF8040F58B108F0C5FC019B003318BFBE
:10B4D000012302339A448244D8F80080E2E7012431
:10B4E000FAE7002CE2D1029B50461B68984783463E
:10B4F0000028DBD05B230746A84607F8013BDFF8AE
:10B500008890731E44700293D8F80000CDF80C8028
:10B5100008F0A0FC82460246D8F800103846F5F73D
:10B5200069FC029B57449C42039B07D04FF02C02BE
:10B530003A70019AF2B9013700223A70D9F8002026
:10B54000186801349047A64208F10408DCD1D9F804
:10B550000030284698475D233B7000237B702EE720
:10B5600054F8040B00B19847BC423368F8D1284620
:10B5700098473BE72022023707F8012CDCE700BFA1
:10B58000056E060054D9022050D9022010B50028BB
:10B5900052D0047B7BB3062C4ED8DFE804F00F18A2
:10B5A00004212642480005211846FFF721FD0446E4
:10B5B00010B1224908F0F0FB204610BD06211846C4
:10B5C000FFF716FD04460028F6D01D49F2E70521D5
:10B5D0001846FFF70DFD04460028EDD01949E9E7AC
:10B5E0001946BDE81040FFF74FBD1946BDE81040B1
:10B5F0000069FFF711BE062C1ED8DFE804F0090B26
:10B60000040D0F1117000D48BDE81040FFF728BDCD
:10B610000B48F9E70B48F7E70021E2E70021E5E7EF
:10B620000023BDE810400830FFF7B4BE0023BDE89A
:10B630001040083000F008B80024BDE7F56D0600A2
:10B64000FA6D0600006E06002DE9F04F1546002247
:10B6500080468A4689B01C46036801926BB9019BFB
:10B66000002B37D184B16DB10AF104012046FFF7F8
:10B67000BFFC044688B9002417E0019A1B68013218
:10B680000192EBE70321F1E7AA4B1B681DB10AF118
:10B6900004009847EDE70320FBE77B23037045B9DF
:10B6A000431C7D221A7000225A70204609B0BDE862
:10B6B000F08F0A22831C427009251A460AF1FF31D5
:10B6C000D01A814203DC0029A8BF5B18E9E702F821
:10B6D000015BF5E7002C00F09580002D0CBF0127E1
:10B6E00002272046791CD4F80890FFF781FC002837
:10B6F000C1D07B230370F5B9431C00224FF0090B26
:10B700001A70A368D8F800603B44A3600AF10108EE
:10B71000AEB9002D68D00AF102012046FFF768FC9F
:10B720000028A8D0002D6AD17D2303700023437028
:10B7300024684C44B9E70A22831C4270DDE765B1F6
:10B7400041462046FFF754FC002894D003461A1ABD
:10B75000904546DCA3684344A3602146306AFFF766
:10B760005BFD2046FFF72DFB3946A0602046FFF722
:10B770003FFC00283FF47FAF4FF03A0303700DB158
:10B7800080F801B0A3682A463B444146A360304696
:10B790002346FFF7FBFE2046FFF713FB2B1C18BFC9
:10B7A00001233268A060002A18BF01332046591CCB
:10B7B0000193FFF71DFC00283FF45DAF3268019B49
:10B7C0001AB12C22013000F8012C1DB10A220130DF
:10B7D00000F8012C00220270A26836681344A360AE
:10B7E00096E703F801BBB2E7022196E703F8011BD5
:10B7F0001A1A9245FADC2AEAEA79484494E70346A1
:10B800000921F5E7019BDFF82C919F003846D9F814
:10B8100000309847064600283FF42DAFD9F8003095
:10B8200038469847029020B9434B30461B689847EA
:10B830003BE73A462146304608F066F93A4621464B
:10B84000029808F061F90AF10103D8F80070049336
:10B850000DB30AF108040AF1030B002D14BF5B4677
:10B8600000234FF0000B029A0233A2F10409321FA9
:10B87000039205938FB9BBF1000F33D02E4D0024F6
:10B880002F46019A2B68A24243D1029898472B6811
:10B8900030469847EFE60724DDE70021386AFFF7D6
:10B8A000BBFC2A4649F8040F804600230499384619
:10B8B000FFF76CFE039A42F8040F0392B8F1000FF1
:10B8C0000DD060B108F0C6FA0690404608F0C2FA02
:10B8D000059B1C44069B1C4404443F68CAE74FF088
:10B8E000010BFAE7134B20461B68984704460028D3
:10B8F000C4D07B230370C5B9471C00233B70049B55
:10B90000DDF8089023EAE3730396079305B33B46FB
:10B9100018E0029A52F8240000B1984756F8240023
:10B920003B6800B198470134ABE70A23871C43709A
:10B93000E3E700BF54D9022050D902204FF009029A
:10B9400003F8012B0499DA1B9142F7DC079B1F4493
:10B95000D9F80000CDF8149008F07CFAD9F800105E
:10B96000804602463846F5F745FA3A2307EB0802C7
:10B9700007F80830002D40D102F10108039B404632
:10B980001968069308F008FA039B186808F062FA31
:10B99000019B08EB00075A1E93451EBF2C2201375E
:10B9A00008F800201DB10A23013707F8013C0023E5
:10B9B000DFF86C803B70059BD8F800201868904732
:10B9C000039BD8F8002004330393069B0BF1010B73
:10B9D00018689047019B09F104095B4596D10298CC
:10B9E000D8F800209047D8F8003030469847A5B9DD
:10B9F0007D233B7000237B7057E64FF0090302F173
:10BA000002085370BAE703F8011BDA1B9245FADC0F
:10BA1000BAF1000FA8BF5744EAE73B460921F4E713
:10BA200050D902202DE9F84320B9081C18BF012085
:10BA3000BDE8F883002937D08946471E17F8016F03
:10BA400007F0ACFC30444378C84603F00303012BF5
:10BA500008BF203619F8015B07F0A0FC2B462844EC
:10BA600042783C7802F00302012A08BF20339E424C
:10BA700016D007F093FC2044437898F8005003F068
:10BA80000303012B08BF203407F088FC2946284413
:10BA9000437803F00303012B08BF2031601AC7E786
:10BAA000002CCBD12046C3E70120C1E710B50A49DD
:10BAB0000A4A20B90A4B0B600A4B136010BD036899
:10BAC000074C002B08BF23460B6043680549002B39
:10BAD00008BF0B46F1E700BF54D9022050D902201D
:10BAE000B9330500C933050070B504460E4D04B9DD
:10BAF00070BDE3682668D90503D4A06808B1FFF7D4
:10BB0000F3FFE368DA0503D4206908B12B6898478E
:10BB1000E3689B0503D4206A08B12B689847204648
:10BB20002B6898473446E2E750D902202DE9F843C4
:10BB300005460E4691460027FFF750F9DFF8508082
:10BB40000446C8F8007060B12846FFF731F9014695
:10BB50002046FFF753F9054630B92046FFF7C4FFEA
:10BB60002C462046BDE8F883B9F1000F0BD0FFF753
:10BB70001FF90378054633B12046FFF7B5FF3C4671
:10BB8000C8F80050EDE7002EEBD03560E9E700BFC4
:10BB9000F407022000221146FFF7C8BF00231A460F
:10BBA0001946FFF7F3BC38B50D46846824B1294621
:10BBB000206AFFF737FF08B9204638BD2468F5E74B
:10BBC00049B1836813B98160704713461A68002A27
:10BBD000FBD119604B60704770B505460E461446A0
:10BBE00072B1106A10B1074B1B6898473046FFF7D7
:10BBF00037FA214620622846BDE87040FFF7E0BFD3
:10BC000070BD00BF50D9022008B5FFF7E7F808B1B2
:10BC10000223C36008BD13B58DED000BFFF7DEF8FE
:10BC2000044650B19DED000B032380ED060BC3606D
:10BC300051EC100BF4F7DCFE6061204602B010BD41
:10BC400038B50546FFF7CAF8044628B10423C36097
:10BC50002846FFF705FA2061204638BD08B5FFF7F2
:10BC6000BDF808B10523C36008BD08B5FFF7B6F8F5
:10BC700008B10623C36008BD2DE9F04180460F4698
:10BC80000025FFF7EBFF2C4606460EB1BC4202DB57
:10BC90003046BDE8F08158F82400F4F7A5FB41ECEC
:10BCA000100BFFF7B8FF1CB9B06001340546ECE794
:10BCB00028604560F9E704F0B8BC04F0BBBC0000A4
:10BCC0000348044B0360044B4360FFF7EFBE00BF23
:10BCD000F8070220BBBC0400B7BC0400002208B572
:10BCE00011462A20F8F7FEFC0DF0ECFA002008BD02
:10BCF000684620F007018D4601B5F8F731FD0FF0D9
:10BD0000B7FEF8F71FFDF8F713FBBDE801408546C5
:10BD10007047684620F007018D4601B5F8F720FD11
:10BD20000DF022FCF8F70EFDF8F702FBBDE801402C
:10BD300085467047684620F007018D4601B5F8F743
:10BD40000FFD0DF043FFF8F7FDFCF8F7F1FABDE841
:10BD5000014085467047002070472F2810B50446E3
:10BD600072D027DC162809D012DC092806D009DC9D
:10BD7000022803D0052801D0012817D1F8F740FF89
:10BD8000046010BD0D28F9D00E28F7D00C28F4E778
:10BD90002A2849D005DC23283DD0292840D018285E
:10BDA000EBE72C2848D043DB2D2849D0F8F728FFB3
:10BDB000162333E06928E1D016DC362850D009DCA0
:10BDC000322845D0332847D03028EFD1F8F718FF74
:10BDD000702323E0392847D03C2849D03828E5D1C2
:10BDE000F8F70EFF7F2319E07E284DD009DC732879
:10BDF00042D07D2844D07028D8D1F8F701FF7523B0
:10BE00000CE080284AD044DB8128CFD1F8F7F8FE37
:10BE100040F2D47302E0F8F7F3FE0B230360B0E7BF
:10BE2000F8F7EEFE6B23F9E7F8F7EAFE6D23F5E786
:10BE3000F8F7E6FE7B23F1E7F8F7E2FE7C23EDE777
:10BE4000F8F7DEFE5F23E9E7F8F7DAFE6A23E5E7B5
:10BE5000F8F7D6FE7323E1E7F8F7D2FE7223DDE7A9
:10BE6000F8F7CEFE6823D9E7F8F7CAFE8023D5E7B6
:10BE7000F8F7C6FE7423D1E7F8F7C2FE7723CDE7C3
:10BE8000F8F7BEFE8C23C9E7F8F7BAFE40F2D1738B
:10BE9000C4E7F8F7B5FE40F2D273BFE7F8F7B0FE9B
:10BEA00040F2D373BAE700004FF08052014BC3F861
:10BEB0000021704700E100E04FF08052014BC3F8D1
:10BEC0008021704700E100E04FF00052014BC3F8C1
:10BED0000021704700E100E04FF00052014BC3F831
:10BEE0008021704700E100E008B51D2000220621F6
:10BEF000F8F7F8FBBDE808401D20F8F7CFBB08B500
:10BF00001C2000220621F8F7EDFBBDE808401C20AC
:10BF1000F8F7C4BB30B589B06C46074D0FCD0FC4E0
:10BF200095E80F0084E80F00002269460348F6F701
:10BF30007DFF09B030BD00BF08500600246E06002A
:10BF400008B5FFF7DCFFFFF7E5FFBDE80840FFF7A6
:10BF5000CBBF00002DE9F04107460D460C46DFF847
:10BF6000248014B92046BDE8F081FF2C264628BF66
:10BF7000FF26291B324639444046F6F7FFFFA41B33
:10BF8000EFE700BF246E06000138052812D8DFE86D
:10BF900000F00307090B0D0F02230B600020704710
:10BFA0000523FAE70623F8E70723F6E70423F4E777
:10BFB0000123F2E74FF0FF30704710F0400318BF45
:10BFC0000223820748BF43F0080318467047112830
:10BFD00014D005DCC0B1062815D06FF07A00704788
:10BFE00040F2111398420BD040F2012398420BD03B
:10BFF000B0F5817FF1D14FF4827070470220704715
:10C000004FF48770704701207047000008B5024860
:10C01000F7F726FF002008BD2C6E060038B5044651
:10C0200004B938BD6069E56904F0FFFA204604F000
:10C03000FCFA2C46F4E770B5044618461546FFF79F
:10C04000BCFF2A4603462046BDE8704010F08AB97E
:10C0500070B5044618461546FFF7AFFF2A4603465B
:10C060002046BDE8704010F0C9B9F0B591B0044663
:10C070000D46164600214022684607F045FD042380
:10C080000022AA420CDB32462946684610F06CFAC0
:10C090000022062316460127AA4221DB11B0F0BD7B
:10C0A00054F832104DF83210E15A0132CF0742BF36
:10C0B0003DF8030040F001002DF80300480742BF9F
:10C0C0003DF8030040F002002DF80300090742BFCD
:10C0D0003DF8031041F004012DF803100833D0E7B8
:10C0E0003DF80310E65211F0010F18BFE75289071F
:10C0F00048BFE15A02F1010244BF41F00401E1529C
:10C100000DEB030131F8021C490742BFE15A41F02F
:10C110000801E1520833BFE710F0B2B910F0F8B8E7
:10C120000B894A684380034630B523F8042B01F19C
:10C13000100202F1100452F8045BA24243F8045BBF
:10C14000F9D10B6A037530BD2DE9F047002514467F
:10C150008AB006460F462022294602A89846019535
:10C1600007F0D2FC44B32022294602A807F0CCFCF9
:10C170006368E0680393A3680493FFF728FF0590C2
:10C180007B3000F0858002AA3946304601AB10F0C2
:10C19000E7F90027019EC8F800704FF0110940F23E
:10C1A000111A054600284ED0D8F80000FFF736FFD8
:10C1B0000023C8F8003048E02246E5E7202004F0DC
:10C1C00039FA044600285ED0B36872688360F36869
:10C1D000C0E90655022B056042603FD00EDC002B03
:10C1E0003AD0012B3DD06FF07A03E3600023636106
:10C1F000204604F01AFA6FF00605D5E7B3F5877FFD
:10C200000AD040F201218B4204D0B3F5827FEAD1FB
:10C210004FF48173E36001E0C0F80CA0022A22D140
:10C22000082004F007FA606150B3082372692361A3
:10C230001389438053680380D368436037BBC8F8D1
:10C2400000402746F669002EB8D1019810F08AF90F
:10C2500028460AB0BDE8F087C560DFE7C0F80C905B
:10C26000DCE70623D6E70A2AC2D1182004F0E2F957
:10C27000606128B1182371692361FFF751FFDDE781
:10C28000204604F0D2F96FF009058DE7FC61D8E78C
:10C290006FF00605DCE72423F0B50B7043880A46EF
:10C2A0000B810346044633F8041B02F1100651606B
:10C2B00000F11407354618685968083303C5BB42B6
:10C2C0002E46F7D1237D1362F0BD2DE9F0438DB0EA
:10C2D000149C05460E46174698466CB91846FFF75B
:10C2E0006CFECDE9004403463A463146284610F03C
:10C2F0001DF80DB0BDE8F0832388022B0FD110216B
:10C30000628804936368404606938DF80C10ADF87C
:10C310001420FFF752FE03AB01910093E3E70A2BD1
:10C320000CD10DF10C0949462046FFF7B4FF4046F9
:10C33000FFF743FE2423CDE90093D4E7F8F760FC30
:10C340006FF0850303604FF0FF30D2E72DE9F0472F
:10C35000814686B01846DDE90E469246FFF72DFE6F
:10C36000034654B9CDE900445246484610F02AF835
:10C370000546284606B0BDE8F0874FF0080806AD30
:10C3800045F80C8D04AF019500975246484610F0D1
:10C3900019F8059B0546022B08D1BDF8182023800B
:10C3A000079B62806360C6F80080E2E70A2BE0D159
:10C3B00039462046FFF7B4FE18233360D9E7B1F5BC
:10C3C0008D7F7FB505460C461E460FD103A910464A
:10C3D000FFF7DAFD002809DB089B039A009321464A
:10C3E0003346284610F084F804B070BDF8F708FC16
:10C3F0006FF06C0303604FF0FF30F5E7F0B50827EE
:10C4000085B0164604AA0C4642F80C7D0DEB0701D8
:10C4100010F046F8051E1ADB039B022B09D137608A
:10C42000BDF810202380059B62806360284605B01C
:10C43000F0BD0A2B06D1182302A933602046FFF76E
:10C440006FFEF3E7F8F7DCFB6FF0850303604FF056
:10C45000FF35EBE738B505461046FFF7B8FD10F19C
:10C460007B0F044605D002462846BDE838400FF051
:10C470003DBFF8F7C5FB04604FF0FF3038BD10B585
:10C480000B4609888AB0022904460DD110225C8827
:10C490005B6802918DF80420ADF80C40049301A96B
:10C4A00010F014F80AB010BD0A2907D101A91846E6
:10C4B000FFF7F1FE242201A92046F1E7F8F7A0FBDF
:10C4C0006FF0850303604FF0FF30EBE7B1F58D7F30
:10C4D0007FB505460C461E460ED103A91046FFF750
:10C4E00053FD002808DB089B21460093284633466D
:10C4F00010F01AF804B070BDF8F782FB6FF06C030F
:10C5000003604FF0FF30F5E710B50B4609888AB09D
:10C51000022904460DD110225C885B6802918DF8D7
:10C520000420ADF80C40049301A90FF097FF0AB066
:10C5300010BD0A2907D101A91846FFF7ACFE242235
:10C5400001A92046F1E7F8F75BFB6FF08503036074
:10C550004FF0FF30EBE7000038B513460C4661B9E9
:10C56000074D184695F851202946F4F743FC95F8F5
:10C57000512080F85120204638BD6FF08500FBE740
:10C58000FC0C0220000000002DE9F04F4E4B9DB046
:10C59000D3E900454FF6FF7605F014FAB0FBF6F349
:10C5A000C3EB0343C01AF3F70FFF41EC100B05F088
:10C5B0005FFD43A3D3E9002351EC100BF3F77EFF9B
:10C5C00022462B46F3F7C4FD404B8B46D3E9008946
:10C5D000824605F0F7F9B0FBF6F6C6EB0646801B7F
:10C5E000F3F7F2FE41EC100B05F04EFC34A3D3E957
:10C5F000002351EC100BF3F761FF42464B46F3F773
:10C60000A7FD0F46064605F0DDF94FF47A73B0FB3F
:10C61000F3F02F4A2F4913780C68DFF8CCC01B1BAE
:10C620000344DBB23B2B086013702B481DD94FF03D
:10C630003C0EB3FBFEF10EFB113313700378013394
:10C64000DBB23B2B037010D9B3FBFEF80EFB1833A3
:10C650004FF0180E9CF8001003704B1CDBB2B3FBBC
:10C66000FEF10EFB11338CF80030CDE90467CDE903
:10C6700002AB12789CF800300192027851210092AE
:10C6800007A8164A07F0A8FA00231A4607A9194472
:10C6900049782A290DD1124C009207AB114A512139
:10C6A000204607F099FA84F8510000201DB0BDE83B
:10C6B000F08F0133522B01D04A40E7E70022EAE72E
:10C6C0007B14AE47E17A743F00080220080802207C
:10C6D0005AD90220F80C022059D90220986E06007F
:10C6E000FC0C0220D96E060058D902200B7870B5D8
:10C6F000012B0D46164684680CD14FF0FF310F48D0
:10C7000003F0F4FF2B880D482663A38604F04EF84F
:10C71000002070BD01234FF00002094963F30202BB
:10C72000084B6FF3C5025B1ADB08074863F38F12EF
:10C730000649F6F7E5FD6FF08500EAE7500D0220A7
:10C74000E44E0600EC4E0600E06E0600766E060033
:10C7500070B5064618A1D1E90001134B86B0C3E9B4
:10C7600000010FA1D1E90001104B0024C3E9000131
:10C770000F48B56803F0B4FF6FF00503CDE904443A
:10C78000CDE90243CDE900640A4B4FF4806205F124
:10C79000380105F5876004F0EFFD204606B070BD56
:10C7A000FCA9F1D2CD089040000802200808022020
:10C7B000500D0220C1C70400E17A14AE47B5B8405D
:10C7C00070B5054686680A4C4FF4FA6004F01CFC0C
:10C7D0004FF0FF31204603F089FF336B1BB106F1A8
:10C7E000340128469847204603F0E0FFECE700BFFD
:10C7F000500D022000000000D0B514460F4606463A
:10C80000F4F7F6F82060F3F7EFFD02460B463046EA
:10C810003946F3F79BFC04A3D3E90023F3F74EFE5C
:10C82000F4F7E6F86060D0BD0000000080842E417F
:10C830000020704738B51446032922D8DFE801F0FC
:10C8400002090D11104BD3E90001FFF7D5FF0020BD
:10C8500038BD0D4BD3E90201F7E70B4BD3E90401D7
:10C86000F3E7094DD5E90001FFF7C6FFD5E902015D
:10C8700004F10802FFF7C0FFD5E9040104F110023A
:10C88000E3E76FF08500E3E7680D022008B58368F1
:10C890000878012804D100201A630A889A8608BD06
:10C8A00001234FF00002084963F30202074B6FF3C4
:10C8B000C5025B1ADB08064863F38F120549F6F7D9
:10C8C0001FFD6FF08500EAE7E44E0600EC4F06001E
:10C8D0002C6F0600046F060008B505F073F84FF6DC
:10C8E000FF73B0FBF3F3C3EB0343C01AF3F76CFD24
:10C8F00041EC100B05F0BCFB0022054B51EC100B7A
:10C90000F3F7DCFD00220023F3F722FC08BD00BF93
:10C910000000344030B56FF005030024856887B00F
:10C92000CDE90243CDE90004CDE90444054B4FF4C1
:10C93000007205F1380105F50E7004F01DFD20466A
:10C9400007B030BD49C9040070B50446856805F1DB
:10C9500034064FF47A7004F057FB2B6B002BF8D0A1
:10C96000314620469847F4E7022838B5284C294D2F
:10C9700025D003282FD0012815D0FFF7ADFF286858
:10C98000F3F732FD0022244BF3F798FDC4E90001D0
:10C990002868F3F729FD01F100431946F4F728F858
:10C9A0002860002038BDFFF797FF2868F3F71CFDCB
:10C9B0000022194BF3F782FDC4E90201E8E7FFF713
:10C9C0008BFF2868F3F710FD0022134BF3F776FD79
:10C9D000C4E90401DCE7FFF77FFFC4E9000101209F
:10C9E00004F012FBFFF778FFC4E90201012004F014
:10C9F0000BFBFFF771FF2868F3F7F6FC0022064BEC
:10CA0000F3F75CFDC4E90001C4E90201E0E700BFFF
:10CA1000680D02205CD9022000003440012908B5CD
:10CA2000084602D005D3022905D1FFF79DFF00205B
:10CA300008BD0020F9E70320F7E700002DE9F843DF
:10CA400006460F460024DFF87080DFF8709026FA63
:10CA500004F327FA04F21A43D2071FD5D8F80000CE
:10CA600003F0010342680021556819F80420A84723
:10CA7000054698B101234FF000020B4963F302020F
:10CA80000A4B6FF3C5025B1ADB0863F38F12084988
:10CA90000848F6F735FC2846BDE8F8830134042C35
:10CAA000D5D10025F7E700BFE44E0600E44E0600AE
:10CAB0008F6F060041700600803A02205B7006000E
:10CAC0002DE9F341002425462C4E2D4F30687A5D28
:10CAD00043680021D3F8088001ABC04700283FD04D
:10CAE00001234FF00002274963F30202264B6FF344
:10CAF000C5025B1ADB0863F38F1224492448F6F75A
:10CB0000FFFB244BD3E8EF2FC3E8E14F0029F9D115
:10CB1000214B224D1A7872BB214B1B682BB129681F
:10CB2000A14202D06140204698470A221D491E4872
:10CB30002C6004F0ADFD80B101234FF000021149DB
:10CB400063F30202104B6FF3C5025B1ADB0863F359
:10CB50008F1216491648F6F7D3FB02B0BDE8F081F4
:10CB6000019BDB4303F00103AB400135042D44EA94
:10CB70000304ABD1C5E700221A70D6E7803A022041
:10CB8000A16F0600E44E0600E44E0600566F060054
:10CB9000A56F06009410022060D902208C1002209C
:10CBA000681002206C100220C87B0220626F060011
:10CBB000BE6F0600F8B5204803F0E2FA1F4D28606A
:10CBC000A0B901234FF000021D4963F302021D4B7F
:10CBD00060F3C5025B1ADB0863F38F121A491B4826
:10CBE000F6F78EFB6FF012063046F8BD0024184FA2
:10CBF00028683A5D436800211E680123B047064655
:10CC000088B101234FF000020D4963F302020D4B7E
:10CC10006FF3C5025B1ADB0863F38F120A490D48F4
:10CC2000F6F76EFBE0E70134042CE1D1BDE8F840F3
:10CC30000F21FFF703BF00BF00700600803A0220FB
:10CC4000E44E0600E44E0600726F06000770060010
:10CC50005B70060023700600054BD3E8AF3F00B1C0
:10CC60000360044811B102685A400A6003607047CB
:10CC70009410022090100220F8B508B12E4B1860D5
:10CC80002E4803F07DFA2E4E3060A0B901234FF0FC
:10CC900000022C4963F302022B4B60F3C5025B1ABE
:10CCA000DB0863F38F1229492948F6F729FB6FF057
:10CCB00012042046F8BD0025264F30687A5D43688F
:10CCC00000211C684FF48073A047044688B10123FB
:10CCD0004FF000021B4963F302021B4B6FF3C502C6
:10CCE0005B1ADB0819491C4863F38F12F6F708FB3F
:10CCF000DFE70135042DE0D11849194804F076FC2E
:10CD000022461749174804F0C3FC044678B10123B2
:10CD10004FF000020B4963F302020B4B6FF3C502A5
:10CD20005B1ADB0863F38F1208490F48DEE7014600
:10CD3000FFF792FFBDE700BF6810022000700600F9
:10CD4000803A0220E44E0600E44E06007F6F0600A3
:10CD500007700600A16F0600DF6F0600C1CA04005D
:10CD60006C100220C87B0220BE6F060040EA01035F
:10CD700033F00F0301D1FFF761BE6FF0150070476C
:10CD80000F21FFF7F3BF10B51C688C420DD2091BB1
:10CD900001290AD0115D224409020180527802342F
:10CDA0001143018000201C6010BD6FF01500FBE7EF
:10CDB000F0B5002426461D688D4210D210F805C03B
:10CDC00001350CF07F07A7401CF0800F04F1070429
:10CDD0003E44E4B2F0D100201D601660F0BD6FF05B
:10CDE0001500FBE710B59A42029C02D86FF01500BF
:10CDF00010BD90F85400042808BFC85C03F101037B
:10CE000004BF00F0010020709A42EFD9CB5C0020F3
:10CE10006370EDE72DE9FF411C469B7D0DF1100885
:10CE20006FF30003A37548F80C2D0278054662F3F2
:10CE30004103A37503780246C3F3410323720DF146
:10CE40000E0043460E46FFF79EFF00230746C4E947
:10CE5000003300BB019BBDF80E20F11A91420DD3A7
:10CE60000AB1E918216013440193237A626043B93F
:10CE7000019A0023964212D2C4E903336FF01507DA
:10CE800009E043462A46314604F11400FFF77BFFD0
:10CE90000028EDD00746384604B0BDE8F081B61A48
:10CEA000C4E90333F7D01544C4E90356F3E737B5B3
:10CEB0001D4602AC44F8042D234602462846FFF7DF
:10CEC00062FF03B030BD37B51D4602AC44F8042DF7
:10CED000234602462846FFF756FF03B030BD37B55C
:10CEE0001D4602AC44F8042D234602462846FFF7AF
:10CEF0004AFF03B030BD37B51D4602AC44F8042DDF
:10CF0000234602462846FFF73EFF03B030BD73B507
:10CF100006461C4602A840F8042D03463246204629
:10CF20000D46FFF730FF48B9019B9D4208D3ED1A2B
:10CF3000C4E9010002D01E44C4E9016502B070BD1D
:10CF40006FF01500FAE737B51D4602AC44F8042D22
:10CF5000234602462846FFF716FF03B030BD10B542
:10CF600040F2FA741368A3420ED8C3F5FF64033489
:10CF7000012C09D0040ACC541368194448700020CD
:10CF800013680233136010BD6FF01500FBE7F8B5AE
:10CF9000064640F2FA7013680F468342154617D8CA
:10CFA0007068C3F5FF630333841CA34213D380B2BC
:10CFB000FFF7D5FF044648B91068D6E90012384497
:10CFC000F3F718FF2B68726813442B602046F8BDF6
:10CFD0006FF01504FAE76FF00B04F7E770B50B4636
:10CFE00000240134DB09A4B2FBD1E44315682E19F7
:10CFF00028550C4604F07F0598B2E40900F10100C1
:10D0000018BF65F07F0535540133002CF2D1013192
:10D01000166011FA80F070BD2DE9F34100248846B6
:10D020001E46089F0094154622B3036840F2FB7227
:10D03000053321461846019306F066FD6A4601460F
:10D040002846FFF78CFF054688B90099B1F1805F4B
:10D050000AD201AA4046FFF7C1FF019B3860336046
:10D06000284602B0BDE8F0814FF0FF30F5E73C60A4
:10D070003460F5E76FF01505F2E700002DE9F7439E
:10D080000F460021036C90F855400546904690F8F5
:10D0900054004E4A4E4E0533042808BF1646184623
:10D0A00040F2FB720193009106F02EFD6A460146A4
:10D0B0003046FFF76CFFC4F34004034670B9DDE966
:10D0C000002140F2FA76B24288BF6FF0150395F85E
:10D0D00054009FBF8854009A01320092DDF80090FE
:10D0E00009F101020092002B65D16A46019978206E
:10D0F000FFF735FF034600285DD16A46019905F127
:10D100004C00FFF744FF064600285DD1E86A640042
:10D11000F0B16A460199FFF73AFF034600284AD169
:10D12000EB6A95F855201B7A02F00102DB0044F00F
:10D13000040403F0180344EA42141C432B6B0199C6
:10D140006A4663B31846FFF722FF0346002832D130
:10D15000686A48B16A460199FFF719FF034650BB58
:10D16000A86AF8B944F0800495F85400C31E5842E8
:10D1700058412B6C994489F805400099B1F1805FC2
:10D180001FD2400001AA40F01000FFF727FF019BCB
:10D19000C8F800003B60304603B0BDE8F083FFF7FD
:10D1A000DEFED2E76A460199FFF7F1FE44F0C004C3
:10D1B00003460028D8D000221E46C8F800203A6056
:10D1C000E9E74FF0FF30E2E70346F4E7947006002A
:10D1D00084700600F7B51F46002300930B7A0C46B7
:10D1E000164613B18B8A002B54D0036C40F2FB72AD
:10D1F000053300211846019306F086FC6A46014675
:10D200002046FFF7C4FE054640B9237A5BB940F2D9
:10D21000FA72009B93420ED96FF015000023054669
:10D220003B6033602DE06A460199A08AFFF797FEC4
:10D230000028F3D1EBE72269C3F5FF610331914286
:10D2400025D30198E1681844F3F7D4FD00992369C8
:10D250001944B1F1805F009116D2A37D01AA03F0B9
:10D260000100C3F3400343F0300343EAC003207AD4
:10D27000400000F006001843FFF7B0FE019B386045
:10D280003360284603B0F0BD4FF0FF30F6E76FF093
:10D290000B00C3E76FF01505F3E707B509880093A6
:10D2A00013460A4640210844FFF7B6FE03B05DF876
:10D2B00004FB0000024B00200B6002231360704748
:10D2C000807006002DE9F74F0D4600211F46EB88C0
:10D2D00016460091002B3AD0036C40F2FB720533E6
:10D2E0001846019306F010FC6A460146E888FFF7ED
:10D2F00036FE044698BB80464FF00C0940F2FA7A9D
:10D3000009FB08FB28686A4601995844FFF73FFE6D
:10D31000044620BB2B685B44197ADDE90032534593
:10D320001BD8D1540099AB8808F10108013143455D
:10D330000091E5D8B1F1805F02D34FF0FF3003E0F8
:10D3400001AA8220FFF74AFE3860019B09E06FF0D6
:10D350001504204603B0BDE8F08F6FF015040023DC
:10D360003B603360F5E72DE9F7430E460021984610
:10D37000036C1746053340F2FB7218460091019387
:10D3800006F0C2FB6A460146F088FFF7E8FD044656
:10D39000F0B905464FF00C0930686A4609FB0500F4
:10D3A0000199FFF7F4FD0135044688B9B388AB4213
:10D3B000F2D80099B1F1805F02D34FF0FF3003E063
:10D3C00001AAA220FFF70AFEC8F80000019B02E0B4
:10D3D0000023C8F8003020463B6003B0BDE8F0836E
:10D3E000024B00200B60022313607047A070060000
:10D3F00000232DE9F04F80468A4616468FB00DF186
:10D40000380949F8283D0393049FB74243D2039B50
:10D410000AEB07050593012305AA0493F11B4B466C
:10D420002846FFF7C5FC002840F08680DDE904248B
:10D430001444B4F5006F2DD807EB040BB3457DD829
:10D440001AF807300D9003F0F003502B50D026D877
:10D45000302B39D0402B42D0202B25D107AB8DF873
:10D46000180000932946134640462246FFF7BAFCAF
:10D47000054690BB9DF81D202AB9D8F83C3043F0F2
:10D480000403C8F83C300D92002206A9404600F083
:10D49000C3F94DB1264630460FB0BDE8F08F702B72
:10D4A00038D004D8602B2CD0CDF810B0ACE7902B3E
:10D4B00039D0B02BF8D1082321468DF818302846F2
:10D4C00007ABFFF740FD07E0022321468DF8183037
:10D4D000284607ABFFF79EFC05460D95D4E70323CE
:10D4E00021468DF81830284607ABFFF7E0FCF3E73C
:10D4F000042321468DF81830284607ABFFF7E3FCDC
:10D50000EAE7052321468DF81830284607ABFFF7D8
:10D51000E6FCE1E7062321468DF81830284607ABE4
:10D52000FFF7E9FCD8E7072321468DF81830284695
:10D5300007ABFFF7ECFCCFE73446ABE73C46A9E787
:10D540000E4B10B51B684BB90D4821230D4A0E49EF
:10D55000F5F7ECFB0D48F5F7E9FBFEE75B684BB927
:10D5600007482223074A0A49F5F7E0FB0748F5F781
:10D57000DDFBFEE7BDE81040184700BF7C3A022003
:10D58000D9520600BB700600F6700600F75206007E
:10D590000171060070B5274D066A2B680446308875
:10D5A0004BB925481923254A2549F5F7BFFB2548DE
:10D5B000F5F7BCFBFEE71B684BB91F481A231F4A4F
:10D5C0002149F5F7B3FB1F48F5F7B0FBFEE706224C
:10D5D000012198470028606004DAF7F711FB006822
:10D5E000404270BD3388022B2B6814BF18220822DA
:10D5F0004BB911484523114A1149F5F797FB1148DA
:10D60000F5F794FBFEE75B694BB90B4846230B4AE1
:10D610000E49F5F78BFB0B48F5F788FBFEE7216A0F
:10D620009847002803DA6068FFF78AFFD5E70020F3
:10D63000D7E700BF7C3A0220D9520600BB70060033
:10D64000F6700600F75206001371060026710600F8
:10D650002DE9F8430746884615460024DFF8709008
:10D66000AC4201D3002024E0D9F80030786808EB00
:10D6700004012A1B4BB911487E23114A1149F5F7C1
:10D6800055FB1148F5F752FBFEE7DE6A4EB90B4831
:10D690007F230B4A0D49F5F749FB0B48F5F746FB8D
:10D6A000FEE70023B047002805DAF7F7A9FA00687B
:10D6B0004042BDE8F8830444D2E700BFD9520600D7
:10D6C000BB700600F6700600F75206004B710600AC
:10D6D0007C3A022038B5144B14461B684068126827
:10D6E0004BB912486923124A1249F5F71FFB124839
:10D6F000F5F71CFBFEE75D6A4DB90C486A230C4A3E
:10D700000E49F5F713FB0C48F5F710FBFEE7402335
:10D71000A847002804DAF7F773FA0068404238BDDA
:10D7200020600020FBE700BF7C3A0220D9520600AF
:10D73000BB700600F6700600F75206003A7106004C
:10D7400008B54068FFF7FCFE002804DAF7F758FA3E
:10D750000068404208BD0020FCE700000378024A50
:10D760001B01D358184700BF7071060010B4044B5A
:10D77000047803EB04135B685DF8044B184700BFA3
:10D780007071060010B4044B047803EB04139B681B
:10D790005DF8044B184700BF707106000278024B19
:10D7A00003EB0213DB68184770710600014802F0B2
:10D7B000FDBF00BF843A0220030706D410F0040F17
:10D7C0000CBF6FF07F00002070476FF00F007047B4
:10D7D0004FF0FF31014802F089BF00BF843A0220B8
:10D7E00037B50025036C0446C56333B102A941F87F
:10D7F000043D084802F012FE2564636C3BB102A9A7
:10D8000041F8043D034802F009FE0023636403B0BD
:10D8100030BD00BF983A022070B5446B05460E46F5
:10D8200044B1FFF7C3FF31462846A047BDE870402A
:10D83000FFF7CEBF70BD00000F4B10B51A6888B05F
:10D84000904204BF00221A60C36B044613F0140315
:10D8500013BF01238DF800306FF06E03079114BFE2
:10D860008DF800300793FFF7BBFF01226946204681
:10D87000FFF7D2FF08B010BD9810022010B5044683
:10D88000FFF78CFF002812DABDE8104001234FF0AB
:10D8900000020A4963F30202094B6FF3C5025B1AE7
:10D8A000DB0863F38F1207490748F5F729BD2046C7
:10D8B000BDE810406FF07001FFF7BEBFE44E0600F8
:10D8C0005C4F060090710600AF710600C36B70B527
:10D8D00013F0120F05460E461BD0FFF75FFF041E24
:10D8E00012DA01234FF000020B4963F302020B4BE3
:10D8F0006FF3C5025B1ADB0863F38F12084909480E
:10D90000F5F7FEFC204670BD31462846FFF794FF30
:10D91000F8E76FF00C04F5E7E44E06005C4F0600F4
:10D920009D710600AF71060038B5C36B044643F025
:10D930000803C363FFF71AFFE36B054623F00803F0
:10D94000E36338B101462046FFF7C0FF6FF00405DE
:10D95000284638BD04F036F8A063F9E710B5002476
:10D96000084802F0BDFEFFF733FF074B4FF400629B
:10D970001C6006490223064802F016FDFFF716FF59
:10D98000204610BD843A0220981002209C100220EC
:10D99000983A022037B5044610B3FFF719FF582212
:10D9A0000021204606F0B0F80423002584F8543006
:10D9B00002232A4684F8553001A90A4802F006FDE0
:10D9C000A842A8BF019D0022256401A9054802F0D4
:10D9D000FDFC0028B4BF0023019B6364FFF7E6FE53
:10D9E00003B030BD983A022073B50446002845D0F4
:10D9F000C36C002B42D0FFF7EBFE224B1A681E4689
:10DA00004AB12046FFF7ECFE6FF00B05FFF7CEFEA4
:10DA1000284602B070BD1C60236C002BF1D0636CF3
:10DA2000002BEED02046FFF799FEF8B9E36B01AA70
:10DA300043F00203E36369462046FFF71FFB90B9FA
:10DA4000DDE90012E36B204643F00803E363FFF7D0
:10DA50008DFEE36B054623F00803E36318B903F07A
:10DA6000B1FFA063D2E72046FFF708FF2046FFF78B
:10DA7000B7FE00236FF06E053360C7E76FF0150542
:10DA8000C6E700BF9810022073B50E460546D0B118
:10DA9000C9B1FFF79DFEE86BFFF78EFE044668B93B
:10DAA00001AB6A4631462846FFF794FB044628B985
:10DAB000DDE900122846FFF737FF0446FFF776FE40
:10DAC000204602B070BD6FF01504F9E773B50E463D
:10DAD0000546D0B1C9B1FFF77BFEE86BFFF76CFEDE
:10DAE000044668B901AB6A4631462846FFF7D5FBC4
:10DAF000044628B9DDE900122846FFF715FF044661
:10DB0000FFF754FE204602B070BD6FF01504F9E730
:10DB100037B50546D8B1FFF75BFEE86BFFF74CFE63
:10DB2000044678B901AA69462846FFF7C3FB0446B4
:10DB300040B9DDE900122846FFF7F6FE044608B9B1
:10DB40001023EB63FFF732FE204603B030BD6FF0C9
:10DB50001504F9E773B50E460546D0B1C9B1FFF714
:10DB600037FEE86BFFF728FE044668B901AB6A464A
:10DB700031462846FFF7A6FB044628B9DDE9001226
:10DB80002846FFF7D1FE0446FFF710FE204602B0FC
:10DB900070BD6FF01504F9E773B50E460546D0B1B8
:10DBA000C9B1FFF715FEE86BFFF706FE044668B93A
:10DBB00001AB6A4631462846FFF7D5FB044628B933
:10DBC000DDE900122846FFF7AFFE0446FFF7EEFD41
:10DBD000204602B070BD6FF01504F9E737B5054671
:10DBE000C0B1FFF7F5FDE86BFFF7E6FD044660B94D
:10DBF00001AA69462846FFF7F3FB044628B9DDE988
:10DC000000122846FFF790FE0446FFF7CFFD20469E
:10DC100003B030BD6FF01504F9E7000038B5FFF729
:10DC2000D7FD0D4B1C6834B1E36BDB0607D5002133
:10DC30002046FFF74BFEFFF7B9FD002038BDA56B6E
:10DC400003F0C0FE054B5B1B1844054B9842F2D80D
:10DC50002046FFF7C3FFEEE798100220402BFEFF9F
:10DC60003F2BFE7F73B50446002849D0FFF7B0FD77
:10DC7000E36B13F0100605D000212046FFF726FEC7
:10DC8000054614E09B0738D5A36C02AAC3F50061D2
:10DC900042F8041D616C20461944FFF773FD051E10
:10DCA0000ADA15F10B0F26D02046FFF7E7FDFFF744
:10DCB0007DFD284602B070BD01990029DDD0A26C1F
:10DCC00020460A44A264616CFFF792FBA26C0146F5
:10DCD000904207D96FF004012046FFF7F7FD6FF07F
:10DCE0000405E4E7121AA264002AE0D0606C014443
:10DCF00005F0A8FEDBE73546D9E76FF00C05D6E75F
:10DD00006FF01505D5E700000E4B10B51B684BB939
:10DD10000D4821230D4A0E49F5F708F80D48F5F78F
:10DD200005F8FEE75B684BB907482223074A0A4912
:10DD3000F4F7FCFF0748F4F7F9FFFEE7BDE81040F1
:10DD4000184700BF7C3A0220D9520600BB7006007B
:10DD5000F6700600F75206000171060013B5104C6C
:10DD600024684CB90F4857230F4A1049F4F7DEFFD7
:10DD70000F48F4F7DBFFFEE7E4694CB90948582384
:10DD8000094A0C49F4F7D2FF0948F4F7CFFFFEE740
:10DD9000009313460A464FF48D71A04702B010BDA0
:10DDA0007C3A0220D9520600BB700600F6700600CD
:10DDB000F7520600DC7106002DE9F041414D076A7B
:10DDC0002B68044638884BB93F4819233F4A4049DD
:10DDD000F4F7ACFF3F48F4F7A9FFFEE71B684BB927
:10DDE00039481A23394A3C49F4F7A0FF3948F4F777
:10DDF0009DFFFEE74FF48172012198470028606083
:10DE000005DAF6F7FDFE00684042BDE8F081042324
:10DE100004F108020521FFF7A1FF002803DA60687A
:10DE2000FFF772FFEDE72269A2B9A269EAB9E669D4
:10DE300036BB3B88022B2B680CBF082218226BBB19
:10DE400021484523214A2249F4F770FF2148F4F77D
:10DE50006DFFFEE7E368002BE7D09B0003216068BD
:10DE6000FFF77CFF0028E0DAD9E76369002BDED0FA
:10DE70009B0001216068FFF771FF0028D7DACEE729
:10DE80003046D4F8048005F0E5FF3246034602210F
:10DE90004046FFF763FF0028CBDAC0E75B694BB968
:10DEA00009484623094A0D49F4F740FF0948F4F7A9
:10DEB0003DFFFEE7216A606898470028AFDB00203D
:10DEC000A3E700BF7C3A0220D9520600BB700600CF
:10DED000F6700600F7520600137106002671060060
:10DEE0002DE9F8430746884615460024DFF8709070
:10DEF000AC4201D3002024E0D9F80030786808EB68
:10DF000004012A1B4BB911487E23114A1149F4F729
:10DF10000DFF1148F4F70AFFFEE7DE6A4EB90B4821
:10DF20007F230B4A0D49F4F701FF0B48F4F7FEFE7F
:10DF3000FEE70023B047002805DAF6F761FE006827
:10DF40004042BDE8F8830444D2E700BFD95206003E
:10DF5000BB700600F6700600F75206004B71060013
:10DF60007C3A022038B5144B14461B68406812688E
:10DF70004BB912486923124A1249F4F7D7FE1248E6
:10DF8000F4F7D4FEFEE75D6A4DB90C486A230C4AEB
:10DF90000E49F4F7CBFE0C48F4F7C8FEFEE7402329
:10DFA000A847002804DAF6F72BFE0068404238BD87
:10DFB00020600020FBE700BF7C3A0220D952060017
:10DFC000BB700600F6700600F75206003A710600B4
:10DFD00008B54068FFF798FE002804DAF6F710FE4F
:10DFE0000068404208BD0020FCE70000044B1870A8
:10DFF000044B1B6813B109B108461847704700BFAE
:10E000009C200220A020022038B50D4C0546237824
:10E0100083B903688BB100F0FDFF50B900F05BF9E4
:10E0200038B901F041F920B9064B2A681A6001237A
:10E03000237038BD6FF00C00FBE76FF01500F8E7B8
:10E040009C200220A0200220044B1B78012B01D829
:10E0500001F0F2B96FF00C00704700BF9C20022065
:10E060001FB50446F0B1124B1B78072B1DD81022A8
:10E070000021684605F048FD42F24B53029301230C
:10E08000204669468DF80C3000F02AF9044630B974
:10E09000684601F063FA0446019802F0C6FA204689
:10E0A00004B010BD6FF01504F9E76FF00C04F6E74B
:10E0B0009C2002207FB50B4B1B780C2B0FD8142211
:10E0C000002101A805F020FD05230C2001A98DF8F1
:10E0D0000430FFF78BFF002007B05DF804FB6FF002
:10E0E0000C00F9E79C20022030B50F4B85B01B785F
:10E0F00005460C2B11D898B101A900F0D1F90446BE
:10E1000040B9EB6801A8039301F0DEFA04460298D7
:10E1100002F08BFA204605B030BD6FF00C04F9E731
:10E120006FF01504F6E700BF9C20022030B50F4BBE
:10E1300085B01B7805460C2B11D898B101A900F0C9
:10E14000AFF9044640B9EB6801A8039301F0BFFAA8
:10E150000446029802F069FA204605B030BD6FF01F
:10E160000C04F9E76FF01504F6E700BF9C200220CD
:10E17000014B197800F050BF9C20022001F0C6BA74
:10E1800070B50C4601210646D0E900054008084458
:10E1900002F056FA78BBBDE8704001234FF0000250
:10E1A000164963F30202164B60F3C5025B1ADB08E3
:10E1B00063F38F1213491448F5F7A2B815F813202A
:10E1C000294449781201D2B201F00F010A4440F803
:10E1D00023200133326859008A42EFD8D10707D58E
:10E1E000154415F8012C1201D2B240F82320013356
:10E1F000C4E9003070BD0023ECE700BFE44E060028
:10E20000D44F06000F7206004A72060038B543EC80
:10E21000102B04460D46FDF7FEFC024628B12046B1
:10E220002946FDF7D9FC002038BD6FF00B00FBE755
:10E2300038B5044610460D46FDF702FD024628B1EA
:10E2400020462946FDF7C8FC002038BD6FF00B00C2
:10E25000FBE708B1FDF7A7BC704738B5054608468F
:10E260000C4605F0F7FD21460246284605F020FE43
:10E27000B0FA80F0400938BD38B504460D46FDF7C8
:10E28000C3FC024628B120462946FDF7A5FC002024
:10E2900038BD6FF00B00FBE738B50D46044610B1F2
:10E2A000C368042B04D000236FF001006B6038BDFD
:10E2B000006905F0CFFD2860013002F0BBF968600D
:10E2C00030B12A682169013205F038FE0020EEE7FE
:10E2D0006FF00B00EBE708B5FDF7F2FC002008BD7E
:10E2E0002DE9F04F85B0009148B95C48A6235C4AFF
:10E2F0005C49F4F71BFD5C48F4F718FDFEE7009B52
:10E300004BB95648A723564A5849F4F70FFD5648CB
:10E31000F4F70CFDFEE7002310F8042BCDE90233DF
:10E32000534B02A953F832300193FFF729FFFDF751
:10E330009CFC0646FDF799FC8246FDF796FC81465B
:10E34000FDF793FC8046FDF790FC0546FDF78DFC3C
:10E350000746DDE90210FDF78FFC83465EB1BAF196
:10E36000000F08D0B9F1000F05D0B8F1000F02D0AE
:10E370000DB107B1E8B93046FDF7B6FB5046FDF7E1
:10E38000B3FB4846FDF7B0FB4046FDF7ADFB284622
:10E39000FDF7AAFB3846FDF7A7FB5846FDF7A4FB9F
:10E3A000039802F042F96FF00B04204605B0BDE877
:10E3B000F08F304B002230492846FFF727FF019AA3
:10E3C00004462E492846FFF733FF04440298F1F72C
:10E3D000FBFF0B4602462A492846FFF717FF294A4A
:10E3E000044429494046FFF723FF2A4604442749AD
:10E3F0004046FDF7F1FB019A20493846FFF718FF28
:10E400005A46234904443846FDF7E6FB4246214973
:10E410004846FDF7E1FB3A461F494846FDF7DCFB5D
:10E420004A461E495046FDF7D7FB3046524616492C
:10E43000FDF7D2FB3046002C9ED1FDF7AFFB054621
:10E44000039802F0F2F83046FDF74EFB009B284699
:10E450005D6005F0FFFC009B1860A6E7D95206003E
:10E46000A8730600F2730600F75206000774060050
:10E47000947406000000F03F1D7406002774060027
:10E480002E7406003574060042740600B755060067
:10E49000487406005074060058740600667406003E
:10E4A000F8B50F46064648B92C48F2232C4A2D49A8
:10E4B000F4F73CFC2C48F4F739FCFEE783684BB9D1
:10E4C0002648F323264A2949F4F730FC2648F4F776
:10E4D0002DFCFEE743684BB92048F423204A244929
:10E4E000F4F724FC2048F4F721FCFEE749B91B4867
:10E4F000F5231B4A1F49F4F719FC1B48F4F716FCD7
:10E50000FEE7FDF7B2FB0546B8B11B4B32781B495D
:10E5100053F82220FFF78CFEB268044618492846BB
:10E52000FFF786FE174A044417492846FFF780FE86
:10E530002418284604D0FDF7D7FA6FF00B040AE040
:10E54000FDF72CFB06462846FDF7CEFA7E603046E6
:10E5500005F080FC38602046F8BD00BFD9520600A7
:10E56000A873060023730600F752060039730600ED
:10E570005973060007740600707406006F73060076
:10E5800035560600757306007A73060070B50546A9
:10E590000C4651B945484FF48A73454A4549F4F74A
:10E5A000C5FB4548F4F7C2FBFEE750B93F4840F2CF
:10E5B00015133F4A4149F4F7B9FB3F48F4F7B6FB5E
:10E5C000FEE7406850B939484FF48B73384A3C49EC
:10E5D000F4F7ACFB3848F4F7A9FBFEE72B6853B916
:10E5E000324840F21713324A3649F4F79FFB32485B
:10E5F000F4F79CFBFEE7FDF7CDFA0646A0B9012231
:10E600004FF00003304962F30203304A60F3C50360
:10E61000521AD20862F38F132D496A682D48F4F715
:10E6200083FE6FF0010070BD2B49FFF712FE2B49EE
:10E630000546FFF70EFE2A49002808BF2846FFF7C7
:10E6400008FE2549FFF705FE10B1C368042B03D06F
:10E650003046FDF749FAE4E7056922492846FFF705
:10E66000FCFD30B1062323703046FDF73DFA002053
:10E67000D9E71D492846FFF7F0FD08B10723F2E767
:10E680001A492846FFF7E9FD08B10823EBE71849C6
:10E690002846FFF7E2FD08B10923E4E715492846BB
:10E6A000FFF7DBFD0028DFD00A23DCE7D9520600A4
:10E6B000A873060096720600F7520600F273060071
:10E6C000B5720600CF720600E44E0600D44F060075
:10E6D00029720600DF72060042740600FA72060014
:10E6E0005074060002730600357406000B730600B2
:10E6F000386B06001C7306002DE9F04F044685B008
:10E70000894651B97B4840F24B137B4A7B49F4F769
:10E710000DFB7B48F4F70AFBFEE7FDF7A6FA074678
:10E72000FDF7A3FA8046FDF7A0FA0646FDF79DFA2D
:10E73000054627B1B8F1000F01D006B150B93846EF
:10E74000FDF7D2F94046FDF7CFF93046FDF7CCF999
:10E7500028465AE0A01F042800F2B980DFE800F044
:10E76000033A81B78800674A67493046FFF760FD82
:10E77000664A044666492846FFF75AFD654904443F
:10E780002846FFF779FD644904442846FFF774FDE5
:10E7900004442A4661493046FDF71EFA3246604974
:10E7A0004046FDF719FA384642465949FDF714FA32
:10E7B0003846002CC4D1FDF7F1F905463846FDF77F
:10E7C00093F925B3C9F80450284605F043FBC9F86E
:10E7D00000008AE0FDF749FA82465248FDF730FA18
:10E7E0008346BAF1000F00D0A0B93846FDF77CF996
:10E7F0004046FDF779F93046FDF776F92846FDF7F2
:10E8000073F95046FDF770F95846FDF76DF96FF052
:10E810000B046AE0444B002244495046FFF7F6FCE3
:10E820005A46044642495046FDF7D6F90022414B6C
:10E8300041495046FFF7EAFC404A0444344928461F
:10E84000FFF7F6FC5246044432492846FDF7C4F966
:10E85000002C9ED05046FDF747F95846FDF744F985
:10E8600097E7374A2A492846FFF7E2FC044690E733
:10E87000344A27492846FFF7DBFC26490446284648
:10E88000FFF7FAFC304904443046FFF7F5FC6946CF
:10E89000044402A800F0EEFEFDF7E7F982460028E6
:10E8A0003FF44DAF039A2949FFF7C2FC019A044493
:10E8B00027495046FFF7BCFC5246044416492846F7
:10E8C000FDF78AF9002C3FF464AF5046C6E738469E
:10E8D000FDF70AF94046FDF707F93046FDF704F960
:10E8E0002846FDF701F96FF08504204605B0BDE824
:10E8F000F08F00BFD9520600A87306000774060007
:10E90000F7520600867306008B730600027306003A
:10E9100042740600B7550600917306005074060055
:10E9200066740600987306000000F03F1D74060030
:10E9300027740600000018402E7406003574060087
:10E940000B7306001C73060058740600A0730600C3
:10E95000A47306002DE9F04103468846174650B9D6
:10E9600040484FF4EF73404A4049F4F7DFF940481C
:10E97000F4F7DCF9FEE7406850B93A4840F2DF139B
:10E98000394A3C49F4F7D2F93948F4F7CFF9FEE7B0
:10E990001B6853B933484FF4F073334A3649F4F7E0
:10E9A000C5F93348F4F7C2F9FEE751B92D4840F2F2
:10E9B000E1132D4A3149F4F7B9F92D48F4F7B6F9C6
:10E9C000FEE752B927484FF4F173274A2C49F4F770
:10E9D000ADF92748F4F7AAF9FEE7FDF7DBF805469D
:10E9E000F0B12849FFF735FC27490446FFF731FC11
:10E9F0002649002808BF2046FFF72BFC2149064680
:10EA0000FFF727FC224904463046FFF722FC064662
:10EA10001CB110B1E368042B05D02846FDF764F85B
:10EA20006FF0010411E01B492069FFF716FC002874
:10EA3000F3D019493046FFF70CFC4146FFF72CFC98
:10EA4000044628B12846FDF74FF82046BDE8F0817E
:10EA500012493046FFF7FDFB3946FFF71DFC04461F
:10EA6000F0E700BFD9520600A8730600F273060053
:10EA7000F7520600B5720600CF72060060720600FB
:10EA80007B72060042740600FA720600507406009B
:10EA9000917306001C730600A0730600A4730600A1
